S0220000687474703A2F2F737265636F72642E736F75726365666F7267652E6E65742F1D
S22401000028280820F5F9010017FA010019FA01001BFA01001DFA01001FFA01000000000005
S2240100200000000000000000000000006903010023FA010000000000E10301001D04010028
S22401004029FA010029FA010029FA010029FA010029FA010029FA010029FA010029FA01007A
S22401006029FA010029FA010029FA010029FA010029FA010029FA010029FA010029FA01005A
S22401008029FA010029FA010029FA010029FA010029FA010029FA010029FA010029FA01003A
S2240100A029FA010029FA010029FA010029FA010029FA010029FA010029FA010029FA01001A
S2240100C029FA010029FA010029FA010000F002F800F05EF80AA090E8000C82448344AAF128
S2240100E00107DA4501D100F053F8AFF2090EBAE80F0013F0010F18BFFB1A43F001031847C8
S224010100A83B0100E83B01000A444FF0000C10F8013B13F0070408BF10F8014B1D1108BFD6
S22401012010F8015B641E05D010F8016B641E01F8016BF9D113F0080F1EBF10F8014BAD1CC5
S2240101400C1B09D16D1E58BF01F801CBFAD505E014F8016B01F8016B6D1EF9D59142D6D3CB
S224010160704700000023002400250026103A28BF78C1FBD8520728BF30C148BF0B60704799
S2240101801FB59DE803000FF082FF1FBD10B510BD10F039F81146FFF7F3FF0FB400F00CF8E8
S2240101A00FBC00F05BF80FF09EFE03B4FFF7EEFF03BC10F021F8000004B010F00BFE044815
S2240101C0002110F0DFFE10F017FE0FF08CFE0000D43A020070B50546304981F82C54304813
S2240101E0407820F0F00040302D4948700846407820F00F00C01C4870052008700C2D28D21A
S224010200DFE805F027060E120A161A1E27271F2301F0D0FD04461CE002F008FF044618E0A8
S22401022003F088FD044614E003F07FFB044610E002F091FF04460CE002F05BFF044608E025
S22401024007E003F0BBF8044603E004F0CEF8044600BF00BF204601F0AFFD70BD70B5114CAA
S22401026010F0B8FD0220FFF7B5FF01F0A8FDC56E284600F061FC01F0A2FDD0F888502846D5
S22401028000F05DFC204600F011FC02F054F800F03FF910F0B1FD002070BD000044C9072017
S2240102A0000200100100000270B50446B4F5E02F00D070BD4FF480620D490E480FF048FEE9
S2240102C00D490B482C38C1634FF4E22572B62946204601F0F3F900B1EBE74FF480620549CD
S2240102E0204601F046FA00B1E3E762B600BFE0E770C9072060040010AA5555AAFFFFFFFF7A
S22401030080F309887047EFF309807047684680F3098804480078C00714BF0220032080F332
S22401032014887047943A0200DFF818C0EFF305831B0618BF6047EFF31483DB0708BF604713
S22401034000DF7047C5100200DFF818C0EFF305831B0618BF6047EFF31483DB0708BF6047A9
S22401036000DF70475D130200EFF30980816911F8021CF1B990E80F10E047EFF3098C8CE8A0
S2240103800700144B93E8060091420FD039B12CE9F00FC1F828C00CB411F0D0FB0CBC1A6051
S2240103A0D2F828C0BCE8F00F8CF309886FF0020E704710B5084A1268914209D8074C54F8C8
S2240103C0214090E80F10A047EFF3098C8CE80F0010BD0000D8C80720EC020200EC020200CA
S2240103E011F07EFA0C4B93E80600914210D0EFF3098C2CE9F00FC1F828C00CB411F09EFB6D
S2240104000CBC1A60D2F828C0BCE8F00F8CF309886FF0020E70470000D8C8072011F056FCEF
S224010420E0E7000010F03AFE11F050FCDAE700002DE9F041054632274FF001086C49086851
S22401044010F0F6FD6A49486810F0F2FD6849886810F0EEFD002607E06648815D01220020E9
S2240104600FF0F1F9701CC6B2022EF5DB35B132274FF0020801206049087002E000205E4916
S2240104800870632F00DD6327B8F1000F01D14FF001085A4805700020594908704FF47A7095
S2240104A090FBF8F084B204FB07F0642190FBF1F05449088008460088201A534908805148B4
S2240104C0008810B901204F4908804E4A1288A11A474A106810F0A0FDBDE8F08108B50020FE
S2240104E003460246082100900FF0E6F9002003460246092100900FF0DFF901220821002020
S2240105000FF087F90122092100200FF082F908BD10B5FFF7E3FF002211463C4810F066FDAD
S2240105203349086000221146394810F05FFD3049486000221146374810F058FD2C498860B0
S2240105400020FFF775FF10BD10B504462C480078401C2B4908702748274A1278815C002292
S22401056010460FF070F9224948682649098810F053FD10BD10B504461E481F4A1278815C3A
S224010580012200200FF05FF91C48007898B11C4800781A49097888420DDB1549086810F056
S2240105A047FD134988684FF47A7110F035FD00201349087005E00E4908681349098810F0B8
S2240105C02BFD10BD10B504460D480078401C0C4908700848084A1278815C002210460FF09B
S2240105E032F9034948680749098810F015FD10BD38C90720080200100A0200100C02001092
S2240106000B0200100E02001010020010EC370200F4370200FC37020010B50446022C00D0E1
S22401062010BD4FF4E020FFF73FFE00BFF8E72DE9F0410746884600243BE004EB8400FE4978
S22401064031F82000B84232D104EB840001EB8000407A012801D1BDE8F08104EB8400F649F2
S22401066001EB8006307A07280FD2DFE800F004070A05080B0C0000BF012506E000BF0225A7
S22401068003E000BF00BF042500BF00BF2A46414670680FF05DFC04EB8400E74901EB800016
S2240106A0807AE64909780843E4490870D3E7601CC4B2E34800888442BFDB00BFCBE738B57D
S2240106C00546002417E004EB8400DB4931F82000A8420ED1DB48006850B169462846D94A39
S2240106E012689047012803D128460099FFF79FFF00BF601CC4B2D24800888442E3DB38BD3F
S22401070070B5002408E1002504EB8400CA4901EB8000007A072823D2DFE800F0042342616B
S22401072084A7C60004EB8400C34901EB80004068007804EB8401C04A02EB8101097B88427C
S2240107400DDB04EB8400114601EB80004068017804EB840002EB8000007C814200DD012532
S224010760CFE004EB8400B44901EB80004068008804EB8401B04A02EB8101898988420DDB17
S22401078004EB8400114601EB80004068018804EB840002EB8000008A814200DD0125B0E02C
S2240107A004EB8400A44901EB80004068006804EB8401A14A02EB8101C96888420DD304EBBF
S2240107C08400114601EB80004068016804EB840002EB80000069814200D9012591E004EB50
S2240107E08400954901EB8000406890F9000004EB8401914A02EB810191F90C1088420FDBDC
S22401080004EB8400114601EB8000406890F9001004EB840002EB800090F91000814200DD42
S22401082001256EE004EB8400834901EB80004068B0F9000004EB84017F4A02EB8101B1F9EC
S2240108400C1088420FDB04EB8400114601EB80004068B0F9001004EB840002EB8000B0F9A2
S2240108601000814200DD01254BE004EB8400724901EB80004068006804EB84016E4A02EBAE
S2240108808101C96888420DDB04EB8400114601EB80004068016804EB840002EB800000695D
S2240108A0814200DD01252CE004EB8401624A02EB81014968086820F00041C1F1FF41C90F95
S2240108C0E9B904EB84025C4B03EB8202D16804EB840203EB82025268106812F05DFD0ED353
S2240108E004EB8402544B03EB8202116904EB840203EB82025268106812F04EFE00D2012593
S22401090000BF00BF35B104EB84014B4A32F82100FFF7D5FE601CC4B2494800888442FFF68A
S224010920F2AE70BD38B5002469E004EB8400424931F8200040F23F11884248D004EB84006C
S2240109403D4931F82000B0F5A07F40D004EB840031F8200040F24111884238D004EB840069
S224010960354931F82000B0F5A17F30D004EB840031F8200040F24311884228D004EB84006E
S2240109802D4931F8200040F25F1188421FD004EB8400294931F82000B0F5B07F17D004EB5F
S2240109A0840031F8200040F2611188420FD004EB8400214931F82000B0F5B17F07D004EB56
S2240109C0840031F8200040F26311884215D11D48006890B104EB8401174A32F82100694611
S2240109E0184A12689047012807D104EB8401124A32F821000099FFF71AFE601CC4B2104831
S224010A000088844291DB38BD38B5002420E00D480068D8B104EB8401074A32F8210069460B
S224010A20084A12689047012810D104EB8401024A32F82100009907E000C00720C8C70720DB
S224010A40BCC70720C0C70720FFF7F1FD601CC4B2FE4800888442DADB38BD10B54FF44031AB
S224010A60086880F3098800BF08460CF061FD4FF440304468A04710BD70B54FF4F0244FF4C3
S224010A80E0252C222146F2480FF0A7FA4FF480622946EF482C300FF0A0FAED48C06BED4966
S224010AA0884201D0002070BD0120FCE710B50446FFF7E2FF38B9FFF7A7FFE548C0F8284282
S224010AC00220FFF7A9FDE24890F82C02012801D1FFF7C3FFDE48D0F82802A04219D0DC48B8
S224010AE0D0F828020016B0EB246F02D0FFF78CFF07E0D948006810B1D74800688047FFF7F2
S224010B0011FFD348C0F828420220FFF785FD09F051FACF48006BD1490968884208D0CF48DE
S224010B200168CB480163FFF7EBFD0220FFF774FD0220CB49087010BDCA4908607047C649AC
S224010B40086070472DE9FE43074688461646ADF8006003208DF804008DF802708DF80380F2
S224010B600020CDF80600002530E005EB8500BE4931F82000B04227D105EB850001EB8009B6
S224010B8099F808008DF805009DF8050007280FD2DFE800F004070A05080B0C0000BF0124AE
S224010BA006E000BF022403E000BF00BF042400BF00BFC4F104030DF1060298182246D9F8B2
S224010BC004100FF0C5F905E0681CC5B29F4800888542CADB00BF9DE8070006F084FDBDE81C
S224010BE0FE8310B50220FFF717FD10BD2DE9F0478046894616461D466878C0F3C207072F7D
S224010C000FD2DFE807F004070A05080B0C0000BF012406E000BF022403E000BF00BF0424BE
S224010C2000BF00BFC4F1080041193046FFF7FFFCFFF7D7FF324649464046FFF783FFBDE83C
S224010C40F08770B505460E4600240AE004EB8400854931F8202031462846FFF773FF601CD2
S224010C60C4B27A4800888442F0DB70BDF8B506460F461446607800F00705284609F088F98C
S224010C80012800D0F8BD60880090284609F059F9012800D0F6E7012D1FD0022D2FD0052D1C
S224010CA035D1BDF800004FF6FF21884208D1FFF7ABFEFFF796FF39463046FFF7C2FF0BE0AA
S224010CC0BDF80000FFF7FBFCFFF78BFFBDF8002039463046FFF736FF1AE0BDF800004FF603
S224010CE0FF21884204D139463046FFF7AAFF05E0BDF8002039463046FFF724FF08E0234682
S224010D00BDF8002039463046FFF770FF00E000BF00BF00BFB6E75248007800F0040038B1F5
S224010D204F48007820F004004D490870042070474B48007800F0020038B14948007820F0A2
S224010D400200474908700220F1E70120EFE710B504463F484463FFF744FF10BD3C4890F843
S224010D60340070473A4890F8A800032806DB384890F8A800182801DC012070470020FCE71C
S224010D80334890F8A8001B2813D0314890F8A8001E280ED02E4890F82C0401280BD12C4808
S224010DA090F8A800032806DB294890F8A800172801DC012070470020FCE701460B291DD2EF
S224010DC0DFE801F006080A0C0E10121416181A00062013E0012011E002200FE006200DE056
S224010DE000200BE0012009E0062007E0032005E0062003E0062001E0062000BF00BF704758
S224010E002DE9F04105460F462C461148E1688166E06841420E48C166217C80F8E510617CBB
S224010E2080F88310618BA0F87A10E18AA0F85010618AA0F84C10A18AA0F84E10207812F096
S224010E4097FA8046094912F07DF911E0BCC7072044C90720AA5555AAC4C7072000020010DA
S224010E60C8C70720C0C7072000C00720ACC52737064612F045FAF749C865607812F078FA0C
S224010E808046F54912F05EF9064612F039FAF1490866A07812F06CFA8046EF4912F052F9FB
S224010EA0064612F02DFAEB494866E07812F060FAE849C1F8A000B4F90400002801DB01469B
S224010EC000E041428AB2E349A1F84220B4F90800002801DB014600E041428AB2DD49A1F8E8
S224010EE04620B4F90600002801DB014600E041428AB2D849A1F84420B4F90A00002801DB10
S224010F00014600E041428AB2D249A1F84820B4F90400002801DD012100E00021CD4880F862
S224010F204A10207EFFF749FFCA4981F87900FFF758FE09F03FF8BDE8F081C64890F82C021A
S224010F40704710B50446C34880F82C420220FFF763FB09F02FF810BDF0B585B006460F46F6
S224010F6014461D469DF8030065F3C6008DF80300009864F31A200090B2208DF800000098C8
S224010F80CDF8090004208DF8080000231A46EF21062007F097FC019001AA3946304606F062
S224010FA09BFE05B0F0BD2DE9FF4105460E46144620680290606803909DF80B000321B1EB0C
S224010FC0D00F01D0BDE8FF810298C0F31220A34A811A904275D01ADCA14AA0EB02019042D7
S224010FE071D00BDC9F49084420B3B0F57F7F2ED0A0F2FD30F0B3012828D14FE001296DD001
S22401100003297ED0042975D00629F5D18FE0072971D008DC01296FD004296ED005296DD0E6
S2240110200629E9D1C5E0082969D09F2968D0A029E2D1E6E0039800900A21009890FBF1F016
S224011040009069464FF49E70FFF7F1FAE9E003980090009812F074F980467F4912F072F824
S224011060074612F031F90090694640F23F10FFF7DEFAD6E0FFE703980090009812F060F9A9
S2240110808046754912F05EF8074612F01DF9009069464FF4A070FFF7CAFAC2E003980090F0
S2240110A0009812F04DF980466B4912F04BF8074612F00AF90090694640F24110FFF7B7FAD0
S2240110C0AFE03CE0FFE7039800EB80004000019001A940F23310FFF7AAFAA2E0039800EBE1
S2240110E080004000019001A940F23510FFF79FFA97E006E010E08CE029E030E044E06DE0A6
S22401110074E0039800EB80004000019001A94FF49A70FFF78CFA84E0039800EB8000400081
S224011120019001A94FF49B70FFF781FA79E00398009069464FF4B270FFF779FA71E00398C2
S224011140019001A94FF4A170FFF771FA69E00398019001A940F24310FFF769FA61E00398C0
S22401116000904FF6FF71009888420CD13E48817A807B00F0030041EA0020009069464FF4A9
S2240111809C70FFF754FA4CE0039800904FF6FF71009888420CD13448817A807B00F0030049
S2240111A041EA0020009069464FF49D70FFF73FFA37E0039800904FF6FF71009888420CD1EA
S2240111C02948817A807B00F0030041EA00200090694640F23910FFF72AFA22E00398009063
S2240111E069464FF4AC70FFF722FA1AE00399C8B2FFF7E3FD009069464FF4A870FFF717FA42
S2240112000FE003980090694640F25110FFF70FFA07E00398009069464FF4AC70FFF707FA56
S22401122000BF00BFFFF7DDFC0298C0F31222002331462846FFF790FE00BFC3E6014607296F
S22401124020D2DFE801F004131517191B1D00042018E0000044C90720ACC527370EFE070018
S22401126003FE0700FC05F8FF38C80720052009E0022007E0072005E0002003E0002001E01A
S224011280002000BF00BF70472DE9F04186B00746884615462E463068C0F31220BC4A811A6E
S2240112A090421ED010DCBB4AA0EB0201904231D005DCB9490844E8B101284CD122E00129DC
S2240112C030D00C2947D108E001290ED01E293ED09A292FD09B293ED134E0B048C06C019018
S2240112E03CE0AE48006D019038E0AC48D0F84E00019033E0A948B0F842000A2190FBF1F49C
S22401130001942BE0A548B0F846000A2190FBF1F4019423E0A148B0F844000A2190FBF1F4A9
S22401132001941BE09D48B0F848000A2190FBF1F4019413E0994991F87900FFF77FFF04467D
S22401134001940BE09548B0F87A40019406E09348046B019402E006B0BDE8F08100BF9DF86C
S224011360030020F0F80018308DF80300B4208DF800003068010A009861F31A200090009842
S224011380CDF80D000198CDF8110008208DF80C0000231A46EF21062007F094FA029002AAD1
S2240113A04146384606F098FC00BFD4E72DE9FE4F07468A4616464FF00008306801907068FA
S2240113C00290DDF80500000AA0F57F40A03800287ED1BDF8090003287BD14FF026089DF8B7
S2240113E009006F4908706D49C86D11F0C1FF83466C4912F005F8814611F082FF68494870D3
S2240114006649086E11F0B4FF8346664911F0F8FF814611F075FF624988706049486E11F03E
S224011420A7FF83465F4911F0EBFF814611F068FF5B49C8705948B0F842400C71200A48716E
S2240114405648B0F846408C71200AC871002008725248B0F844404C72200A88724F48B0F8D9
S2240114604840CC72200A0873002048734B48856E8D73280AC873280C0874280E48744749FB
S224011480D1F8A00011F03CFF45498874434890F8E500C8744148B0F84E10002009F0BFFE7E
S2240114A005463F490D75280A4875280C8875280EC8753A48B0F84C10002009F0B0FE0546A6
S2240114C037490D76280A4876280C8876280E01E02BE027E0C876314890F8790008772F480A
S2240114E0B0F87A404C77200A88772C4890F88300C8772A48B0F84C4081F82040200A81F8B8
S22401150021002648B0F84E4081F82240200A81F823002248B0F8504081F82440200A81F83D
S224011520250000E000BF00BF00BF00BF384606F025FB814600204B464FF6A072414600902A
S224011540174807F0AAFFBDE8FE8F10B50446FFF7F4FC60B1608840F23D11B1EB501F06D104
S2240115606079172803D10020FFF7EBFC0EE0FFF7E4FC01280AD060889721B1EB501F05D134
S2240115806079802802D10120FFF7DBFC10BD000013FE070006FE0700FD01F8FF44C90720EA
S2240115A088CD0720ACC5273702460120704710B5834C84498448A04710BD83490860002184
S2240115C0814A51609160D16011617E4A116051609160704710B504463720FFF7EEFFFFF724
S2240115E0E6FF7848406820607648007810BD08B5002000906846FFF7EDFF08B9009808BDFA
S2240116004FF0FF30FBE710B504463620FFF7D5FFFFF7CDFF6B48406820606A48007810BDB1
S22401162008B5002000906846FFF7EDFF08B9009808BD4FF0FF30FBE7644800684FF47A71F7
S224011640B0FBF1F0704770B504460D46A54201DAFF2070BD3420FFF7B0FF5B48446085604C
S224011660FFF7EAFF5849C860FFF7A1FF55480078EFE770B504460D46A54201DAFF2070BD6B
S2240116803220FFF79AFF504844608560FFF78FFF4C480078F3E70146B1F5803F02D2C1F3A4
S2240116A007307047B1F5002F06D2A1F58030102202EBD030C0B2F4E7FF20F2E72DE9F04198
S2240116C006460C463046FFF7E6FF07462046FFF7E2FF804641463846FFF7CBFF054615B1EF
S2240116E02846BDE8F08141463846FFF7ACFF05462846F6E770B505460E461446E11704EB1F
S22401170091718910A4EB810109B1FF2070BD3820FFF753FF2C4845608660C460FFF747FF12
S22401172028480078F2E770B505460E461446B4F5807F0AD0B4F5007F07D0B4F5806F04D0D7
S224011740B4F5805F01D0FF2070BDE8B208B1FF20FAE73320FFF731FF1B4845608660C46000
S224011760FFF76AFF18490861FFF721FF15480078EAE72DE9F04705460F4616462846FFF7D1
S2240117808AFF8046A819FFF786FF814649464046FFF76FFF044614B12046BDE8F08732466F
S2240117A039462846FFF7BFFF04460CB12046F4E7324639462846FFF79DFF04462046ECE7C0
S2240117C0F11FFF1FC4CD0720B0CD07204C0400100146022901DB0020704701EB8100F94A44
S2240117E012F82000F8E770B50446F7480DF00FFB0546002120460DF041FA00F0C000F8B1C2
S2240118000122114620460DF08AFAA06840F07F40A060A06820F07F40A060012200212046E9
S2240118200DF07DFA0122114620460DF078FA082120460DF0E5FA0022012120460DF06FFA64
S22401184070BD70B5044672B620460DF0DDFA054662B670BD70B504460D46022C01DB002008
S22401186070BD04EB8400D74901EB80002946C26820469047F4E77FB50646D448864201D050
S224011880012000E000200546D14951F8250000210FF0F4FA04460CB3694630460DF053F9C9
S2240118A001281BD1009820600198C4F805000299C4F809109DF80C0020719DF80D00607384
S2240118C000208DF80E0021462846FFF7C3FF28B9BF4951F8250021460FF0F4FA7FBD7CB5AA
S2240118E0BC4903C9CDE90001002421E004EB8400B44911F82000D0B15DF824000DF084FA27
S224011900054605F0010018B15DF82400FFF7B3FF40F20260284018B15DF82400FFF791FFD2
S22401192005F0040018B15DF82400FFF75CFF641C022CDBDB7CBD02460020704770B50446EA
S224011940022C01DB002070BD0CB9A04800E0A2480546002004EB84019A4A02EB8101887089
S22401196004EB840102EB8101487004EB840102EB8101C870012004EB840102F8210097481C
S22401198004EB840102EB8101C860954919200BF0D3FD1920F021002807DACA06160E914A32
S2240119A000F00F031B1FD65403E0CA06130E8E4A135400BF8D4928460BF03CFE01221146F6
S2240119C028460DF0ACF90122002128460DF070F90122114628460DF06BF9012202212846DC
S2240119E00DF066F90122032128460DF061F90022012128460DF093F90122002128460DF08F
S224011A008EF9022170480DF074F9192000F0C6F8012098E710B50446022C01DB002010BD67
S224011A20192000F0C6F8002004EB8401654A02EB8101887004EB840102EB8101487004EB85
S224011A40840102EB8101C87004EB840102EB8101886004EB840102F82100604804EB8401DE
S224011A6002EB8101C8600120D9E710B50446192000F09FF8022C01DB002010BD192000F0F9
S224011A808DF80120F9E7022800DB704700EB80024C4B03EB8202D16000BFF6E7022800DBB6
S224011AA0704700EB8002474B03EB8202D16000BFF6E7022800DB7047484900EB8002414BE5
S224011AC003EB8202D16000BFF5E70146002070472DE9FF4105460C46022D03DB002004B0D0
S224011AE0BDE8F08101260DB9384800E03A4807462068009001208DF80D00D4F80500019081
S224011B00D4F80900029020798DF80C0000208DF80E00694638460CF03DFF012800D00026F7
S224011B203046DCE770B504460D46022C01DB002070BD04EB8400234901EB8000C07820B9F1
S224011B4029462046FFF7C4FFF2E70220F0E7022800DB7047002100EB80021A4B03EB8202FE
S224011B60917000EB800203EB8202517000EB800203EB8202D17000BFEBE710B50446022CD0
S224011B8000DB10BD002004EB84010E4A02EB810188602046FFF7DBFF00BFF2E700F01F0275
S224011BA0012191404209920002F1E022C2F80011704700F01F02012191400D4A430942F8F7
S224011BC023107047D4CD072000C00340004004404C03001004380200008004403719010014
S224011BE0DF18010018ED00E000E400E090D0030080E100E02DE9FE4306460C4606B114B921
S224011C000020BDE8FE83092001218140654A430942F8231000BF002507E000231A46294647
S224011C2061480DF026FB681CC5B2072DF5DB0C200DF03EF9804606FB04F1B8FBF1F70FB959
S224011C400020DEE700208DF80400029701AA002155480DF0E4F900232246194652480DF093
S224011C6008FB01208DF8010000208DF8000001208DF8030000208DF8020069464A480DF081
S224011C8041FA49480DF035FA002147480DF025FA002145480DF015FA0120B2E72DE9F041BF
S224011CA004460E4617460FB1032500E00225072C2FD2DFE804F02E040B12192027002B4625
S224011CC03246012138480DF0D4FA24E02B463246022135480DF0CDFA1DE02B4632460321BE
S224011CE031480DF0C6FA16E02B46324604212E480DF0BFFA0FE02B46324605212A480DF00B
S224011D00B8FA08E02B463246062127480DF0B1FA01E0BDE8F08100BF00BFFAE770B5044637
S224011D200D46072C24D2DFE804F02304050B11171D001EE0002202211B480DF0F5FA18E060
S224011D400022032118480DF0EFFA12E00022042115480DF0E9FA0CE00022052112480DF0F0
S224011D60E3FA06E0002206210F480DF0DDFA00E070BD00BF012229462046FFF78FFF0A488C
S224011D800DF0B7F90122214607480DF0EAFA012105480DF096F9012103480DF09EF900BF1B
S224011DA0E6E7000080E100E000800140FA480068C06E7047F9487047F74908607047F6482A
S224011DC0006870471CB5F4480068C06C0090F2480068C0680190684602F01CFC1CBD0020A1
S224011DE07047EF48407900F0030070472DE9F041EC49ED48006811F003FB064604F05EFED8
S224011E00074611F0B5FA0546314611F09BF9044611F076FA80B2BDE8F0812DE9F04198B0D6
S224011E200321052007F008FEDF4908600621042007F002FE0446DC48006811F0E9F8054681
S224011E402A460B460020D94910F09CFC074610F021FE81B20CA84182D3480168D44811F02A
S224011E6071F9054611F04CFA81B20CA88182FEF779FF00B3CF4890F8A80018280DD1CA48DF
S224011E800168CD4811F05EF9054611F039FA81B20CA84182C94913910FE0C3480168C64816
S224011EA011F050F9054611F02BFA81B20CA84182C349139101E0C1491391BB480168129169
S224011EC0139808B1012000E000208DF84000B648006811F09DF805462A460B460020B3498E
S224011EE010F050FC074610F0D5FD80B2ADF83200AD480168AE4811F025F9054611F000FAAF
S224011F0080B2ADF83400A4480068806A0F90A64800680E900F9808B1012000E000208DF8D9
S224011F20300001208DF85000204611F071F805462A460B460020A34910F024FC074610F020
S224011F40A9FD81B20CA84184204611F061F805462A460B4600209C4910F014FC074610F0FB
S224011F6099FD81B20CA881848B480068C16A17911694904890F8740018B1179808B10120FB
S224011F8000E000208DF850000CA802F0C5FCFEF7E9FE90B1874890F8A800182806D18B48F9
S224011FA009908B480A908B480B903DE08A4809908A480A908A480B9036E07E4890F8790069
S224011FC0072830D2DFE800F01A2821120B1904008448099084480A9084480B9023E0844875
S224011FE0099084480A9084480B901CE08348099083480A9083480B9015E000BF8248099033
S22401200082480A9082480B900DE08248099082480A9082480B9006E08148099081480A902D
S22401202081480B9000BF00BF09A802F080FC5A480068C06B029058480068006C03905D4826
S22401204090F8A800182802D17848019001E07848019051480068806C04904F480068806D47
S22401206005904D480068006D06904B480068406D079049480068C06C089001A802F05DFCD5
S22401208018B0BDE8F081002070471CB5002069490870484890F8A800022804D0454890F897
S2240120A0A800202803DB0021424880F8A810414890F8A8001B2836D00BDC18282DD003DC6C
S2240120C080B1012851D11FE0192817D01A284CD10EE01C282FD01D2833D01E2837D01F28EB
S2240120E043D13CE054482D49C8615448086245E053482A49C861534808623FE052482749DF
S224012100C8615248086239E051482449C8615148086201204749087030E04F481F49C861E0
S2240121204E4808622AE04A481C49C861494808624B48C86022E04B481849C8614A4808629E
S2240121401CE04A481549C8614948086216E03A481249C861394808624148C8600EE0454856
S2240121600E49C8614448086208E0FEF7FBFD20B142480A49C8614248086200BF00BF064877
S2240121800068C069009004480068006A0190684602F094F91CBD0000180200102402001003
S2240121A088030010000020411C020010000023400000F04144C9072000004040075401004B
S2240121C0ED1D0100000012400000164029BD01002BBD010031BD0100D1B90100E1B9010061
S2240121E0F5B901001DBD01001FBD010023BD01000DBC01006FBC010075BC010033BB01007A
S22401220075BB01007BBB01006568010079680100C168010019BA01002DBA010077BA010088
S22401222095BA0100A9BA0100F3BA0100E31D0100DF1D0100200200106FC00100CBC001004A
S22401224075C30100CFC30100F1BD010033BE0100B9BE01000BBF010051C2010063C201008E
S2240122608720010077C50100E9C5010047C70100A3C701007FC90100DBC9010075BF010027
S224012280C3BF010000B58FB0FE48006840680290FC48006880680190FA480068C06803904F
S2240122A0F848006800690490F648006880690690F448006840690590F2480068006E0790C5
S2240122C0F0480068406E0890EE480068806E0990EC480068406F0A90EA480068806F0B90E4
S2240122E0E8480068006F0C90E6480068D0F880000D90E448006890F884008DF83800FEF768
S2240123003FFD08B1E048039001A803F0FBFA0FB000BD10B5DB49096808688047FFF7B2FFC2
S224012320FFF7B3FEFFF779FDFFF74CFDD5490968C86D804710BD10B5D249096891F87C0097
S22401234007F0DAFDFFF7E5FF02F0C5F803F09BFA03F04EFF02F03EFF02F01AFA04F033FA02
S22401236009F098FA06F02EFD10BD0246A2F5987062286ED2DFE800F0EE6D3134373A3D40C8
S2240123804346494C4F5255585B5E61646E717483776D7A6D7D6D806D8689FEECEB8C6D8F69
S2240123A09295989B9E6D6DA1A4A7AAAD676AB0B3EAE9E8E7E6E5E4E3E2E1E0DFDE6DB6BC5B
S2240123C0C2B9BFC5C8EFF2F5F8FBD8D7D6D5D4D3D2D16D6DD0CFCECDCCCBAC48086027E1B4
S2240123E0AB48086024E1AB48086021E1AA4808601EE1AA4808601BE1A948086018E1A94828
S224012400086015E1A848086012E1A84808600FE1A74808600CE1A748086009E1A6480860EA
S22401242006E1A648086003E1A548086000E1A5480860FDE0A4480860FAE0A4480860F7E0B4
S224012440A3480860F4E0A3480860F1E0A2480860EEE0ECE0A1480860EAE0A1480860E7E00C
S224012460A0480860E4E0A0480860E1E09F480860DEE09F480860DBE09E480860D8E09E482E
S2240124800860D5E09D480860D2E09D480860CFE09C480860CCE09C480860C9E09B480860E6
S2240124A0C6E09B480860C3E09A480860C0E09A480860BDE099480860BAE099480860B7E0EE
S2240124C098480860B4E098480860B1E097480860AEE097480860ABE096480860A8E09648EE
S2240124E00860A5E095480860A2E0954808609FE0944808609CE09448086099E0934808609E
S22401250096E09348086093E09248086090E08BE087E080E07CE078E074E070E06CE068E0B9
S22401252064E060E05CE031E02DE020E01CE018E014E010E04EE04AE046E042E03EE03AE007
S22401254036E032E02EE02AE026E022E066E017E013E00FE041E08048086069E07F48086045
S22401256066E07F48086063E07E48086060E07E4808605DE07D4808605AE07D48086057E0F9
S2240125807C48086054E07C48086051E07B4808604EE07B4808604BE07A48086048E07A48B5
S2240125A0086045E07948086042E0794808603FE0784808603CE07848086039E07748086049
S2240125C036E07748086033E07648086030E0764808602DE0754808602AE07548086027E0E1
S2240125E07448086024E07448086021E0734808601EE0734808601BE07248086018E0724875
S224012600086015E07148086012E0714808600FE0704808600CE07048086009E06F48086000
S22401262006E06F48086003E06E48086000E000BF00BF0120704710B5A8B04BF6EF61DDF8D5
S224012640950061F31400CDF895009DF89C0020F0800080308DF89C009DF89B0020F0FE004D
S224012660801C8DF89B009DF89C0020F00F018DF89C1010218DF89A109DF8990020F0F8017F
S224012680B2E0000018020010872001000C3802000E3802001038020012380200143802005E
S2240126A016380200183802001A3802001C3802001E3802002038020022380200243802005C
S2240126C0283802002C38020030380200343802003838020050380200543802003C38020054
S2240126E03E3802003F380200413802004238020043380200443802004038020045380200F8
S224012700463802005838020048380200493802004A3802004B3802004C3802004D38020086
S224012720883802008C3802009038020094380200983802009C380200A03802005A3802005D
S2240127405C3802005E38020060380200623802006438020066380200683802006A3802008B
S2240127606C3802006D3802006E3802007038020072380200743802007638020078380200F8
S224012780A4380200A6380200B2380200B4380200A8380200AA380200AC380200AE38020007
S2240127A0AF380200B6380200B7380200B03802007C38020080380200813802008238020078
S2240127C083380200843802008538020086380200B8380200BC380200BE380200C03802001F
S2240127E0C1380200AD3802008DF899109DF8990020F007018DF899109DF89C0020F070009E
S22401280020308DF89C0040F23D11BDF8970061F34F1007A9ADF89700FB4890F834008DF852
S2240128209D0000208DF89E0002208DF8940007986FF31400079040F23D11BDF81E0061F324
S2240128404F10ADF81E009DF8200020F007008DF820009DF8200020F0F8008DF82000172046
S2240128608DF821009DF8220020F001008DF822009DF8220020F0FE00801C8DF822009DF8A0
S224012880230020F00F008DF823009DF8230020F0700020308DF823009DF8230020F08000D0
S2240128A080308DF8230009986FF31400099040F2FF71BDF8260061F34F10ADF8260007A860
S2240128C0007B20F0070107A80173007B20F0F800F83007A90873FF2107A84173807B20F0D8
S2240128E0010107A88173807B20F0FE00FE3007A9887307A8C07B20F00F0107A8C173C07B23
S22401290020F07000703007A9C87307A8C07B20F080008030C873BD480C900020ADF82C00AF
S2240129200D986FF314000D909721BDF8360061F34F10ADF8360007A8007F20F0070107A8B3
S2240129400177007F20F0F80107A8017780214177807F20F0010107A88177807F20F0FE012B
S22401296007A88177C07F20F00F0107A8C177C07F20F07000203007A9C87707A8C07F20F068
S22401298080008030C8770F98410D49050F9140F2FF72BDF83E1062F34F11ADF83E109DF8FC
S2240129A0400020F007018DF840109DF8400020F0F8018DF84010FF218DF841109DF8420064
S2240129C020F001018DF842109DF8420020F0FE018DF842109DF8430020F00F018DF843107B
S2240129E09DF8430020F0700170318DF843109DF8430020F0800180318DF84310834912919E
S224012A00002107A8018506F017F904469DF89420214601A804F024FF01A9204606F027F974
S224012A200021204604F014FB0121204606F0F4F980214FF46F4004F02DFC81214FF46F4057
S224012A4004F028FC83214FF46F4004F023FCFF214FF42C4004F01EFC90214FF46F4004F03B
S224012A6019FCB0214FF46F4004F014FC84214FF46F4004F00FFC6649087028B010BD654865
S224012A80807E20B1002063498876052070476148407B00F00300012800D1F7E70020F5E790
S224012AA000B589B0002008908DF8040001208DF8100007F005FA8DF81C0001208DF81400DA
S224012AC0002106915448008841F2883148435349098841F28832514300EB2140029001A868
S224012AE002F0FCFB00208DF81C008DF8140001208DF8040001A802F0F1FB01208DF81400A2
S224012B004FF07C51069103208DF8040001A802F0E5FB00208DF8140002208DF80400012060
S224012B208DF8100002208DF81C003B4800883C4948433A4909883A4A514300EB2140029012
S224012B4001A802F0CBFB344800883649484333490988344A514300EB2140029007208DF857
S224012B60040001A802F0BAFB06208DF8040001A802F0B4FB2848008829494843274909880C
S224012B80274A514300EB2140029004208DF8040001A802F0A3FB05208DF8040001A802F01D
S224012BA09DFB09B000BD10B51A48B0F80B10002008F0A1FA10BD10B51B48007802F01EFCEB
S224012BC004462146002008F041FC10BD10B51648007802F013FC04462146002008F01FFB9D
S224012BE010BD70B50621022006F026FF05460E48007802F003FC064610F0BAFB04462946B5
S224012C0010F0FEFB70BD000044C90720F371010015020010DCDC07208C3A02008E3A020057
S224012C20A086010020A107002002001010B51148007802F0E3FB10BD01207047012070478A
S224012C400D48807EC0F3011008B9012070470020FCE710B50121002007F0F9FC08F090FD43
S224012C6010BD0649087070470448007870470020704770472002001038C807201602001079
S224012C800020704770B5FE49B1F8150010F070FB0546FC49284610F0B3FB0646FA4910F087
S224012CA0B7FC0446F94910F04DFA70BD10B5FFF7E9FF0446F649204610F06EFC00D2F44C4D
S224012CC0F449204610F068FB00D2F24C204610F0FBFA00B210BD0120E949B1F803100A29BC
S224012CE000DA0020EC49097801B17047E4494979C1F38101012900D00020E1494979C1F3D6
S224012D000111012900D00020DD49097DC1F30111012900D0002000BFE7E710B5A8B0DF4824
S224012D200168DDF8950061F31400CDF895009DF89C0020F0800080308DF89C009DF89B0036
S224012D4020F0FE00801C8DF89B009DF89C0020F00F018DF89C1010218DF89A109DF8990093
S224012D6020F0F80008308DF899009DF8990020F007018DF899109DF89C0020F0700020307A
S224012D808DF89C0040F23D11BDF8970061F34F1007A9ADF89700C14890F834008DF89D00BA
S224012DA000208DF89E0002208DF8940007986FF31400079040F23D11BDF81E0061F34F10DD
S224012DC0ADF81E009DF8200020F007008DF820009DF8200020F0F80008308DF820001720E8
S224012DE08DF821009DF8220020F001008DF822009DF8220020F0FE00801C8DF822009DF81B
S224012E00230020F00F008DF823009DF8230020F0700020308DF823009DF8230020F080004A
S224012E2080308DF8230009986FF3140009900021BDF8260061F34F10ADF8260007A8007BE0
S224012E4020F0070107A80173007B20F0F800F83007A90873FF2107A84173807B20F00101CB
S224012E6007A88173807B20F0FE00FE3007A9887307A8C07B20F00F0107A8C173C07B20F08F
S224012E807000703007A9C87307A8C07B20F080008030C87382480C9047F23050ADF82C00DC
S224012EA00D986FF314000D909721BDF8360061F34F10ADF8360007A8007F20F0070107A82E
S224012EC00177007F20F0F80107A8017780214177807F20F0010107A88177807F20F0FE01A6
S224012EE007A88177C07F20F00F0107A8C177C07F20F07000203007A9C87707A8C07F20F0E3
S224012F0080008030C8770F98410D49050F9140F2FF72BDF83E1062F34F11ADF83E109DF876
S224012F20400020F007018DF840109DF8400020F0F8018DF84010FF218DF841109DF84200DE
S224012F4020F001018DF842109DF8420020F0FE018DF842109DF8430020F00F018DF84310F5
S224012F609DF8430020F0700170318DF843109DF8430020F0800180318DF843104849129153
S224012F80002107A8018505F057FE04469DF89420214601A804F064FC01A9204605F067FE2A
S224012FA00021204604F054F880214FF46F4004F071F93C49087081214FF46F4004F06AF96B
S224012FC070214FF46F4004F065F990214FF46F4004F060F983214FF46F4004F05BF98421A3
S224012FE04FF46F4004F056F92F49087028B010BD2348807E20B10020214988760520704763
S2240130001F48007D00F00F00F9E770B504460D46B4F5A87F02D12548286004E029462046D4
S224013020FFF7A3F900BF00BF012070BD10B5FEF7C1FE1F4908601F480968C8661E481C4912
S224013040096848601D481A49096808601C481849096888601B481649096848611A481449F7
S22401306009688861002012490968486310490968886301200E49096881F884000C4825E065
S224013080DCDC07200000A04000401C480000204100007A4400007AC41602001044C907200E
S2240130A0F37101001402001015020010C2380200CCC707200B300100F12F01001B2D0100FC
S2240130C0D72C0100AD2C0100812C0100006810BD70B504460D46B4F5A87F02D10A482860EA
S2240130E004E029462046FFF740F900BF00BF012070BD10B5FEF75EFE04490860044809688E
S224013100C8660248006810BDC3380200B0020010D130010070B505460C46A5F2351060B18C
S22401312001280DD01B2802D020280CD102E00F4820600DE00E4820600AE00E48206007E026
S2240131400D48206004E021462846FFF70EF900BF00BF012070BD10B5FEF72CFE0749086076
S22401316007480968C8660548006810BDC4380200C5380200C6380200C8380200D0C707201C
S2240131801531010010B5A748007802F037F910BD10B5A548007802F031F910BD70B5062168
S2240131A0012006F049FC05469F48007802F026F9064610F0DDF80446294610F021F970BDD1
S2240131C070B500240025994890F8BE00052811D2DFE800F00F0603090C000124002509E02D
S2240131E00124002506E00024002503E00024002500E000BF00BF2146002007F028FA2946B7
S224013200012007F024FA08F0BBFA70BD00B589B000200890844800788DF8040001208DF87F
S224013220100000208DF81C0001208DF8140080490691804800884FF47A7148437E4909883C
S2240132404FF47A72514300EB2140029001A802F045F8744800788DF8040001A802F03EF861
S224013260724890F8BE00022823D000208DF8140070480088714948436F4909886F4A514357
S22401328000EB2140029002208DF8040001208DF8100002208DF81C0066480088114648430E
S2240132A065490988514300EB2140029001A802F015F800208DF814005E4800886049484394
S2240132C05D4909885E4A514300EB2140029007208DF8040001A802F001F806208DF80400A4
S2240132E001A801F0FBFF09B000BD2DE9F0414E48007802F083F805464A48007802F07EF83F
S22401330006462946002008F056F807463146012008F051F80446454890F8BE00042805D141
S224013320214638460FF0A0FEBDE8F0812146384610F06EF9F8E710B5FFF7D7FF0446214682
S224013340002007F0EBFF10BD70B5FFF7CEFF05462946002007F0F4FE06460FF0F1FF044669
S2240133603849204610F018F900D2364C3649204610F012F800D2344C20460FF0A5FF00B2FF
S22401338070BD70B505460C46A5F2471058B109280CD1264890F8BE00022801D12B4800E030
S2240133A02B48206007E02B48206004E021462846FEF7DBFF00BF00BF012070BD10B5FEF72C
S2240133C0F9FC2549086025480968C866244822490968C860234820490968886422481E499E
S2240133E00968C86521481C490968886500201A490968C8621E4818490968C8641D481649B7
S224013400096808651C4814490968486500201249096881F87C001049096881F884000E48EB
S224013420006810BDD9C70720D8C7072044C90720CDCC4C3F8C3A02008E3A0200A0860100B3
S22401344020A1070000007A4400007AC4CC380200CB380200CA380200D4C70720833301001A
S22401346049330100373301000D320100C13101009D310100913101008531010070B5044673
S224013480FE49B1F8CC20B1F8CA10501A0FF058FF0546FB4920460FF0B3FF064629460FF0A7
S2240134A051FE70BD70B54FF4E0242046818AF348A0F840102046C18AF048A0F84210204651
S2240134C0018BEE48A0F844102046418BEB48A0F846102046818BE948A0F848102046817FEC
S2240134E0E64880F84A102046018CE448A0F84C102046418CE148A0F84E102046416ADF4829
S224013500C1652046816ADD4801662046C16ADB4841662046016BD94881662046416BD7483C
S224013520C1662046018FD548A0F87010D5480178D24880F87210204690F83B10CF4880F8C1
S2240135407910204690F83C10CC4880F88310204690F83D10C94880F88610204690F83E10ED
S224013560C64880F887102046016CC448C0F8A0102046416CC148C0F8A410204690F8530018
S224013580022803D11D21BD4880F8A810BD480E300188BA48A0F8CA104FF4E020B0F84A102F
S2240135A0B648A0F8CC104FF4E020B0F84C10B348A0F8CE104FF4E020B0F84E10AF48A0F803
S2240135C0D0104FF4E02090F85010AC4880F8D4104FF4E02090F85010A84880F8FA104FF4AA
S2240135E0E02090F85110A54880F8D5104FF4E02090F85210A14880F8D6104FF4E02090F853
S22401360054109E4880F8D7104FF4E020B0F856109A48A0F8D8104FF4E02090F8531097483B
S22401362080F8DA10062180F87910014691F886000FF09EFE0546FFF721FF9049C1F8F00026
S224013640FDF7CFFA70BD10B58C49B1F8D8008E49B1F9001006F0E0FF04460FF071FE10BD74
S2240136602DE9F041854991F8E4000FF081FE054683490FF067FD04468449B1F815000FF0F6
S22401368077FE074621464FF07E500FF0C1FF804639460FF0B5FE054621467D4800680FF05A
S2240136A0AFFE064629460FF0DFFC794908607949774800680FF0A4FE804677490FF0A8FFE2
S2240136C0064676490FF03EFD05460FF0FDFD00B2BDE8F08110B5694890F8D70048B10120A4
S2240136E001F08CFEB0F5006F01DB012010BD0020FCE7012001F082FEB0F5006F01DA0120C6
S224013700F4E70020F2E710B55C4890F8D50020B1FFF7E0FF6249087011E05C48407E00F0FD
S224013720030008B9012000E00020544991F84214484008B1012000E00020594908704F480F
S22401374090F8430456490978884208D0544801784A4880F8431440F2731003F00CFF504811
S224013760007828B9454890F9D4004749088004E0424890F9FA004449088010BD70B53F4968
S22401378091F886000FF0F4FD0646FFF777FE3B49C1F8F000FFF7B7FF4148007838B9FFF7AC
S2240137A05FFF3649B1F84014081A84B206E0FFF757FF3249B1F84014084484B22F48B0F886
S2240137C0D0003149B1F90010401AA04206DA2B48B0F8D0002C490988401A84B22748B0F82B
S2240137E0CE002949B1F90010401AA04206DD2348B0F8CE0024490988401A84B22248B0F928
S2240138000010204606F008FF054628460FF098FD064624490FF0C0FE01D24FF47A752846F9
S2240138200FF08EFD064620490FF0B6FD00D21F4D284670BD01201549B1F803100A2900DA70
S22401384000201B49097801B170471049497901F0030101B100200D494979C1F3810101299A
S22401386000D0002009494979C1F30111012900D000200649097DC1F301111BE044C9072094
S2240138800000C8423A000700DCC70720DCDC0720E8C707200000A04000401C480000204173
S2240138A0E4C7072000007A4400007AC418FCFFFF16020010012900D0002000BFC4E770B551
S2240138C005460C4640F24111681A8D421CD008DCB5F5997F0CD0A5F23F1078B101281CD1DD
S2240138E00FE0012813D0022814D00F2815D102E01F48206016E01F48206013E01E4820601D
S22401390010E01E4820600DE01D4820600AE01D48206007E01C48206004E021462846FEF7B1
S22401392024FD00BF00BF012070BD10B5FFF77EFB1649086016480968C86616481349096871
S2240139408860002011490968886110490968486111480E490968086110480C49096888669C
S2240139600F480A490968C1F888000848006810BDD0380200D2380200D4380200D83802002A
S224013980DC380200E0380200E4380200E0C70720BF380100353801007D370100473601006C
S2240139A0A53401002DE9F041FB4991F8E4000FF0DFFC0546F9490FF0C5FB0446F849B1F8D5
S2240139C015000FF0D5FC064621464FF07E500FF01FFE804631460FF013FD05462146F148E9
S2240139E000680FF00DFD074629460FF03DFBED490860ED49EB4800680FF002FD0746EB496F
S224013A000FF006FE05460FF05FFC00B2BDE8F08170B5E7490968486E804768B1E54800782F
S224013A2001F0ECFC06463146002007F00FFD05460FF086FC044605E0FFF7B4FF05460FF0D3
S224013A407FFC0446DC4920460FF0A6FD00D2DA4CDA4920460FF0A0FC00D2D84C20460FF0F7
S224013A6033FC00B270BD002070470120CA4991F8E51029B9CA49B1F803100A2900DA0020CB
S224013A80C7494979C1F38101012900D00020C4494979C1F30111012900D00020C049097DC0
S224013AA0C1F30111012900D00020704710B5A8B0B9480168DDF8950061F31400CDF89500B6
S224013AC09DF89C0020F0800080308DF89C009DF89B0020F0FE00801C8DF89B009DF89C0023
S224013AE020F00F018DF89C1010218DF89A109DF8990020F0F80008308DF899009DF8990055
S224013B0020F007018DF899109DF89C0020F0700020308DF89C0040F23D11BDF8970061F317
S224013B204F1007A9ADF897009B4890F834008DF89D0000208DF89E0001208DF89400079857
S224013B406FF31400079040F23D11BDF81E0061F34F10ADF81E009DF8200020F007008DF838
S224013B6020009DF8200020F0F80008308DF8200017208DF821009DF8220020F001008DF85B
S224013B8022009DF8220020F0FE00801C8DF822009DF8230020F00F008DF823009DF82300BE
S224013BA020F0700020308DF823009DF8230020F0800080308DF8230009986FF31400099037
S224013BC00021BDF8260061F34F10ADF8260007A8007B20F0070107A80173007B20F0F8007D
S224013BE0F83007A90873FF2107A84173807B20F0010107A88173807B20F0FE00FE3007A952
S224013C00887307A8C07B20F00F0107A8C173C07B20F07000703007A9C87307A8C07B20F076
S224013C2080008030C87366480C9047F23050ADF82C0007A805F000F804460122214601A826
S224013C4003F00EFE01A9204605F011F80021204603F0FEF980214FF46F4003F01BFB5949A2
S224013C60087081214FF46F4003F014FB70214FF46F4003F00FFB90214FF46F4003F00AFB15
S224013C8083214FF46F4003F005FB84214FF46F4003F000FB4C49087028B010BD4048807ED8
S224013CA020B100203E498876052070473C48007D00F00F00F9E770B505460C46B5F5A17F40
S224013CC021D00ADCB5F5997F11D0A5F23F1088B1012812D0022825D112E0A5F24310A8B1E5
S224013CE00D2816D0262817D027281BD117E0374820601CE03648206019E03648206016E056
S224013D003548206013E03548206010E0344820600DE0344820600AE03348206007E0334894
S224013D20206004E021462846FEF71FFB00BF00BF012070BD10B5FEF73DF81D4908602C4838
S224013D400968C8662B481A49096848602A481849096808602948164909688860002014497D
S224013D6009684861124909688861254810490968086124480E490968C86000200C4909688C
S224013D8048630B49096888634FF07E500849096848670748006810BD44C907200000C84282
S224013DA0DCDC0720B80200100000A04000401C48B40200102002001000007A4400007AC4DC
S224013DC0F37101001402001015020010E8380200EC380200F0380200F4380200F838020059
S224013DE0FC380200003902000239020004390200B73C01009D3C0100AD3A01006B3A010074
S224013E00673A0100113A010010B5FB49B1F8D800FA49B1F9001006F0FFFB04460FF090FA64
S224013E2010BD10B50446204607F05CFB10BD00B589B00120F24908708DF80400002008901C
S224013E4001208DF8100000208DF81C0001208DF81400EC490691EC480088EC494843EC49AE
S224013E600988EA4A514300EB2140029001A801F035FA03208DF8040000208DF8140001A82E
S224013E8001F02CFA01208DF81C0002208DF8040001A801F023FA00208DF8040001A801F09E
S224013EA01DFAD9480088DB494843D9490988D94A514300EB2140029007208DF8040001A8EC
S224013EC001F00CFA06208DF8040001A801F006FA09B000BD2DE9F047C74991F8E4000FF05D
S224013EE047FA0546CC490FF02DF90446CB49B1F815000FF03DFA804621464FF07E500FF06B
S224013F0087FB074641460FF07BFA05462146C44800680FF075FA064629460FF0A5F8C049DD
S224013F200860C049BE4800680FF06AFA8146BE490FF06EFB0746BD490FF004F906460FF069
S224013F40C3F905B228460FF0FBF9BDE8F08770B5FFF7C0FF0546B648007810B94FF07E50FA
S224013F6000E0B448014628460FF04AFA0446B24920460FF011FB00D2AF4CB04920460FF086
S224013F800BFA00D2AD4C20460FF09EF900B270BD70B50621012005F04FFD0546984800781F
S224013FA001F02CFA06460FF0E3F9044629460FF027FA70BD2DE9F04105460E461746002153
S224013FC09F4800680CF05AFF044664B12570668021469B4800680CF08EFF20B90221994845
S224013FE000680CF0B7FFBDE8F08170B5824890F8E90000EB800045000020934908700CF00B
S22401400031FF92490968421A7B4890F8E700904948437D4909884143774890F8E7008C4B4C
S22401402058437B4B1B88584301EB2040824201D9012000E00020044644B1002211461046C2
S224014040FFF7B8FF03208349087004E0002229B20220FFF7AFFF70BD10B5674890F8E9008D
S224014060404200EB80004FF6FF7101EA40040CF0F9FE79490968421A5F4890F8E600744915
S22401408048436149098841435B4890F8E600704B58435F4B1B88584301EB2040824201D997
S2240140A0012000E00020684909780843664908700846007828B9002221B20220FFF77AFF08
S2240140C010BD002211461046FFF774FF5848007850B96248007838B90CF0C4FE5B490860D7
S2240140E002205C49087010E05148007801280BD15A480078012807D10CF0B4FE53490860A8
S22401410002205449087000E0DAE700BFD8E710B50122052102200BF096FB00204A4908705C
S22401412001204C4908700CF09DFE4B49086010BD70B53148B0F8EA004FF6FF7101EA800596
S224014140032001F05BF9044605F11400844209DD294890F8E80008B9012000E000203F49A6
S224014160087010E0A5F11400A04209DD224890F8E80008B1012000E000203849087002E0D0
S2240141800220364908703348007830B1012807D0022808D003280AD108E0FFF7B8FF06E0A9
S2240141A0FFF75AFF03E0FFF720FF00E000BF00BF70BD01201949497901F0030101B100201B
S2240141C01649B1F803100A2900DA002013494979C1F38101012900D0002010494979C1F354
S2240141E00111012900D000200C49097DC1F30111012900D00020704744C90720ECC707200D
S22401420020020010CDCC4C3F8C3A0200A08601008E3A020020A107000000C842DCDC0720D8
S22401422008C807200000A04000401C4800002041F4C70720000080BF00007A4400007AC47F
S224014240CC020010C8020010F6C70720FCC7072040420F00F5C70720F8C7072000C8072089
S22401426070B505460C46A5F2471030B1092807D00E2808D17E4820600BE07E48206008E031
S2240142807D48206005E0214628467C4A1268904700BF00BF012070BD10B5022001F0AEF8B8
S2240142A0B0F5006F0FDB002001F0A8F840F2FF71884208DA724890F8D70008B1012000E028
S2240142C00020044626E0022001F098F840F2FF7188420EDA002001F091F8B0F5006F08DBE0
S2240142E0674890F8D70008B9012000E00020044610E0022001F082F840F2FF71884208DAB3
S224014300002001F07BF840F2FF71884201DA032400E00224204610BD10B5594890F8EC0092
S224014320B0B1574890F8D50090B95648407E00F0030008B9012000E00020514991F8421427
S224014340484008B1012000E000204F49087003E0FFF7A2FF4C490870494890F843044A496B
S2240143600978884208D048480178454880F8431440F2731003F0FFF84348007828B94048A4
S22401438090F9D4004149088004E03D4890F9FA003E49088010BD10B5FFF7BEFF3A4800786E
S2240143A0032806D13A480078032802D1002038490870334890F8EC0028B9354800780328F4
S2240143C001D0082010BD0022052102200BF03BFA2C48807E20B100202A4988760520F1E7A6
S2240143E02848007D00F00F00ECE710B5002029490870FEF71BFE28490860284809684860B9
S22401440025480068C06E1D490860254822490968C866244820490968886023481E490968DD
S2240144200867AFF293401C490968C8641F481A49096848611E4818490968C8651A211048B5
S22401444080F8A81000201449096881F87C001249096881F8840017480F490968C1F8800019
S22401446015480D49096888660B48006810BD000006390200073902000839020004C80720E3
S22401448044C90720DCDC0720F4C70720ECC70720F5C7072021020010F0C707209743010078
S2240144A061420100B3410100314101004F3F01002F3E0100233E0100093E01004A49D0E9F7
S2240144C000230CC1704710B54748006810B146490868804710BD10B5002144480CF052FD62
S2240144E0434908600022012142480CF07FFD424908600022114641480CF078FD4049086025
S224014500002140480CF0C8FC3F490860FFF7DBFF10BD10B504460121354800680CF01AFD76
S22401452010BD70470EB55EE04FF0FF3100200CF01DFD8DE807000098082853D1019800F05A
S224014540040060B1314890F84A0008B1012000E000200246244800214368084698470198D5
S22401456000F0020000283DD0002500260021264800680CF0B5FC8DE807000098202830D1C2
S224014580019C207850B1B4F90200002801DD012000E000200646B4F90200C50F1C4890F84E
S2240145A0340065F301001A4981F83400084690F8340066F3830081F83400144F97F84A7019
S2240145C00FB1012700E000273A46B4F902102078054F7B68984721460B4800680CF072FC6D
S2240145E000BF00BF00BF9FE7BC0200100C390200C802001028390200D8020010303902004B
S224014600DC0200101C390200CC02001044C9072038C80720AE49D0E900230CC17047AC48CB
S22401462070477CB505460E4645B1012D08D0022D03D0032D06D1012404E000BF002401E01B
S224014640022400BF00BF204601F067F99DF8000065F303008DF800009E4800788DF80100A0
S2240146603068CDF8020030798DF80600684602F04FFF7CBD70B504460D46974800EB0410DA
S224014680006860B9944800EB041095E84E004EC0914901EB041108688047904870BD0220A6
S2240146A0FBF7C6FE0020F9E710B5044689480078A04207D087480078022803D00420FBF7D3
S2240146C0B7FE0DE0022C03DB0320FBF7B1FE07E0814800EB0410406810B90520FBF7A8FE85
S2240146E07C4804707C4901EB04114868804710BD10B578480078022806D07749754A12786C
S22401470001EB02118868804702207249087010BD10B570480078022806D06F496D4A1278CD
S22401472001EB0211C868804702206A49087010BD70B504466A4920460EF004FD04466949E0
S22401474020460EF029FF00D2664C674920460EF023FE00D2644C654920460EF051FE0646DF
S22401476063490EF081FC05460EF0CAFD81B26148C18470BD70B55648406840B15449486805
S224014780804705460EF0DCFD0446FFF7D1FF70BD10B5002158480CF0F5FB58490860002250
S2240147A0012157480CF022FC5649086008F010FA08F094FB002154480CF06EFB5349086062
S2240147C010BD10B5044601214C4800680CF0C2FB10BD3EB54B4800680CF02AFC4FF0FF31D4
S2240147E0464800680CF0AAFB0021494800680CF077FB8DE8070010E00098202806D1019CD4
S2240148002146434800680CF05DFB00BF0021404800680CF065FB8DE8070000982028EBD0A1
S2240148203EBD0EB553E04FF0FF3100200CF09EFB8DE807000098082848D1019800F0040073
S22401484018B1FFF755FFFFF7C4FF019800F0010008B1FFF78FFF019800F00200002835D007
S22401486000212A4800680CF03BFB8DE80700009820282BD1019C207800F00F0020B101287F
S22401488013D002281BD115E00221224800680CF061FBC8200CF092FA6078FFF705FF642110
S2240148A0184800680CF0B8FB09E0FFF721FFFFF790FF04E0FFF72CFFFFF78BFF00BF00BFF4
S2240148C02146124800680CF0FDFA00BF00BFAAE7E4020010E00200106008001023460100DD
S2240148E00000C84200002041000020C10000FA4400409C4638C8072038390200EC0200106E
S22401490054390200FC02001048390200F0020010CC0200101CC8072010B5044630222146BE
S224014920FB480BF05AFB0120FA49087010BD10B5F94990E81C001CC110BD10B5044620229F
S2240149402146F6480BF049FB10BD0020F449A1F803000846407920F00C000C304871084641
S224014960407920F03000303048710020A1F801000846407B20F00301E94841734FF4FB40E5
S224014980E749A1F80B000846407E20F00300C01C48764FF4FA41E248A0F81510007D20F092
S2240149A030003030DE4908750846007D20F00F01DB480175704710B504464FF4FA61D948B4
S2240149C000680CF029FBFFF7C0FF0321D64880F83610D648007801F0E5FD0221D448006884
S2240149E00CF0B8FA0821D24800680CF0B3FA10BD10B5C948006810B1C74908688047CD4887
S224014A000088CD494843CD490988CB4A514300EB2140CB49086000221146CA480CF0E6FAE8
S224014A20C04908604FF4FA61BE4800680CF0F4FA00220121C4480CF0D9FAC449086005214F
S224014A40C24800680CF0E8FA10BD10B504460121BF4800680CF07EFA10BD10B54FF4FA61EF
S224014A60B04800680CF0D8FA10BD2DE9F0410025A748007C002833D0A548C06980B3A449FD
S224014A80C8698047044620460EF072FC8046A048816940460EF0B4FC0746AE490EF0B0FC42
S224014AA006460EF02DFCA04988719948408AA04203DC9748808AA04212DA012501219A484E
S224014AC080F8361037300021016001710121373880F83710807900EB800041009248018760
S224014AE08B48007890B38A48C06878B38849C8688047044620460EF03BFC804684488168D5
S224014B0040460EF07DFC074692490EF079FC06460EF0F6FB8449C8717D484088A04203DC68
S224014B207B488088A04211DA012501217E4880F836103730002101600171373880F8371082
S224014B40C07900EB8000410077480187704890F82000C8B36E48C06AB0B36D49C86A804756
S224014B60044620460EF004FC80466948816A40460EF046FC074677490EF042FC06460EF0C6
S224014B80BFFB6949097960F30601674801716048408CA04203DC5E48808CA04214DA0125C9
S224014BA00121614880F8361037300021016001710221373880F83710007900F07F0000EBE7
S224014BC0800041005848018785F00100BDE8F0812DE9F0410124042000F01EFC07465E49CC
S224014BE00EF00EFC0546052000F016FC07465A490EF006FC0646594928460EF0CDFC14D23C
S224014C00574801780078401C554A107064290FDD0921454880F8361037300021016001713A
S224014C20002400201146087002E000204C4908704A4930460EF0B0FC14D24A480178007830
S224014C40401C484A107064290FDD0A21364880F8361037300021016001710024002011460A
S224014C60087002E000203F4908702046BDE8F0812DE9F0470CF0F6F804462E4800883A4936
S224014C8048432E490988384A514300EB214037490968611A88423AD2264909884FF47A72A8
S224014CA05143264A12884FF47A735A4301EB22400EF046FB82462E490EF0A2FB80462B49E2
S224014CC00968601A0EF054FB814641460EF03AFA064612494869804726490988A0EB010863
S224014CE040460EF02DFB074631460EF02BFA05460EF0EAFA01B20C48A0F81F100246B2F92D
S224014D002100B2F91F10002936DB0A4635E05DE0BC08001000030010EC080010F8080010BB
S224014D20DCDC07200803001038C80720150200101CC807208C3A020040420F008E3A0200F7
S224014D40040300105C390200643902000C030010100300100000204100007A4400409C457E
S224014D60140300101503001020A107001C03001000007A43200300104A42002801DB03461E
S224014D8000E043429A4206DDFD48B0F81F10A0F82110FC480460FC480088FC494843FC497B
S224014DA00988FA4A514300EB2140F6490968611A884204D2F248B0F81F10A0F82110F54856
S224014DC00460F54948698047F4490880BDE8F0872DE9FE4F00200290EF4988688047044684
S224014DE0ED49486880470546EB49086880470646FBF791FF0746FFF738FE08B9012002908F
S224014E00E7484068002864D0E54948688047012820D1DB48807E20F030001030D8498876DA
S224014E20084690F83E0020F00700401C81F83E000321D34880F83D1090F83E0020F0F8015B
S224014E40CF4880F83E10012002900221CC4880F8361005E0CA48807E20F03001C84881768A
S224014E60CF48806818B3CE4988688047F8B9C44890F82D0020F00C01C14880F82D1090F8BF
S224014E80330020F00C01BE4880F83310082180F8361037300021016001713738807E20F03C
S224014EA030002030B64988760120029018E0B44890F82D0020F00C00001DB14981F82D003A
S224014EC0084690F8330020F00C00001D81F8330006E0AB48807E20F030003030A849887678
S224014EE0AD48C06998B1AC49C86980478046AD4940460EF085FA81460EF002FAA049B1F846
S224014F00191060F30B019E48A0F8191000BFA2484069002879D0A049486980470146009061
S224014F20002006F093FA01900EF00AFA83469E490EF008F9804698494869804783465946FF
S224014F40002006F038FA81464FF0000A954940460EF022FB01D2DFF84C82944940460EF09B
S224014F601BFA01D2DFF844828B48806940B18A498869804783465946012006F01CFA824611
S224014F804946002006F05DFB5146012006F059FB874948460EF03CFB864901900EF0D2F851
S224014FA083460EF0ADF901467548B0F82F0061F309007349A1F82F007D4950460EF028FB45
S224014FC07C4901900EF0BEF883460EF099F96C49098E60F38B016A480186414676480EF0C1
S224014FE00FFA764900900EF03FF8754901900EF03BF883460EF084F96149B1F81B1060F389
S2240150000B015F48A0F81B1000BF6548806810B163498868804707F00400042813D102216E
S224015020684800680BF096FFC8200BF0C7FE052000F073FC6448007801F0B4FAC8200BF0F0
S224015040BDFE04F0B7FF07F0020002280CD1524908698047012002900421494880F83610EB
S224015060373000210160017102F08FFA70B90321434880F8361037300021016001713738F4
S22401508080F83710042000F048FC06E000F042FC042802D1002000F040FC394890F82D005E
S2240150A0C0F38100012807D1354890F82D0065F38300334981F82D00314890F83300C0F39F
S2240150C08100012807D12E4890F8330065F383002B4981F833002A4890F82D0064F3051089
S2240150E0274981F82D00084690F8330064F3051081F83300084690F82D0066F3010081F89D
S2240151002D002549C86880471D49A1F82B00012C09D005211A4880F8361037300021016098
S2240151200171012002904EB10621154880F83610373000210160017101200290FFF798FD6A
S2240151400BF090FE21490968B0FBF1F0C0430C49097960F3C7110A480171FFF739FD08B9A3
S22401516001200290029848B10221164800680BF0F1FE0421164800680BF0ECFEBDE8FE8F0E
S22401518038C80720180300108C3A0200404B4C008E3A02001C030010F808001020030010DC
S2240151A0EC0800100000C842000020410000C8C2C3F5C8BF75C84D3B0000A0410000FA44CD
S2240151C0000040421CC807201402001004030010EC02001010B5FFF70BFC00210F480BF0CC
S2240151E0D1FE0F49086010BD0EB516E04FF0FF3100200BF0BBFE8DE80700009808280BD131
S224015200019800F0020008B1FFF727FC019800F0010008B1FFF7DCFD00BFE7E76C390200E5
S2240152201003001070B504460D46FA4800EB4410057634B1012C09D0022C0CD0032C14D17E
S2240152400EE02946012004F0DFFC0FE02946022004F0DAFC0AE02946032004F0D5FC05E08B
S2240152602946042004F0D0FC00E000BF00BF70BD10B500242FE0E74800EB4410C06900B902
S22401528028E0E54A02EB44025178E34A12F81400012208F0D1F830B1DE4800EB4410C16936
S2240152A00020884710E0DC4A02EB44025178DA4A12F81400002208F0BFF828B1D54800EBF3
S2240152C04410C169012088474FF40001002008F0DEF800BF641C032CCDDD10BD2DE9F843F2
S2240152E004464FF000082178CA4A02EB4110202221460AF072FE2078032801DDBDE8F88358
S2240153002078C54901EB40004578207811F810600EB1022E31D12078BE4901EB4010406873
S224015320BE4988421BD10020034602462946009030460AF0C1FA00221E2101200AF069FAF0
S224015340012000FA05F10022304608F057F8012000FA05F10246304608F050F80DE000203B
S22401536000FA05F10246304608F048F8002000FA05F10122304608F041F8002709E0A5486A
S22401538000EB47104068A549884201D14FF001087F1C032FF3DDB8F1000F20D0A0491520E8
S2240153A008F0CAF81520012181404209920002F1E022C2F8001100BFE121002809DACA06DC
S2240153C04FEA126C974A00F00F031B1F02F803C003E0CA06130E944A135400BF08E0152041
S2240153E001218140914A430942F8231000BF00BF217E2078FFF716FF00BF7FE701468C4830
S22401540030F8110070478A48808970478848C08970478748C088704770B505460A2D42D2AB
S224015420DFE805F0050B11171D23292F353B0621022004F001FB044636E00621012004F095
S224015440FBFA044630E00621002004F0F5FA04462AE00621042004F0EFFA044624E00021E2
S224015460052004F0E9FA04461EE00121052004F0E3FA044618E00321052004F0DDFA04462A
S22401548012E00221052004F0D7FA04460CE00421052004F0D1FA044606E00521084604F030
S2240154A0CBFA044600E000BF00BF614931F815000DF05EFF064621460DF0A2FF70BD08B5FC
S2240154C05C4890F87900032802D0042801D100BF0CE0002002230122172100900AF0ECF96C
S2240154E00122172100200AF094F900BF00BF002002230122182100900AF0DEF901221821C8
S22401550000200AF086F9002002230122192100900AF0D2F90122192100200AF07AF90020EB
S224015520022303221E21009001200AF0C5F901221E2110460AF06DF90020022303221F21B1
S224015540009001200AF0B8F901221F2110460AF060F944F62061384807F0A0FE00220221C8
S224015560354807F0FCFE00220121334807F0F7FE00221146304807F0F2FE002204212E4877
S22401558007F0EDFE002205212B4807F0E8FE08BD10B5FFF794FF04F053FB10BD2DE9F0471C
S2240155A004460D461B4800EB4410007C10B101282DD103E01E4820F8145028E0154800EB2D
S2240155C0441041694FF07E500EF022F8814628460DF0CEFE824649460DF012FF0746144995
S2240155E031F814000DF0C4FE81460A4800EB4410416948460DF004FF804639460DF034FDA6
S22401560006460DF07DFE0A4921F8140000BF00BFBDE8F087C8CE07207C39020041420F00A0
S2240156207152010018ED00E000E400E080E100E008D0072044C90720004003402DE9F041B9
S22401564004460D4617464FF0000801222146A64807F085FE052C02D1384604F0C0FB0026BA
S2240156600EE00121A04807F046FE21469E4807F0B4FE21469C4807F085FE8044701C86B2AE
S224015680AE42EEDB00222146974807F068FEB8FBF5F080B2BDE8F08170B505460E460024BE
S2240156A00A2D70D2DFE805F0051A2F445970868D94AA062231460220FFF7C0FF044672B61B
S2240156C0C4F3870189488172A010000A8749897B60F301018548817362B6A6E006223146E0
S2240156E00120FFF7ABFF044672B6C4F387017F48C172A010000A7D49897B60F383017B481A
S224015700817362B691E0062231460020FFF796FF044672B6C4F3870174480173A010000A21
S2240157207249897B60F305117048817362B67CE0062231460420FFF781FF044672B6C4F3B9
S22401574087016A484173A010000A6849897B60F387116648817362B667E00022314605203C
S224015760FFF76CFF044672B6C4F387015F488174A010C0F301215D48807D61F303005B4953
S224015780887562B651E04FE0012231460520FFF755FF044672B6C4F387015448C174A01053
S2240157A0C0F301205149897D60F307114F48817562B63AE0032231460520FFF73FFF044606
S2240157C033E0022231460520FFF738FF04462CE0042231460520FFF731FF044672B6C4F35C
S2240157E0870142480175A010C0F301213F48C07D61F303003D49C87562B616E0052231460C
S2240158001046FFF71BFF044672B6C4F3870137484175A010C0F301203449C97D60F3071184
S2240158203248C17562B600E000BF00BFA1B22846FFF7B4FE70BD70B50BF014FB0546002408
S2240158401EE02B4800EB44104068C0B1284800EB44108068281A264901EB44114968884275
S2240158600DD3234A02EB4412117B214A02EB44121078FFF711FF1E4800EB44108560641CC0
S2240158800A2CDEDB70BD10B5FFF782FE002119480BF078FB184908600022012117480BF054
S2240158A0A5FB174908600121154800680BF0B4FB10BD10B5044601210F4800680BF04AFBEC
S2240158C010BD0EB50FE04FF0FF3101200BF04EFB8DE807000098082805D1019800F00100CB
S2240158E008B1FFF7A8FFEEE70040034038C80720C8CE072084390200280300109439020047
S2240159002C03001010B5044638222146FC480AF064FB10BDFB4800787047FA490870FA4A97
S224015920907070470020F9490870F74890F82D0020F0C001F44880F82D1090F8330020F04F
S224015940C001F14880F83310807EC0F30110012807D0ED4890F83E0020F00701EA4880F80D
S2240159603E10704710B50120E8490870E64890F82D0020F0C0004030E34981F82D0008464A
S22401598090F8330020F0C000403081F83300E0480078012806D1DF48007800F003FE00200A
S2240159A0DB49087010BD10B504F01CFBDA49087004F018FBD9490870FFF7D4FF002211462A
S2240159C0D7480BF013FBD749086010BD10B542F21071D44800680BF01FFBC9488169012015
S2240159E08847C748806838B1C5498868804704460DF0A6FCCC49086010BD10B5C048816943
S224015A000020884710BD10B504460821C74800680BF0A0FA10BD70B505460E460021C448C2
S224015A2000680BF02BFA044664B1257066802146BF4800680BF05FFA20B90221BD4800686B
S224015A400BF088FA70BD2DE9F04106460C461546B94930460DF076FB0646B74920460DF0C1
S224015A6071FB0446B44928460DF06CFB0546B34930460DF091FD00D2B04EB04920460DF027
S224015A808BFD00D2AD4CAD4928460DF085FD00D2AA4DAB4930460DF07FFC00D2A84EA84966
S224015AA020460DF079FC00D2A54CA54928460DF073FC00D2A24DA34930460DF0A1FC8046FA
S224015AC0A1490DF0D1FA07460DF01AFC81B28E4881849C4920460DF093FC80469A490DF023
S224015AE0C3FA07460DF00CFC81B28748C184954928460DF085FC804693490DF0B5FA0746E5
S224015B000DF0FEFB81B280480185BDE8F0812DE9F05F00257A48806818B17949886880477C
S224015B2005468A49D1F890000DF022FC834688490DF066FC824687490DF062FC8146704862
S224015B40816A48460DF05CFC80468048D0F8E01040460DF055FC07467C48D0F8DC10384614
S224015B600DF04EFC06467C490DF0ECFA044628460DF0E6FB074621460DF0E4FA06460DF076
S224015B80A3FBBDE8F09F2DE9F04105460C46704860616148007885422DD16C49C86D0DF003
S224015BA0E7FB06466B490DF02BFC20606749086E0DF0DEFB074667490DF022FC064661692F
S224015BC00DF0C0FA60606149486E0DF0D1FB074660490DF015FC064661690DF011FCA060FB
S224015BE05A49886E0DF0ACFB20615849C86E0DF0A7FBE0603FE049480078854235D153499A
S224015C00D1F88C000DF0B4FB064652490DF0F8FB20604E49D1F890000DF0AAFB06464D49B2
S224015C200DF0EEFB60604949D1F894000DF0A0FB064648490DF0E4FBA060616960680DF0E9
S224015C40DFFB0646314645480DF07CFA2061616960680DF0D5FB0646314641480DF072FA0C
S224015C60E06040480078207605E0002020606060A0602061E060BDE8F08113B5FFF772FEFE
S224015C80BDF8020042F21071884210DCBDF8020000280CDDBDF80200401D6FF0090190FB0C
S224015CA0F1F004B221460220FFF7B5FE71E0BDF8040042F2107188420FDCBDF804000028C0
S224015CC00BDDBDF80400401D0A2190FBF1F004B221460220FFF79FFE5BE09DF8010000F096
S224015CE0030060B11948B0F846006FF0090190FBF1F004B221460220FFF78DFE49E033E06A
S224015D0034D0072010C8072038C8072011C807200FC80720150200100CC807200DC8072010
S224015D209C39020018C8072014C807201CC80720CC020010C80200100000C842000020414E
S224015D40000020C10000FA4400409C4644C90720CDCCCC3DACC5273700401C4600007A44F7
S224015D6000007AC4210200109DF80100C0F3011058B1FE48B0F848000A2190FBF1F004B2C6
S224015D8021460220FFF747FE03E000210846FFF742FE1CBDF54991F8A8101C2902D01D29FC
S224015DA002D100BF012001E0002000BF00BF70472DE9F34F81B00C46ED48007888B3ED49FB
S224015DC0B1F803000CF0AAFE07460022EA4B0CF0D9FC05460CF0E8FB81464FF07C5148466D
S224015DE00DF0DAFA01D24FF07C5949464FF07E500DF0A8F9009049464FF07D500DF034F956
S224015E00054629464FF07D500DF09CF982464FF07E5B5B465246D9480078009904F051F99B
S224015E2000BF20460DF08CFA054601980DF088FA06462A463146D148007804F0B1FABDE849
S224015E40FE8F2DE9F04788B0CD49486880470446082C05D1CA49C86A804708B0BDE8F08769
S224015E60FFF758FD012800D1F7E7002500260027C348806838B1C2498868804780460DF026
S224015E805FFAC0490860062C5CD2DFE804F03A031E2C1009FFF7B1FD0020FFF73EFD52E050
S224015EA0FFF7ABFD0320FFF738FD01274BE00020FFF733FDB249C869804728B9FFF786FD0A
S224015EC0B1480068AF4908603DE0FFF796FD0020FFF723FDAD4E0127AD49AA4800680DF0AF
S224015EE097FB05462FE0FFF788FD0020FFF715FDA84E0127A649A34800680DF0B5F80546B8
S224015F0021E0A5480078012809D1984890F8830028B1FFF75BFD9C4800689A4908609E4883
S224015F200078022803D09C480078032809D18F4890F8F80028B1FFF749FD934800689149FC
S224015F40086000E000BF00BF8D49C8698047D0B18B49086A804705468B48016828460DF027
S224015F6057FB81468748016828460DF051FB824649460DF045FA804600210DF00DFA4AD873
S224015F80FFF73BFD47E07E48406998B3774AD2F8DC107B4A906A0DF033FA82467348D0F841
S224015FA0E01050460DF02CFA81467C490DF0CAF8804641467148007804F0B8F8704948695B
S224015FC0804781466E490869804782464946FFF7EFFE05466A4890F83400012809D165489B
S224015FE0407900F0030020B16D4928460DF008FA054610E0FFE7022C02D0032C02D100E0F8
S22401600000BF07E05E49C868804780460DF098F9054600BF00BF5A48006B98B15848016BB7
S22401602007A888470798416828460DF0B5FA01D2079845680798016828460DF0ADF901D26F
S224016040079805684E48806810B1FFF7A3FE08B12E4621E007BB454AD2F8A410484A506A0F
S2240160600DF0CEF982464148D0F8A01050460DF0C7F9814649490DF065F8804641464948A9
S224016080007804F053F82A463E4801684548007804F086F9064600BF012C03D03849C869AF
S2240160A0804718B136490868804718B9022C01D0032C14D13C48007888B937480470324608
S2240160C0304801682846FFF7BEFC30460DF0FCF80FFA80F841460120FFF79DFC84E0FFF742
S2240160E019FC03281ED10022264801681046FFF7AAFCFFF70CFD81460DF022F98046424654
S22401610000211E48007804F03BFA052C6CD119481B30016805914068014606900598FFF720
S224016120ACFD61E01CB120480078012852D169461C480078FFF727FD69461A48007803F055
S2240161405EFF00220F4801681648007804F018FA69460A480078FFF716FD69460748007826
S22401616003F04DFFFFF7D3FC81461FE044C9072021020010DCDC072000408F400DC80720FE
S22401618034D0072028C8072014C807200000FAC30000FA440000FA430FC8072000401C46DC
S2240161A0000080BF0CC8072011C807200DF0C8F88046424600213948007804F0E1F900228A
S2240161C0374801681046FFF73EFC00210846FFF722FC09E00022324801681046FFF733FC5F
S2240161E000210846FFF717FC2E48047000BF34E610B500212C480AF0C5FE2C490860002248
S22401620001212B480AF0F2FE2A4908600022114629480AF0EBFE29490860FFF7C4FB64213D
S224016220244800680AF0F8FE4FF47A71234800680AF0F2FE10BD10B5044601211B480068E0
S2240162400AF088FE10BD10B504464FF47A711B4800680AF0E1FE10BD0EB51DE04FF0FF310E
S22401626000200AF083FE8DE807000098082812D1019800F0020010B1FFF774FB0CE0019820
S22401628000F0010008B1FFF7DCFD019800F0080008B1FFF7B2FB00BFE0E700000DC8072010
S2240162A028C807200FC80720A43902001CC80720B439020020C80720BC39020024C80720D1
S2240162C070B504460D4616469D48006828B13246294620469A4B1B68984770BD70B5044644
S2240162E00D46984951F8240029460AF004FE28B1002229462046FFF7E3FF06E00221924801
S22401630000680AF027FE012070BD0020FCE710B504462046FBF712FB8C492046FBF7B3FB50
S22401632010BD10B504462046FBF774FB10BD70B504460D46864951F8240029460AF0DBFDA8
S22401634028B1012229462046FFF7BAFF06E004217D4800680AF0FEFD012070BD0020FCE739
S2240163603EB504467A4951F8240000210AF0B8FD8DE8070012E00098202807D1019D744959
S22401638051F8240029460AF09DFD00BF704951F8240000210AF0A4FD8DE80700009820288A
S2240163A0E9D03EBD6649086070476A4A42F82010704708B50020034603221521009009F076
S2240163C07BFA0020034603221621009009F074FA0020034602220421009009F06DFA0020C4
S2240163E0034602220521009009F066FA08BD10B5FFF7DFFF5848007800B110BD0021574867
S2240164000AF0C0FD50490860002155480AF044FD4C490860002153480AF03EFD4C490860DA
S224016420002151480AF038FD4649486000214F480AF032FD4649486001204749087000BF36
S224016440DBE710B54448007800B910BD3E4800680AF0BAFD00204049087000BFF5E786B094
S2240164606DE04FF0FF3100200AF080FD03AB07C30398082862D1049800F0020058B3002490
S22401648027E0304951F8240000210AF029FD8DE80700009820281AD1019E2046FBF798F9F9
S2240164A048B12C4850F8240028B12A4850F82420314620469047234951F8240031460AF028
S2240164C001FD0221204800680AF044FD00BF601CC4B2022CD5DB049800F0040070B3002424
S2240164E02AE01B4951F8240000210AF0F9FC8DE80700009820281DD1019E2046FBF768F909
S22401650060B100BF31462046FBF70CFB0546002DF8D0022D02D12046FBF72FFB0C4951F86D
S224016520240031460AF0CEFC0421074800680AF011FD00BF601CC4B2022CD2DB00BF90E750
S224016540380300104C03001040030010DD62010044030010300300103C030010C439020010
S224016560D4390200E0390200EC390200F839020010B50446AF48007840280ED0AD490A7855
S2240165800978491CAB4B1970C2EBC201AA4A02EB81001C22214609F020FDA6480078401E3F
S2240165A0C0B210BD70B50446A2480078844200DB70BDC4EBC401A04A02EB8101497A9F4A7E
S2240165C0515C9F4A52F8210000210AF057FC0546002D47D0C4EBC400974951F82000286073
S2240165E0C4EBC40001EB8000007A28712A79C4EBC4000B4603EB80004168681D09F0A8FC03
S224016600C4EBC4008C4901EB800090F90A0000280FDBC4EBC4020B4603EB8202917AC4EB29
S224016620C40203EB8202507A2A4601F055FB064609E0C4EBC401804A02EB8101487A29468E
S22401664001F0A2FB06466EB1C4EBC4017A4A02EB8101497A794A515C794A52F821002946C4
S2240166600AF030FC00BFA3E7C0EBC002724B03EB8202117670472DE9F0410AF0F3FB054651
S22401668000248AE00026C4EBC4006B4901EB8000007E00B980E0C4EBC400674901EB800087
S2240166A0007C002856D004EB8400664901EB8000007AE8B3C4EBC4035F4F07EB83031A7A37
S2240166C0C4EBC40307EB8303596804EB84035D4F07EB830303F1090009F00EFC40B304EB89
S2240166E08400394651F82000281AC4EBC401524A02EB81014969884220D30126C4EBC4035B
S224016700174607EB83031A7AC4EBC40307EB8303596804EB84034B4F07EB830303F10900D6
S22401672009F016FC04EB8400394641F8205000E004E004EB840001EB80004560C4EBC400F2
S2240167403D4901EB8000007A04EB84013D4A02EB81010872C4EBC400374901EB8000C0685C
S224016760A8B104EB8400374901EB80004068281AC4EBC401304A02EB8101C968884206D340
S224016780012604EB84002F4901EB8000456016B1E0B2FFF707FF00BF641C26480078844290
S2240167A0FFF670AFBDE8F0812748008842F2107148432649098842F21072514300EB2140DC
S2240167C023490860704710B5FFF7EEFF002121480AF0D8FB20490860002201211F480AF0B3
S2240167E005FC1F4908600A211D4800680AF014FC10BD10B504460121174800680AF0AAFB5C
S22401680010BD0EB514E04FF0FF3100200AF0AEFB8DE807000098082809D1019800F0010014
S22401682028B1FFF728FF02F0FDFA02F095FE00BFE9E7000074030010B4D0072080C80720BE
S22401684044030010B4D707208C3A02008E3A020078030010043A02007C030010143A0200ED
S2240168608003001010B503201649087000211548007803F0C9F910BD10B512480078012888
S22401688006D0022806D0032806D0042808D105E0002405E0012403E0022401E0032400BF33
S2240168A000BF2046FEF7AAFD074908800846008840F2FF71884201DA012010BD0020FCE72B
S2240168C001207047840300108603001001690978012902D008290ED106E07A4A01690B682C
S2240168E093604968D16007E0764A01690B6813604968516000E0704700BF00BFFBE710B5A8
S22401690004466068B0F56F4F03D12046FFF7DEFF00E000BF00BF10BD70B58EB006460C46C3
S224016920154600206849087008986FF31400089040F23D11BDF8220061F34F10ADF822002E
S2240169409DF8240020F007008DF8240042208DF825009DF8260020F001008DF826009DF8A0
S224016960260020F0FE001A308DF826009DF8270020F00F008DF827009DF8270020F0700025
S22401698020308DF827009DF8270020F0800080308DF827000A986FF314000A900021BDF8C5
S2240169A02A0061F34F10ADF82A0008A8007B20F0070108A80173007B20F0F800F83008A962
S2240169C00873FF2108A84173807B20F0010108A88173807B20F0FE00FE3008A9887308A86E
S2240169E0C07B20F00F0108A8C173C07B20F07000703008A9C87308A8C07B20F080008030E0
S224016A00C87332480D900020ADF830005CB19DF8240064F3C7008DF824002B48007802F0BF
S224016A2026F92B49087065B19DF8240065F3C7008DF8240008A92448007802F018F92449A9
S224016A400870214800788DF80D0000231A46EF21062001F037FF01901D48007840B28DF880
S224016A600E001C48029008208DF80C001A4800881A4948431A490988184A514300EB214045
S224016A8004901348007840B28DF80E0001208DF814000020069001208DF81C0001A8FFF733
S224016AA067FD0EB070BD0748408800B2A0F51C5010380A2190FBF1F000B270470148807B2B
S224016AC070470000CCDC072034C80720FF68010035C807202CC807208C3A0200A086010071
S224016AE08E3A020010B5FE49FE4A1278895CFE4A52F8210000210AF0C1F90446D4B1FB4869
S224016B00206008202071FA480168C4F805104068C4F809002146F348007801F035F948B11B
S224016B20EF49F04A1278895CEF4A52F8210021460AF0C8F910BD70B50AF094F9ED49096888
S224016B40B0FBF1F4EC48C088251AEB49CC80EB48007838B10846D0F80100E94908600020FF
S224016B60E6490870E448D0F80100E5490968401A90FBF5F0E3490860DF48D0F80100E0495D
S224016B80086070BD10B5044620690078312802D0EA280CD108E0D849206902680A60007951
S224016BA00871FFF7C8FF03E0FFF79CFF00BF00BF00BF10BD10B504466068B0F52C4F06D04E
S224016BC0B0F56F4F08D12046FFF7DCFF05E0CA4821698978417100E000BF00BF10BD00B528
S224016BE0A9B00020C849087001208DF89800DDF899006FF3140000F21540CDF899009DF831
S224016C00A00020F0800080308DF8A0009DF89F0020F0FE018DF89F109DF8A00020F00F019D
S224016C208DF8A01017218DF89E109DF89D0020F0F8018DF89D109DF89D0020F007018DF872
S224016C409D109DF8A00020F0700020308DF8A0009721BDF89B0061F34F1008A9ADF89B00AB
S224016C601C208DF8A10001208DF8A200A648007800EB400051F830006FF3140000F20740AB
S224016C80A149097801EB410108AA42F8310097219D48007800EB400002EBC000408861F32F
S224016CA04F109949097801EB410102EBC10148809548007800EB400008A901EBC000007911
S224016CC020F007009049097801EB410102EBC10108718D48007800EB400008A901EBC00012
S224016CE0007920F0F8008849097801EB410102EBC101087110208449097801EB410102EBCC
S224016D00C10148718048007800EB400008A901EBC000807920F001007B49097801EB4101AD
S224016D2002EBC10188717848007800EB400008A901EBC000807920F0FE007349097801EBB5
S224016D40410102EBC10188716F48007800EB400008A901EBC000C07920F00F006A49097800
S224016D6001EB410102EBC101C8716748007800EB400008A901EBC000C07920F0700020303F
S224016D806149097801EB410102EBC101C8715E48007800EB400008A901EBC000C07920F0BD
S224016DA0800080305849097801EB410102EBC101C8715548007800EB400008A901EBC000C8
S224016DC080686FF314005049097801EB410102EBC101886000214C48007800EB400002EB2B
S224016DE0C000408961F34F104749097801EB410102EBC10148814448007800EB400008A9BA
S224016E0001EBC000007B20F007013F48007800EB400002EBC00001733B48007800EB4000BC
S224016E2008A901EBC000007B20F0F800F8303649097801EB410102EBC1010873FF21324852
S224016E40007800EB400002EBC00041732E48007800EB400008A901EBC000807B20F00101A5
S224016E602948007800EB400002EBC00081732648007800EB400008A901EBC000807B20F0DE
S224016E80FE00FE302049097801EB410102EBC10188731D48007800EB400008A901EBC00099
S224016EA0C07B20F00F011848007800EB400002EBC000C1731448007800EB400008A901EBF1
S224016EC0C000C07B20F0700070300F49097801EB410102EBC101C8730B48007816E00000DF
S224016EE080C80720A40300104403001000A0FF181C3A0200A803001088030010AC030010EB
S224016F00B0030010A0030010A503001000EB400008A901EBC000C07B20F0800080304249AF
S224016F20097801EB410102EBC101C8733F483E49097801EB410102EBC101486100203A49FA
S224016F40097801EB410102EBC101088208A801F073FE37490870084600788DF80D000023BE
S224016F602022FF21062001F0ADFC01902E48007840B28DF80E002F48029008208DF80C0023
S224016F802D4800884CF2503148432C4909884CF25032514300EB21400490FF208DF80E00B8
S224016FA000208DF8140001208DF81C0001A8FFF7DFFA214800884FF47A7148431F49098835
S224016FC04FF47A72514300EB21401D49086029B000BD10B51B49164A1278895C1A4A52F892
S224016FE02100002109F04AFF0446E4B117482060082020710F488168C4F80510C068C4F89B
S22401700009002246084801780948007800F064FE48B10C49064A1278895C0B4A52F8210048
S224017020214609F04FFF10BDA5030010B56B0100A4030010900300108C3A02008E3A02000A
S224017040A803001080C80720440300100000EF18FA4A1070FA4A1170704770B50546F949B0
S224017060F64A1278895CF84A52F82100002109F005FF0446F4B1F548206008202071641CAB
S22401708000206060A060286860606868A060641E2246EB480178E948007800F01DFE48B1A7
S2240170A0E849E64A1278895CE74A52F82100214609F008FF70BD70B5044620690078B12881
S2240170C079D00DDC7F2838D005DCB0B1052825D00C286ED129E0882848D0A028F9D150E05F
S2240170E0B42879D004DCB2286DD0B3287DD16BE0DF280AD0EA2878D16FE0D1480178CF48C6
S22401710000782269F9F7B2FD70E02069407820B9642009F053FE02F04DFF67E0CC4821696C
S2240171200A6802608988818060E0C94821690A68C0F806200979817258E00221C5480068F3
S22401714009F008FF72B6C248123021690A680260496841601238007D00F00F0008B9FEF789
S224017160E1FB62B6BC48FFF778FF3FE0B8481B3021690A680260496841600120B44988766E
S22401718034E00021B548006809F078FE054675B12069B0F8010028802946B048006809F0CD
S2240171A0AAFE20B90221AE48006809F0D3FE1DE001E01AE010E0A2480178A04800782269E7
S2240171C0F9F7F1FE12E011E09D4801789B4800782269FAF759F809E008E099480178974857
S2240171E000782269FAF7E2F800E070BD00BF00BFFBE710B504466068B0F5594F3FD009DC36
S224017200B0F52D4F13D0B0F5574F36D0B0F5584F3DD133E0B0F56B4F25D0B0F56C4F21D001
S224017220B0F56F4F33D12046FFF745FF30E002218848006809F08EFE72B685480B30216997
S2240172400A6802608A888280897981710B38407B00F0030008B9FEF765FB62B67E48FFF771
S224017260FCFE15E000BF207BFF2805D0627BA38898B2216901F079FF0AE000BF00BF637B38
S224017280A28890B20822216902F09BFA00E000BF00BF10BD30B587B004460D4601208DF8B7
S2240172A01800664800788DF80900B4F56F4F73D100208DF8100000231A46EF21062001F0F2
S2240172C001FB00905E48007840B28DF80A00832D50D008DC702D74D0802D0BD0812D25D0BD
S2240172E0822D22D134E0842D6AD0902D55D0B02DF7D178E058482338019008208DF80800C7
S224017300584800885849484358490988564A514300EB214003900023FF22EF21062001F063
S224017320D1FA0090FF208DF80A0085E04A481B38019008208DF808004A4800884C49484374
S2240173404A4909884A4A514300EB2140039073E041481338019008208DF80800414800887E
S2240173604449484341490988424A514300EB2140039061E038480B38019005208DF808008E
S224017380384800883B49484338490988394A514300EB214003904FE06EE02F48801F0190A4
S2240173A006208DF808002F480088314948432F4909882F4A514300EB214003903CE000E01F
S2240173C023E025480F30019003208DF80800254800882849484325490988264A514300EBD8
S2240173E02140039028E01C480B30019004208DF808001C4800881F4948431C4909881D4A6E
S224017400514300EB2140039016E013481230019007208DF808000020039001208DF81000B2
S224017420104800881349484310490988114A514300EB2140059000BF65E0000036C807209C
S22401744037C8072080C80720440300100000EF18DCDC0720100300105BC80720F0020010E5
S224017460EC0200108C3A020040420F008E3A020020A10700A0860100B4F52C4F1CD10023C2
S2240174801A46AC21032001F01DFA00905B48019003208DF808005A4800885A4948435A491F
S2240174A00988584A514300EB214003905748007840B28DF80A0026E04FF67070844222D1A4
S2240174C0012D1ED100237022FF21062001F0FAF900904A481130019003208DF808000120E5
S2240174E08DF81000464800884949484346490988474A514300EB21400390FF208DF80A00EC
S22401750000E000BF00BF6846FFF732F807B030BD70B505463F49404A1278895C3F4A52F8D1
S2240175202100002109F0AAFC04461CB33C482060082020710020C4F80500C4F80900A12027
S22401754060712968C4F80610A9886181A979217322462E4801783048007800F0BDFB48B140
S2240175602C492D4A1278895C2C4A52F82100214609F0A8FC70BD10B504462246234801783D
S22401758025480078F9F7DEFA10BD10B51F4801782148007800F0F0FC10BD70B505461D4966
S2240175A01D4A1278895C1D4A52F82100002109F065FC044604B31A48206008202071641C86
S2240175C000206060A06028686060A8882081A879A072641E22460D4801780F48007800F0FA
S2240175E07BFB48B10B490C4A1278895C0B4A52F82100214609F066FC70BD000063C80720FC
S2240176008C3A0200A08601008E3A020037C8072020A1070080C8072036C8072044030010D2
S2240176200000EF18002004E00021744A1154411CC8B20228F8DB70472DE9F0410546FF26B3
S224017640FF27286810B9FF20BDE8F081002414E06A48005D78B90120684908552746AB7958
S2240176602A796879296800F0ADF90646B74201D0FF20E9E703E0601CC4B2022CE8DB00BFCF
S224017680FF2E01D03846DFE7FF20DDE710B50446204600F015FA10BD70B505460E46144660
S2240176A026B1022E0CD0032E12D10DE03DB9F9F755FB2178884202D02078F9F748FB08E0C2
S2240176C00A2000F015FA04E02046F9F73EFF00E000BF00BF70BD10B5494800F037FC0A20D6
S2240176E000F006FA10BD37B59DF80210454A515C454A52F82100002109F0C0FB0446002CB3
S22401770052D008202071002060719DF80500002141EAC0009DF804100843C5B2A571601DF3
S224017720BDF80010A4F80710DDF80610C4F8091000231A46EF21062001F0C4F820609DF890
S2240177400300FF2817D10023FF22EF21062001F0B9F820609DF80200214600F015FB18B3AC
S2240177609DF80210274A515C274A52F82100214609F0A8FB18E000231A46EF21062001F0BD
S224017780A1F820609DF803109DF80200224600F0A3FA48B19DF802101A4A515C1A4A52F837
S2240177A02100214609F08EFB3EBD70B505460E461449495D144A52F82100002109F05EFBBB
S2240177C00446D4B102202071D12060715521A17100231A46EF21062001F074F820602246D9
S2240177E03146284600F078FA38B10649495D064A52F82100214609F065FB70BD78C807204F
S2240178009976010080C807204403001010B504462069007810B1DF2811D107E056480178D4
S224017820564800782269F9F721FA09E02069407820B9642009F0C2FA02F0BCFB00E010BD04
S22401784000BF00BFFBE710B504466068B0F56F4F03D12046FFF7DAFF00E000BF00BF10BD54
S22401786070B586B006460C461546444804704248057000986FF31400009040F23D11BDF8DC
S224017880020061F34F10ADF802009DF8040020F007008DF804009DF8040020F0F8008DF827
S2240178A0040081208DF805009DF8060020F001008DF806009DF8060020F0FE008DF8060028
S2240178C09DF8070020F00F008DF807009DF8070020F070008DF807009DF8070020F0800087
S2240178E080308DF8070002986FF3140002900021BDF80A0061F34F10ADF80A009DF80C00C1
S22401790020F007018DF80C109DF80C0020F0F800F8308DF80C00FF218DF80D109DF80E00E1
S22401792020F001018DF80E109DF80E0020F0FE00FE308DF80E009DF80F0020F00F018DF8D1
S2240179400F109DF80F0020F0700070308DF80F009DF80F0020F0800080308DF80F00AFF291
S224017960191005900020ADF8100018226946304608F033FB06B070BDB5030010B403001077
S22401798070B500240DE0002507E00020F54901EB441121F81500681CC5B2102DF5DB601C4E
S2240179A0C4B2022CEFDB00221146EF4809F01EFBEE49086000221146ED4809F017FBED4903
S2240179C0086070BD2DE9F0470746884691461E464FF0000AB8F1000F02D1FF20BDE8F0875A
S2240179E0002463E00020E44901EB44110877E24800EB4410007B002856D14FF0010ADE486A
S224017A0000EB4410D8F800104160D8F804108160D94800EB441080F80E900020D64901EB3A
S224017A204411C873D44901EB44114874D24800EB441047730120D04901EB44110873CE4877
S224017A4000EB44108674CD48075506EBC601880008F08DF9C84901EB44114861C64800EBC4
S224017A604410406908B90220B8E7002514E00020C14901EB4411496905EBC50201F8220079
S224017A800021BD4800EB4410406905EBC50200EB82000162681CC5B2B542E8DB0120B64976
S224017AA001EB4411087303E0601CC4B2022C99DB00BFBAF1000F01D020468FE7FF208DE7D4
S224017AC010B50446AC4800EB4410007B78B10020A94901EB44110873A74800EB4410406915
S224017AE028B1A54901EB4411486908F07BF910BD70B50646002532E09F4901EB4511497BF8
S224017B009F4A52F821004FF0FF3109F0B7F9044624B3994800EB45100674FE23FF22EA21EA
S224017B20062000F0CFFE20600320207100206071EE21A1710021E1718F4901EB4511487BC6
S224017B402146FEF7F4FB48B98B4901EB4511497B8B4A52F82100214609F0B4F96D1C022DF4
S224017B60CADB40F2E2418148006809F055FA70BD0146814800EB4110007B704701467E48D4
S224017B8000EB4110807B704770B504460E4626B9794800EB4410807C70BD774800EB441028
S224017BA0007B20B9744800EB4410807CF4E7002501E0681CC5B2704800EB4410406905EB08
S224017BC0C50110F8210028B16B4800EB4410807CA842EEDC684800EB4410406905EBC501E7
S224017BE010F82100A8BB0120634901EB4411496905EBC50201F82200FE205F4901EB44115A
S224017C00496905EBC50201EB820148705A4901EB4411496905EBC50201EB820101F10C0014
S224017C201822314608F0D9F9534800EB4410406905EBC50100EB8100808B58B101204E4952
S224017C4001EB4411496905EBC50201EB820188700AE00BE00020484901EB4411496905EBA4
S224017C60C50201EB82018870284695E7284693E710B500211EE000223F4B03EB40135B6969
S224017C8001EBC10403F82420FE223B4B03EB40135B6901EBC10403EB84035A700023364AB0
S224017CA002EB4012526901EBC10402EB840213624A1CD1B2304A02EB4012927C8A42DADCF9
S224017CC010BD10B52C4B03EB40135B6901EBC10403EB84035A7010BD70B504460E461546B5
S224017CE0254800EB4410007B022801D0012070BD214800EB4410406906EBC60110F82100DC
S224017D0078B31D4800EB4410406906EBC60100EB81004078FE2801D10220E8E72868C0F3DD
S224017D200740EF280CDC144800EB4410406906EBC60100EB81004078296841EA0020286073
S224017D400D4901EB4411897B2868084328600A4901EB4411487B2946FEF7E9FA08B10020A8
S224017D60C5E70FE088330010243A020084C807202C3A020088C807204833001080C80720EB
S224017D80440300100220B2E770B504460D460DB9042070BDFE4800EB4410007B02280FD1E8
S224017DA0FB4901EB4411897B286808432860F84901EB4411487B2946FEF7B9FA0020E8E786
S224017DC00120E6E72DE9D04306460F461446994614B90420BDE8D083ED4800EB4610007BD2
S224017DE0022801D00120F5E7A088C0F30720EF2801D9012000E0002008B10320EAE7FF2F96
S224017E0015D0E34800EB4610406907EBC70110F8210050B1DE4800EB4610406907EBC701B4
S224017E2000EB81004078FE2801D10220D2E7A068082801D90420CDE72078002141EA806097
S224017E40616840EA01202860207A28714FF0000807E0FF21681D00F8081008F1010000F080
S224017E60FF08B8F1080FF4DB681DA268216908F06FF82A4639463046FFF72EFF48B1C44960
S224017E8001EB4611497BC34A52F82100294609F019F800209EE72DE9F04106460C4614B98D
S224017EA00420BDE8F081BA4800EB4610007B022845D1A088C0F30720EF2801D9012000E090
S224017EC0002008B10320ECE7A068082801D90420E7E7AF4901EB4611497BAE4A52F8210067
S224017EE0002108F0CBFF05464DB32279A388C3F307212078002300F0E5FC2860207A287163
S224017F00002704E0FF21681DC155781CC7B2082FF8DB681DA268216908F01AF82946304676
S224017F20FFF732FF48B19A4901EB4611497B994A52F82100294608F0C5FF0020B1E70120DF
S224017F40AFE7934A02EB4012916170470146002004E08F4A02EB40121160401C0228F8DB93
S224017F607047002005E00021894A02EB40121160401C0228F7DB704710B502460020844B90
S224017F8003EB42135B6901EBC10403EB84035B78FE2B00D0012010BD30B5034600207C4CDE
S224017FA004EB4314646901EBC10504EB85046478944200D1012030BD70B504460D4674486F
S224017FC000EB4410406905EBC50100EB8100807898B16F4A02EB4412526905EBC50302EBF4
S224017FE08302918B6A4A02EB4412526905EBC50302EB8302906809F00FF870BD2DE9F84388
S22401800004460E4690460EB9BDE8F883604901EB4411497B5F4A52F82100002108F02EFFF7
S2240180200546002D7ED096F8029030880090B9F1000F00D0E8E70020286008202871BDF896
S2240180400000B0F56E4F77D100270BE00020504901EB4411497B504A02EB411121F8170097
S224018060781CC7B2102FF1DB494800EB4410C07B002860D0464800EB4410007B02285AD1E2
S224018080434800EB4410407C01280AD1404800EB4410837BFF22EE21062000F013FC2860AE
S2240180A006E0FE23FF22EE21062000F00BFC2860374800EB44104168C5F805108068C5F800
S2240180C00900334901EB4411487B2946FEF72FF948B92F4901EB4411497B2E4A52F8210024
S2240180E0294608F0EFFE2A4800EB4410407B2A4901EB4010264901EB4411897B091130F815
S2240181001100234901EB4411897B01F00F020121914008431E4901EB4411497B1E4A02EB96
S224018120411101E046E007E0194A02EB4412927B121121F812003CE0B8F1010F38D11448BE
S22401814000EB4410C07B48B3114800EB4410007B02282DD10023FF22E821062000F0B2FB59
S224018160286001206871FF21A971E971297269723178A9727178E972B1782973044901EB67
S2240181804411487B2946FEF7D2F838B9004906E048330010440300108833001008E001EBF2
S2240181A04411497BFE4A52F82100294608F08AFE00BF00BF00BF27E770B504460D46164695
S2240181C0F84800EB4410006800B970BDF54800EB44103246294603682046984700BFF4E71F
S2240181E010B504462046FEF7BBF810BD2DE9FC4704460D4690464FF0000AFE2D01DBBDE8CE
S224018200FC87B8F1000F00D1F9E7D8F800000090D8F804000190E34800EB4410807BA84258
S22401822078D1E04800EB4410007B022874D1DD4901EB4411081D694600F0B2FBB0B3D94941
S22401824001EB4411497BD64A52F821004FF0FF3108F014FE0746002F76D0D24800EB4410F4
S224018260837BFF22EE21062000F02CFB386008203871CC4800EB44104168C7F8051080686C
S224018280C7F80900C74901EB4411487B3946FEF74EF8002858D1C34901EB4411497BC04AD6
S2240182A052F82100394608F00DFE4DE0FFE70020BC4901EB441148740120BA4901EB441131
S2240182C00873B84901EB4411487BFFF789FF05F00F01012088401FFA80F9B24800EB4410E1
S2240182E0407BB14901EB4010291130F8110040EA0900AC4901EB4411497BAB4A02EB4111B3
S2240183002A1121F81200A74901EB4411087CFFF7EFFB19E016E0FFE7A24800EB4410007FDF
S22401832090B1A04901EB4411081D694600F038FB28B101209B4901EB4411487704E04FF0D4
S224018340010A01E04FF0010ABAF1000F61D005F00F01012088401FFA80F9924800EB44105D
S224018360407B914901EB4010291130F8110040EA09008C4901EB4411497B8B4A02EB411192
S2240183802A1121F8120000263DE0864800EB4410406906EBC60110F8210090B3814A02EB9C
S2240183A04412526906EBC60302EB830202F114017C4A02EB4412526906EBC60302EB830282
S2240183C002F10C006A4600F0A2FBD0B1754800EB4410406906EBC60100EB810045703146E5
S2240183E02046FFF7E9FD6F4800EB4410406906EBC60100EB810000F10C0203212046FFF7F3
S224018400DBFE701CC6B2674800EB4410807CB042BBDC00BFF3E62DE9F04F85B082460D46C9
S22401842015B905B0BDE8F08F2868C0F3006B2868C0F307492888C0F307282F78BBF1000F5A
S22401844000D0EEE7B9F1EF0F75DC0024EEE0554800EB4410007B002862D0524800EB4410FC
S224018460407B50455CD14F4800EB4410807B404557D100264EE04B4800EB4410406906EB3B
S224018480C60110F82100E8B3464800EB4410406906EBC60100EB81004078B84238D131467F
S2240184A02046FFF789FDB9F1EA0F05D10122691D2046FFF7A3FD2AE0286800F0E050000EEE
S2240184C08DF80000394928680840000A019028790290681D04908DF80C808DF80D70314844
S2240184E000EB4410406906EBC60100EB8100006A60B12C4800EB4410406906EBC60200EBEF
S224018500820000E004E0016A6846884700BF00BF701CC6B2234800EB4410807CB042AADC87
S22401852082E0B8F1FF0F6BD1B9F1EA0F04D0B9F1EE0F0DD106E07DE00022691D2046FFF79D
S2240185405DFD5CE06A1D39462046FFF74FFE56E000264DE0134800EB4410406906EBC6014C
S22401856010F82100F0B30F4800EB4410406906EBC60100EB81004078B84237D1314620462F
S224018580FFF71AFD286800F0E050000E8DF80000064928680840000A01902879029007E0A9
S2240185A04403001048330010883300100000FF01681D0490FF208DF80C008DF80D70BD4838
S2240185C000EB4410406906EBC60100EB8100006A40B1B84800EB4410406906EBC60200EBA2
S2240185E0820000E002E0016A68468847701CC6B2B04800EB4410807CB042ABDC00BF13E0E7
S224018600B8F1FE0F10D1B9F1EA0F0CD1687948B9A879EE2806D1E87920B90022691D204605
S224018620FFF7ECFC00BF00BF601CC4B2022CFFF60EAF68E0286800F0E050000E8DF800007B
S2240186402868C0F31020019028790290681D04908DF80C808DF80D700198B0F5704F0AD3D7
S224018660944800EB4410806928B1924800EB4410816968468847002443E08E4800EB44103B
S224018680007BE0B38B4800EB4410407B504536D100262EE0874800EB4410406906EBC601BA
S2240186A010F8210018B3834800EB4410406906EBC60100EB81004078B84218D13146204671
S2240186C0FFF77AFC7B4800EB4410406906EBC60100EB8100006A50B1764800EB4410406948
S2240186E006EBC60200EB8200016A68468847701CC6B2704800EB4410807CB042CADC601C5B
S224018700C4B2022CB9DB00BF8BE670B504460D4629462046FFF77FFE70BD2DE9F041044623
S224018720012718E0A07B4FEA2018A07B00F00F010120884086B2607B5F4901EB401030F864
S22401874018003040B04201D1012700E0002717B1A07B401CA073A07BFE2801DA002FE1D149
S224018760617B564A52F82100002108F087FB05461DB3A37BFF22EE21062000F0A3F82860CF
S224018780082028716068C5F80500A068C5F809000120207700206077607B2946FDF7C7FD09
S2240187A030B9617B454A52F82100294608F08AFBFA214348006808F02FFCBDE8F08170B59C
S2240187C00546002415E03B4800EB4410007B00B90EE0384800EB4410C07B401C354901EB8B
S2240187E04411C873334901EB4410FFF796FF00BF641C022CE7DB70BD70B50646002555E075
S2240188002C4800EB4514207B00B94EE0607F28B12046FFF782FF0020607745E0607B26491D
S22401882001EB4010A17B091130F81100A17B01F00F02012191400840A17B01F00F020121EE
S224018840914088420BD18020A073E17B481CE073207C814228DA2046FFF75FFF24E0012095
S224018860607402202073607B134901EB4010A17B091130F81100A17B01F00F020121914076
S2240188800843617B0C4A02EB4111A27B121121F81200E8B204F10E020021FFF78DFCE8B2D2
S2240188A000220121FFF788FC00BF6D1C022DA7DB70BD000048330010883300104403001021
S2240188C088C8072030B504460D46072C01DD002030BDA10641EA054141EA0221194308466B
S2240188E0F6E7024602B109B900207047C879C009D379B0EBD31F01D00020F6E7C879C0F35C
S2240189000210D379C3F30213984201D00020ECE7C87900F00F00D37903F00F03984201D04E
S2240189200020E2E7887940089379B0EB530F01D00020DAE7887900F00100937903F001034F
S224018940984201D00020D0E748795379984201D00020CAE70879C0081379B0EBD30F01D063
S2240189600020C2E7087900F00700137903F00703984201D00020B8E7488840095388B0EB2E
S224018980531F01D00020B0E70868C0F314001368C3F31403984201D00020A6E70020A4E755
S2240189A0024602B109B900207047C879C009D379B0EBD31F01DD0120F6E7C879C009D37908
S2240189C0B0EBD31F01DA0020EEE7C879C0F30210D379C3F30213984201DD0120E4E7C87932
S2240189E0C0F30210D379C3F30213984201DA0020DAE7C87900F00F00D37903F00F03984294
S224018A0001DD0120D0E7C87900F00F00D37903F00F03984201DA0020C6E788794008937932
S224018A20B0EB530F01DD0120BEE7887940089379B0EB530F01DA0020B6E7887900F00100B3
S224018A40937903F00103984201DD0120ACE7887900F00100937903F00103984201DA0020D7
S224018A60A2E748795379984201DD01209CE748795379984201DA002096E70879C0081379CA
S224018A80B0EBD30F01DD01208EE70879C0081379B0EBD30F01DA002086E7087900F00700AD
S224018AA0137903F00703984201DD01207CE7087900F00700137903F00703984201DA002015
S224018AC072E7488840095388B0EB531F01DD01206AE7488840095388B0EB531F01DA0020EA
S224018AE062E70868C0F314001368C3F31403984201DD012058E70868C0F314001368C3F328
S224018B001403984201DA00204EE700204CE730B503460BB102B109B9002030BDC879C00965
S224018B20DC7900EAD410CC79E409D57904EAD514A04201D00020F0E7C879C0F30210DC79B0
S224018B40C4F302142040CC79C4F30214D579C5F302152C40A04201D00020DEE7CC79D87919
S224018B6000F00F000440C879D57905F00F052840844201D00020D0E7887940089C7900EAF6
S224018B8054008C796408957904EA5504A04201D00020C2E78C79987900F0010004408879ED
S224018BA0957905F001052840844201D00020B4E748795C7920404C7955792C40A04201D044
S224018BC00020AAE70879C0081C7900EAD4000C79E408157904EAD504A04201D000209CE726
S224018BE00C79187900F0070004400879157905F007052840844201D000208EE74888400961
S224018C005C8800EA54104C886409558804EA5514A04201D0002080E708681C68C4F31404AA
S224018C2020400C681568C5F314052C40A04201D0002072E7012070E710B5044673480078BA
S224018C40022800D110BD71490A780978491C6F4B197002EB42116E4A02EB8100842221466E
S224018C6007F0BBF969480078401EC0B2EAE770B504460D4604EB4410654901EB800090F8D2
S224018C807800052800D170BD04EB4411604A02EB810104EB44125E4B03EB820292F878204C
S224018CA002EB420201EBC2001822294607F095F904EB4410564901EB800090F87800401CF7
S224018CC004EB4411524A02EB810181F8780004EB4410114601EB800090F87800401EC0B278
S224018CE0D1E700204949087070477FB5FEF748FEFEF798FC00245DE004EB4411444A02EBBD
S224018D00810191F88200F8F763FD60B904EB44113F4A02EB810191F88200FDF7F8FA3D49A5
S224018D202046FDF742FB04EB4410394901EB800050F8791F02914068039004EB44103449F7
S224018D4001EB800090F882008DF8050002A8009004EB441001EB800090F881008DF8040092
S224018D6004EB441001EB800090F878008DF806006846FEF761FC0546FF2D00D17FBD002609
S224018D800DE004EB4410224A02EB800006EB460200EBC2012846FEF7F7FE701CC6B204EB92
S224018DA044101B4901EB800090F87800B042E8DC601CC4B21548007884429DDBFEF78BFC52
S224018DC000BFDBE710B5FDF712FBFFF78EFF10BD10B5002404E02046FDF7A3FA601CC4B240
S224018DE0022CF8DB002407E02046FEF741FF2046FEF74CFC601CC4B2022CF5DB10BD10B5A1
S224018E00FFF7E6FFFDF71DFB10BD00008CC80720F83300100B870100FE4A1070FE4A1170BE
S224018E20704770477CB5FD4C2078012806D002286AD0032877D0042874D176E1F849F54A8F
S224018E401278895CF74A52F82100002108F016F80546002D57D0F448286008202871012085
S224018E6068730020C5F80500C5F809006078022802D12020687104E06078012801D1102094
S224018E80687194F80417A971B4F804070112E971B4F80407072190FBF1F02872B4F8040772
S224018EA090FBF1F201FB120010B1287A401C28726078022802D1FF21697201E0297A6972A8
S224018EC0A178A97260880112E972002129732A46D1480178CF480078FEF7FEFE48B907F0CB
S224018EE0C1FF606002202070207A40F00100207209E0CB49C74A1278895CCA4A52F82100E1
S224018F00294607F0DFFF1AE16078022806D06078012805D1207A00F0020008B10320207065
S224018F200DE100E00AE1607802287BD107F09AFF6168421ABD4800884CF250314843BC4993
S224018F4009884CF25033594300EB214082425CD9B349B04A1278895CB24A52F821000021EB
S224018F6007F08CFF0546002D4FD0B248286008202871012068730020C5F80500C5F80900EB
S224018F80B4F80207072190FBF1F0401C687194F80C0728B1B4F80217D4F80807461804E0F3
S224018FA0B4F8021704F109000E183068CDF80100B088ADF80500B0798DF807002A4696487F
S224018FC0017894480078FEF787FE00BBB4F80207C0F1FF00072803DAFF20A4F8020704E070
S224018FE0B4F80207C01DA4F8020794F80E07401C84F80E07B4F80207B4F80417884201DB84
S2240190000420207007F02EFF60608DE00AE08449804A1278895C834A52F82100294607F0B7
S22401902051FF81E0607801287ED1207A00F00200002873D07A49774A1278895C794A52F832
S2240190402100002107F01AFF0546002D6CD07948286008202871012068730020C5F805001C
S224019060C5F80900B4F80207072190FBF1F0401C687194F80C0728B1B4F80217D4F808078E
S224019080461804E0B4F8021704F109000E183168C5F80610B1886981B17929732A465E4834
S2240190A001785C480078FEF717FE58BBB4F8020740F2F961081A072803DA0846A4F8020796
S2240190C004E0B4F80207C01DA4F8020794F80E07401C84F80E07B4F80207B4F8041788429B
S2240190E002DB0420207009E094F80E0794F80D17884203D1207A20F00300207207F0B2FE1B
S224019100606011E04649434A1278895C454A52F82100294607F0D6FE06E0FFE7207A00F083
S224019120010008B107F09EFE09E06078022804D12046FFF776FE0020207000E000BF00BF3E
S2240191407CBD70B5044660880512D72D03D0D82D01D0D92D08D194F80F37B4F80427608845
S22401916004F1090100F02DFB70BD2DE9F04781460D46174609F47F40B0F56C4F7DD12878D7
S22401918010281DD0112804D0132877D0202876D193E0224C6879A97940EA012061888842A4
S2240191A00DD194F80F07B84209D1687884F80D07207A40F002002072002084F80E07A7E04F
S2240191C01D4C2078002877D11549124A1278895C144A52F82100002107F050FE0646002E46
S2240191E069D01648306008203071012070730020C6F80500C6F80900B4F80207072190FB63
S224019200F1F0401C7071012020706879A97940EA012015E0B6030010B7030010103C001047
S22401922080C80720440300100000EC188C3A02008E3A02000000EB14003500100000EC1C80
S22401924060806878A97840EA0120A4F804070020A4F802070120607084F80F7707F002FE86
S224019260606004202072002084F80E0784F80D07112070710A21B17102E04AE038E046E088
S22401928094F80E17F1716979B172A979F172E979317332469D4801789D480078FEF71CFDE4
S2240192A048B19C499A4A1278895C9B4A52F82100314607F007FE00BF2AE0984C2078B0B906
S2240192C0012020706879A97940EA012060806878A97840EA0120A4F804070020A4F80207F1
S2240192E00220607084F80F7707F0BCFD60600FE08B4C2078042809D16078012806D10420A4
S22401930020702046FFF78DFD0020207000E000BFC1E009F47F40B0F56B4FF9D17F4C94F8A5
S2240193200F07B842F4D107F09DFD6060287884F80E0794F80D07401C84F80D072878401E46
S224019340C0EBC000A4F802074FF001080DE015F80810B4F80227501CA4F8020704F10900B9
S224019360815408F1010000F0FF08B8F1080F05DAB4F80207B4F804178842E8DBB4F80207C4
S224019380B4F80417884247DB607801283ED161495F4A1278895C604A52F82100002107F015
S2240193A06DFD06468EB35F48306008203071012070730020C6F80500C6F8090013207071EE
S2240193C094F80417B171B4F804070112F17194F80E173172FF217172A178B1726088011204
S2240193E0F1720021317332464848017848480078FEF772FC48B14749454A1278895C464A3C
S22401940052F82100314607F05DFD00BF002020702046FFF796FE3EE094F80D070A283AD1B9
S2240194203C493B4A1278895C3B4A52F82100002107F024FD06466EB33A483060082030713C
S224019440012070730020C6F80500C6F8090084F80D07112070710A21B17194F80E07401C6C
S224019460F071A178B17260880112F1720021317332462648017826480078FEF72DFC48B1CA
S2240194802449234A1278895C234A52F82100314607F018FD00BFBDE8F0872DE9F0410546B5
S2240194A00C4617461E46DDF818801D48007858BBB8F1000F09D140F2F960844205DC22460A
S2240194C029461748093006F043FD1548A0F8044700201349A1F8020708464780FF2E02D1D6
S2240194E00220487002E001200D4948700C4880F80F6780F80C870120094908700846C0F83D
S22401950008570120BDE8F081FF20FBE7B7030010B603001080C80720440300100035001010
S224019520103C00100000EC1C2DE9F04107460C4615464FF6FF7600220821104606F083F9B3
S22401954029462046F7F75CFC01220821002006F07AF93046BDE8F08110B5FE48007C0028DA
S2240195607ED0FC48007C0628FAD0FA48007C0328F6D0F848807C002872D1F648007C0128A6
S22401958004D0052852D008286BD19FE041F28830F049088307F066FCEE4948610846C07849
S2240195A0022802D10320087402E00820E9490874E848007C082838D0E749E84A1278895C9C
S2240195C0E74A52F82100002107F058FC044664B3E44820600820207101206073FF22082179
S2240195E0601D06F02CFDDB4800786071D9480088E02101EAE001A171A07940F01101A17168
S2240196002246D9480178D5480078FEF765FB60B1D149D24A1278895CD14A52F821002146B5
S22401962007F050FC0120CB4908748AE0C948C078022808D1C748028800F12901FFF774FF5D
S2240196400120C449C870C449C44A1278895CC44A52F82100002107F011FC0446ACB301E0EC
S22401966070E069E0BF4820600820207101206073FF220821601D06F0E2FCB6480078607135
S224019680B4480088E02101EAE001A171A07940F01901A1710021E17221730620AD4908744C
S2240196A02246B1480178AD480078FEF715FB60B1A949AA4A1278895CA94A52F8210021462D
S2240196C007F000FC0520A34908743AE007F0CAFBA0494861A049A14A1278895CA04A52F825
S2240196E02100002107F0CAFB044624B39D4820600820207101206073002060711B21A171F4
S2240197000021E172217306209249087422469648017892480078FEF7DFFA60B18E498F4A1E
S2240197201278895C8E4A52F82100214607F0CAFB08208849087404E000208649087488748E
S22401974000BF37E08348007C062814D1874800888749484387490988854A514300EB214011
S2240197607C494969844A1268511A884203D20020784908741EE07748007CD8B107F072FB97
S22401978074494969421A7348008B4FF47A7148437649098841436F48008B4FF47A73584318
S2240197A0744B1B88584301EB2040824202D900206849087410BD10B507F054FB654948613F
S2240197C010BD2DE9F04780460C4691461F466078C0F3420608F47F48B8F5574F06D0B8F5A9
S2240197E0584F27D0B8F5594F23D124E05948007C03281ED15748407BB8421AD194F80090E6
S224019800B9F1FF0F03D15348B0F8009002E05148A0F80090641C4A4621464E48293006F0E4
S22401982097FB07F01FFB4B4948610520087400208874F4E0F3E04748407BB84239D0454804
S224019840007C98B34449454A1278895C444A52F82100002107F012FB054645B3414828603E
S22401986008202871012068730020C5F80500C5F80900012068711321A971FF220621E81DE8
S22401988006F0DDFB2A463848017834480078FEF723FA48B13049314A1278895C304A52F865
S2240198A02100294607F00EFBBDE8F08701E0FFE700BF2848007C0B284BD2DFE800F0063542
S2240198C036ADAD37797A38AD390001202149087407F0C8FA1F4948610846C67020786178E4
S2240198E001F0E00140EAC1001A4908806078C0F300108870A078E17840EA0120217940EAA7
S22401990001401449886060790873A079E17940EA0120104988800020887408464773042EF2
S22401992001D10020087478E000BF00BF00BF74E0062E3CD107F096FA064948610846C67086
S224019940A079E17940EA0120024988802078617814E061E01C4A001080C80720B60300109C
S224019960440300100000D81CB70300108C3A0200A08601008E3A0200883A020001F0E0017D
S22401998040EAC1002B4908806078C0F300108870A078E17840EA0120217940EA0140254918
S2240199A08860607908730B2008740846477334E000BF042E0AD11F4880681E49C8610020D7
S2240199C0087407F04FFA1B49486124E0012E22D107F048FA17494969401A64281BD2012053
S2240199E01449087407F03EFA124948610846C6706078C0F300108870A078E17840EA012082
S224019A00217940EA01200B49886060790873002088740846477300E000BF00BF00BF00BFCB
S224019A2000BF41E7002003498874704700200149887470471C4A00102DE9F04106460F469F
S224019A40052E11D137B1012F06D0022F06D0032F07D104E03E4C06E03E4C04E000BF3E4CE1
S224019A6001E0002400BF2FE036B1012E09D0022E0CD0042E14D10EE0032000F021FA054694
S224019A8011E0022000F01CFA05460CE0012000F017FA054607E0042000F012FA054602E0CF
S224019AA00020BDE8F08100BF25B1012D04D0022D06D103E0294C05E0294C03E0294C01E0E2
S224019AC0002400BF00BF00BF2046EAE770B50446012C06D0022C11D0032C1CD0042C34D117
S224019AE026E000210220FFF7A7FF05464FF0814109F086FC1C49C1F8300426E0002101201A
S224019B00FFF79AFF05464FF0814109F079FC1649C1F8340419E000210846FFF78DFF054671
S224019B204FF0814109F06CFC0F49C1F838040CE000210420FFF780FF05464FF0814109F085
S224019B405FFC0949C1F83C0400BF00BF70BD000014AE233B99996D3B3333113C2495CE3A40
S224019B60C4B0433B9B3DD03B44C907202DE9F04781460C46B9F1010F09D0B9F1020F0CD046
S224019B80B9F1030F0FD0B9F1040F18D111E000250E26E44880F8754013E008250126E1486B
S224019BA080F876400DE00F250426DE4880F8774007E009250A26DB4880F8784001E0BDE8B3
S224019BC0F08700BF44B1012C02D0022C0BD106E001274FF0000807E00027B84604E00027DF
S224019BE04FF0010800E0EAE700BF3A462946012005F029FE42463146012005F024FE4846B6
S224019C00FFF764FF00BFDAE770B505460C4624B1012C07D0022C0FD109E000212846FFF74E
S224019C20A5FF0AE001212846FFF7A0FF05E002212846FFF79BFF00E070BD00BF00BFFBE7F8
S224019C4008B50020034602460146009005F034FE00200346024601210090084605F02CFEC2
S224019C6000200346024604210090012005F024FE00200346024608210090012005F01CFEA6
S224019C8000200346024609210090012005F014FE0020034602460A210090012005F00CFE9F
S224019CA00020034602460E210090012005F004FE0020034602460F210090012005F0FCFD96
S224019CC000200346024603210090022005F0F4FD00200346024604210090022005F0ECFDAB
S224019CE000200346024605210090022005F0E4FD0020034602460B210090022005F0DCFDA2
S224019D000020034602460C210090022005F0D4FD0020034602460D210090022005F0CCFD98
S224019D2001220021104605F074FD01221146104605F06FFD01220421104605F06AFD0122CF
S224019D400821104605F065FD01220921104605F060FD01220A21104605F05BFD01220E21EF
S224019D60104605F056FD01220F21104605F051FD01220321022005F04CFD01220421022042
S224019D8005F047FD01220521022005F042FD01220B21022005F03DFD01220C21022005F0DE
S224019DA038FD01220D21022005F033FD5D4890F875100120FFF728FF5A4890F8761002200E
S224019DC0FFF722FF574890F877100320FFF71CFF544890F878100420FFF716FF08BD70B5BF
S224019DE00546062D64D2DFE805F003132333435300220B21022005F026FD00220C210220F2
S224019E0005F021FD00220D21022005F01CFD4FE001220B21022005F016FD00220C21022090
S224019E2005F011FD00220D21022005F00CFD3FE000220B21022005F006FD01220C210220B0
S224019E4005F001FD00220D21022005F0FCFC2FE001220B21022005F0F6FC01220C210220D1
S224019E6005F0F1FC00220D21022005F0ECFC1FE000220B21022005F0E6FC00220C210220F4
S224019E8005F0E1FC01220D21022005F0DCFC0FE001220B21022005F0D6FC00220C21022012
S224019EA005F0D1FC01220D21022005F0CCFC00BF00BF002401E000BF641C0A2CFBD370BDB7
S224019EC00146012906D0022908D003290AD0042910D10BE0134A92F875000BE0114A92F807
S224019EE0760007E00F4A92F8770003E00D4A92F8780000BF00BF704738B504460020034694
S224019F0002460621009005F0D7FC01220621002005F07FFC84F001020621002005F093FC58
S224019F2038BD000044C907200146FF2901D102207047FB2903DBFE2901DC0020F8E70120B2
S224019F40F6E70146B1F57F4F05DB4FF6FE70814201DA02207047B1F57B4F04DBB1F57F4F96
S224019F6001DA0020F6E70120F4E70146B1F17F4F04D311F1030F01D802207047B1F17B4F47
S224019F8004D3B1F17F4F01D20020F6E70120F4E70146072901D1022070470120FCE701463B
S224019FA0032901D102207047022901D10020FAE70120F8E7642006F001FF00BFBFF34F8FFD
S224019FC00648006800F4E06005490843001D03490860BFF34F8F00BF00BFFEE70CED00E05B
S224019FE00000FA05F8480078022800D17047F64801780078401CF44A10700846F6E710B5B9
S22401A00000EBC003F14C04EBC303CA681A6100EBC00304EBC3030A69DA6000EBC0030A68BD
S22401A02044F8332000EBC00304EBC3034A685A6000EBC00304EBC3038A685A614FF07E529D
S22401A04000EBC00304EBC303DA6100EBC00304EBC3031A6200EBC00304EBC3035A6200EB73
S22401A060C00304EBC3039A6200EBC00304EBC303CA681A6300EBC00304EBC3030A69DA6242
S22401A08000EBC00304EBC3034A695A630A7E00EBC00304EBC30383F83820012200EBC00358
S22401A0A004EBC30383F83C20002300EBC00204EBC20282F8443000EBC00204EBC2021364C6
S22401A0C010BD2DE9F04104460E4615461F4604EBC400BE4901EBC000C66104EBC40001EBDC
S22401A0E0C000056204EBC40001EBC000476204EBC401B64A02EBC101C86A294609F022F814
S22401A10004EBC401B14A02EBC101C86004EBC40102EBC101086B294609F014F804EBC401B5
S22401A120AA4A02EBC1010861BDE8F08100EBC002A64B03EBC202916270472DE9F04F87B071
S22401A14004460E4617463146384609F061FA054604EBC4009D4901EBC00090F83C00012838
S22401A16015D1012104EBC400984A02EBC00080F84410002004EBC40102EBC10181F83C008B
S22401A18004EBC400114601EBC00005642DE004EBC4008E4901EBC00090F8440028B304EBC1
S22401A1A0C4018A4A02EBC101086C08F031FF21F00041874A874BCDE9000108F0FFFCCDE960
S22401A1C00401284608F024FF21F00041CDE90201DDE9042308F0B6FC07D2002104EBC4009C
S22401A1E07A4A02EBC00080F8441004EBC401774A52F83100294609F003F9059004EBC40080
S22401A200724A02EBC000C169059809F0F9F8804604EBC4006D4901EBC00090F8440028B19E
S22401A22004EBC40001EBC00085600EE004EBC401664A02EBC1018868294608F015FF04EB79
S22401A240C401624A02EBC101886004EBC4025F4B03EBC202D16804EBC40203EBC202906847
S22401A26009F09AF90CD204EBC400584901EBC000C06804EBC401554A02EBC101886019E063
S22401A28004EBC402514B03EBC202116904EBC40203EBC202906809F07FF80BD204EBC400DC
S22401A2A04A4901EBC000006904EBC401474A02EBC101886004EBC402444B03EBC202916825
S22401A2C004EBC40203EBC202506809F099F8049004EBC4003D4A02EBC000016A049809F054
S22401A2E08FF8059004EBC400384A02EBC000416B059809F085F8824604EBC400334A02EBB6
S22401A300C0008169304609F083F904EBC40203902E4800EBC2004169039809F071F804EBA1
S22401A320C4020490294800EBC200416A049809F067F8059004EBC400244A02EBC000416BF1
S22401A340059808F0FFFE814604EBC4001F4901EBC00086615146404608F086FE4946049034
S22401A36009F056F904EBC4020590184800EBC200816A059809F044F883461749584609F0BB
S22401A3800BF902D2DFF850B006E01449584609F003F801D2DFF844B0584607B0BDE8F08F1C
S22401A3A02DE9FE4F04460D46164604EBC400074901EBC00090F8380090B13246294620463E
S22401A3C0FFF7BBFEBDE8FE8FB803001000DD07209A9999999999D93F00007A4400007AC41C
S22401A3E02946304609F014F9029004EBC401874A52F83100029909F003F8834604EBC400CF
S22401A400824A02EBC000C169584608F0F9FF074604EBC4017D4A02EBC1018868029908F00B
S22401A42023FE04EBC401794A02EBC101886004EBC402764B03EBC202D16804EBC40203EBE3
S22401A440C202906809F0A8F80CD204EBC4006F4901EBC000C06804EBC4016C4A02EBC1016B
S22401A460886019E004EBC402684B03EBC202116904EBC40203EBC202906808F08DFF0BD2A1
S22401A48004EBC400614901EBC000006904EBC4015E4A02EBC101886004EBC4025B4B03EB08
S22401A4A0C202116A04EBC40203EBC202906808F0A7FF019004EBC400544A02EBC000416822
S22401A4C0019808F09DFF834604EBC4004F4A02EBC000416B584608F093FF814604EBC40039
S22401A4E04A4A02EBC0008169284609F091F8009004EBC400454A02EBC0004169009808F082
S22401A5007FFF019004EBC400404A02EBC000416A019808F075FF834604EBC4003B4A02EB9E
S22401A520C000416B584608F00DFE804604EBC400364901EBC00085614946384608F094FDE8
S22401A5404146019009F064F8834604EBC4002F4A02EBC000816A584608F052FF82462C49D7
S22401A560504609F019F802D2DFF8A4A006E02949504608F011FF01D2DFF898A0504621E7D0
S22401A58070B504460E46154604EBC4001F4A02EBC000C168284608F0FFFF06D204EBC400B6
S22401A5A01A4901EBC000C5680FE004EBC400174A02EBC0000169284608F0EEFE05D204EB27
S22401A5C0C400124901EBC000056904EBC4000F4901EBC000856004EBC40001EBC00086615A
S22401A5E0012004EBC401094A02EBC10181F83C00002104EBC40002EBC00080F8441004EB8D
S22401A600C40002EBC000016470BD000000DD072000007A4400007AC42DE9F04104460D464D
S22401A620FE49B1F8CA10491B601A08F089FE8046FB480168404608F0E3FE0746F94908F095
S22401A64013FD064608F040FE00B2BDE8F08103B595B0F24890F8BD000D9008F089FEF249C7
S22401A6600E9008F0CDFE0F9008F0D2FC21F00041CDE9100107F098FF1490E848B0F84600A5
S22401A680109008F075FEE949119008F05BFDE849086008460168002008F0BAFFE4490860D0
S22401A6A0DE48B0F84400109008F062FEDF49119008F048FDDF490860D848B0F8420010904A
S22401A6C008F056FED949119008F03CFD80F000401390D248B0F84800109008F049FED349DC
S22401A6E0119008F02FFD1290CC48B0F85600109008F03EFED049119008F082FE1599C1EB7B
S22401A700C10101EB4101CD4A02EB8101C860C348B0F85400109008F02BFEC749119008F024
S22401A7206FFE1599C1EBC10101EB4101C34A02EB81018860159810B101287DD156E0B748DE
S22401A74090F873000D9008F013FEB7490E9008F057FE0F9008F05CFC21F00041CDE910015F
S22401A76007F022FF1490AD48B0F84C104FF6FF7000EA81011598C0EBC00000EB4000AF4AC2
S22401A78002EB8000A0F84810A448B0F850004FF6FF7101EA80011598C0EBC00000EB40000E
S22401A7A002EB8000A0F84A109C48B0F84E004FF6FF7101EA80011598C0EBC00000EB4000F6
S22401A7C002EB8000A0F84C10944890F8520008B1012100E000211598C0EBC00000EB40003D
S22401A7E0964A02EB800080F84E1059E08B4890F8BD000D9008F0BCFD8B490E9008F000FE29
S22401A8000F9008F005FC21F00041CDE9100107F0CBFE14908148B0F8B6004FF6FF7101EA56
S22401A82080011598C0EBC00000EB4000834A02EB8000A0F8481000E031E07848B0F8BA0011
S22401A8404FF6FF7101EA80011598C0EBC00000EB400002EB8000A0F84A107048B0F8B80017
S22401A8604FF6FF7101EA80011598C0EBC00000EB400002EB8000A0F84C10684890F8BC0019
S22401A88008B1012100E000211598C0EBC00000EB40006A4A02EB800080F84E1000E000BFFD
S22401A8A000BF1598C0EBC00000EB4000634901EB800090F84E00002869D0DDE91401C1EBBA
S22401A8C0C10101EB41015D4A02EB810148601698002849D01598C0EBC00000EB400011463B
S22401A8E001EB8000C068059008F092FBCDE90801149808F08DFBCDE9000107F023FECDE934
S22401A90004011598C0EBC00000EB40014B4800EB81008068019008F07BFBCDE90201DDE983
S22401A920042307F02FFFCDE90601DDE9082307F06DFECDE90C011598C0EBC00000EB4001AE
S22401A9403E4800EB81008068099008F061FBCDE90A01DDE90C2307F015FFCDE90E0106F0AE
S22401A96069F881F0004105E0149880F000400F9008F04EFBCDE9100107F016FE1599C1EB71
S22401A980C10101EB41012D4A42F8210079E0149880F000411598C0EBC00000EB4000274A85
S22401A9A042F820101698B8B31598C0EBC00000EB4001104600EB8100C068059008F028FB30
S22401A9C0CDE90801149808F023FBCDE9000107F0B9FDCDE904011598C0EBC00000EB40008E
S22401A9E0164901EB80008068019008F011FBCDE90201DDE9042307F0C5FECDE90601DDE926
S22401AA00082307F003FECDE90C011598C0EBC00000EB4001094813E023E0000044C907208B
S22401AA20E403001000007AC435FA8E3C0000C842BC030010C00300100AD7233C90DD072062
S22401AA4000EB81008068099008F0E2FACDE90A01DDE90C2307F096FECDE90E0105F0EAFF4B
S22401AA6002E0149808F0D4FACDE9100107F09CFD1599C1EBC10101EB4101FE4A02EB810124
S22401AA8048601598C0EBC00000EB4000F94901EB8000C0684FF08041119008F053FB15995A
S22401AAA0C1EBC10101EB4101F24A02EB810108611598C0EBC00000EB4000114601EB8000DA
S22401AAC000690B9008F0A4FACDE90E01149808F09FFACDE9060107F035FDCDE90A01159880
S22401AAE0C0EBC00000EB4000E24901EB80008068079008F08DFACDE90801DDE90A2307F07C
S22401AB0041FECDE90C01DDE90E2307F07FFDCDE9100107F049FD1599C1EBC10101EB410175
S22401AB20D44A02EB810188611598C0EBC00000EB4000114601EB8000806901460F90CE48AE
S22401AB4008F000FBCD49109008F08EFA119008F0D7FB81B21598C0EBC00000EB4000C54AD6
S22401AB6002EB800081821598C0EBC00000EB4000114601EB8000806901460F90BE4808F08C
S22401AB80E1FABE49109008F038FD119008F0B8FB81B21598C0EBC00000EB4000B54A02EB52
S22401ABA08000C1821598C0EBC00000EB4000114601EB8000B0F84C101598C0EBC00000EBBF
S22401ABC0400002EB8000B0F84A00081A0F9008F0B7FB11901598C0EBC00000EB4001A54893
S22401ABE000EB8100406800210F9008F011FD1090119908F0A7FA1599C1EBC10101EB410148
S22401AC009C4A02EB8101C8611598C0EBC00000EB4000114601EB8000B0F84A101598C0EB50
S22401AC20C00000EB400002EB8000B0F84800081A0F9008F085FB11901598C0EBC00000EBE9
S22401AC4040008C4951F8200001460F90002008F0DFFC1090119908F075FA1599C1EBC101CA
S22401AC6001EB4101834A02EB810108621598C0EBC00000EB4000114601EB8000818A15983C
S22401AC80C0EBC00000EB400002EB8000C08A081A109008F055FB01461190794808F052FA6A
S22401ACA01599C1EBC10101EB4101724A02EB810148631598C0EBC00000EB4000114601EBE8
S22401ACC08000406800210F9008F0A2FC11901598C0EBC00000EB4000664901EB8000808AE7
S22401ACE0A0F5FB400F9008F02BFB1090119908F029FA1599C1EBC10101EB41015D4A02EB7E
S22401AD00810188631598C0EBC00000EB4000114651F8200001460F90002008F079FC1190A9
S22401AD201598C0EBC00000EB4000524901EB8000C08AC0F5FB400F9008F002FB10901199AB
S22401AD4008F000FA1599C1EBC10101EB4101494A02EB8101C8631598C0EBC00000EB400041
S22401AD60114601EB800040680021109008F050FC01461190434808F0E5F91599C1EBC101F8
S22401AD8001EB41013B4A02EB810108641598C0EBC00000EB4001104650F821000146109035
S22401ADA0002008F035FC01461190364808F0CAF91599C1EBC10101EB41012E4A02EB8101F2
S22401ADC048641598C0EBC00000EB4001104600EB8100B0F84C101598C0EBC00000EB400074
S22401ADE002EB8000B0F84A00081A0F9008F0A8FA11901598C0EBC00000EB40011D4800EB5E
S22401AE008100808AA0F5FB400F9008F099FA1090119908F097F91599C1EBC10101EB41018B
S22401AE20144A02EB810148621598C0EBC00000EB4000114601EB8000B0F84A101598C0EB35
S22401AE40C00000EB400002EB8000B0F84800081A0F9008F075FA11901598C0EBC00000EBD8
S22401AE604001044800EB8100C08AC0F5FB400F900AE0000090DD072000007A450000FB467C
S22401AE800000FA4400007A4408F05AFA1090119908F058F91599C1EBC10101EB4101FB4A42
S22401AEA002EB810188621598C0EBC00000EB4000114601EB8000B0F84C101598C0EBC00011
S22401AEC000EB400002EB8000B0F84A00081A109008F036FA01461190ED4808F033F9159909
S22401AEE0C1EBC10101EB4101E84A02EB8101C8621598C0EBC00000EB4000114601EB8000DF
S22401AF00B0F84A101598C0EBC00000EB400002EB8000B0F84800081A109008F011FA01467D
S22401AF201190DB4808F00EF91599C1EBC10101EB4101D64A02EB81010863D64801681398D2
S22401AF4008F066FBD249119008F0FCF8D2490860D2480168129808F05BFBCD49119008F03D
S22401AF60F1F8CF4908601598C0EBC00000EB4000C64901EB8000B0F848101598C0EBC0008C
S22401AF8000EB4000C14A02EB8000B0F84C00814201DD012100E000211598C0EBC00000EB4D
S22401AFA04000BA4A02EB800080F84F10BD48B0F8C410B0F8C000081A109008F0C1F9B449A9
S22401AFC0119008F0BFF8B8490860B648B0F8C210B0F8C400081A109008F0B2F9AC491190D3
S22401AFE008F0B0F8B1490860AE48B0F8C610B0F8C000081A109008F0A3F9A549119008F090
S22401B000A1F8AB490860A748B0F8C210B0F8C600081A109008F094F99D49119008F092F80E
S22401B020A44908609F48B0F8C810B0F8C000081A109008F085F99649119008F083F89E49D4
S22401B04008609848B0F8C210B0F8C800081A109008F076F98E49119008F074F8974908606B
S22401B0609048B0F8CC10B0F8CA00081A109008F067F901461190924808F064F8914908608A
S22401B080884890F8E400632803DD0021854880F8E4108448B0F8CE0000210C90FFF7BCFAFE
S22401B0A00D9007F024FD02460B46CDE90E010020854900F065FCCDE9100107F075FA83493F
S22401B0C008607848B0F8D00000210C90FFF7A4FA0D9007F00CFD02460B46CDE90E0100205E
S22401B0E07B4900F061FCCDE9100107F05DFA7749486017B000BD2DE9F04104460D46C4EBA5
S22401B100C40101EB4101614A02EB8101C98A681A08F016F98046C4EBC40000EB40005B4A37
S22401B12002EB8000416B404608F06AF90746694907F09AFF064608F0C7F800B2BDE8F081B5
S22401B1402DE9F04104460D460021284608F024F91FD2C4EBC40000EB40004C4A52F82010C2
S22401B160284608F055FA8046C4EBC40000EB4000464A02EB8000416C404608F041F9074601
S22401B180544907F071FF064608F09EF800B2BDE8F0810021284608F0FFF918D2002128460B
S22401B1A008F036FA8046C4EBC40000EB4000374A02EB8000016C404608F022F9074600219B
S22401B1C007F052FF064608F07FF800B2DFE70020DDE70246C2EBC20000EB40002B4B03EBC4
S22401B1E0800090F84F0058B1C2EBC20000EB400003EB8000B0F84A0088420EDA0020704766
S22401B200C2EBC20000EB4000204B03EB8000B0F84A00884201DD0020F1E70120EFE72DE916
S22401B220F04704460D4629462046FFF7D2FF60BBC4EBC40101EB4101144A02EB8101B1F865
S22401B2404810681A08F07CF88146C4EBC40000EB40000E4A02EB8000816A484608F0D0F83F
S22401B2600746C4EBC40101EB4101084A02EB8101C88A08F07DF88046394607F0F5FE0646DE
S22401B28008F03EF880B2BDE8F08725E090DD072000007A44BC030010C4030010C00300105C
S22401B2A0C803001044C90720CC030010D0030010D4030010D8030010DC030010E003001003
S22401B2C00000FA44E403001000408FC0E803001000408F4000007AC4C4EBC40101EB4101BA
S22401B2E0DC4A02EB8101B1F84A10681A08F028F88046C4EBC40000EB4000D64A02EB800025
S22401B300416A404608F07CF80746D34907F0ACFE064607F0F5FF80B2BDE8F0872DE9F047AE
S22401B32004460D460021284608F036F82AD2C4EBC40000EB4000C74A52F82010284608F02A
S22401B34067F98146C4EBC40000EB4000C14A02EB8000C16B484608F053F80746C4EBC401EC
S22401B36001EB4101BB4A02EB8101C88A08F000F88046394607F078FE064607F0C1FF80B2FC
S22401B380BDE8F0870021284608F042F98046C4EBC40000EB4000AF4A02EB8000816B40468D
S22401B3A008F02EF80746AC4907F05EFE064607F0A7FF80B2E4E72DE9F04104460D4629469B
S22401B3C02046FFF706FF20BBC4EBC40101EB4101A04A02EB8101B1F84810681A07F0B0FF07
S22401B3E00746C4EBC40000EB40009A4A02EB8000016A384608F004F80646C4EBC40000EB84
S22401B4004000944A52F82010304607F02DFEBDE8F081C4EBC40101EB41018E4A02EB8101F7
S22401B420B1F84A10681A07F08BFF0746C4EBC40000EB4000874A02EB8000C169384607F038
S22401B440DFFF0646002107F00FFEE0E72DE9F04104460D4629462046FFF7BBFE08BBC4EBF6
S22401B460C40101EB41017B4A02EB8101B1F84810681A07F065FF8046C4EBC40000EB40005D
S22401B480744A02EB8000016B404607F0B9FF0746724907F0E9FD064607F016FF00B2BDE846
S22401B4A0F081C4EBC40101EB41016A4A02EB8101B1F84A10681A07F043FF8046C4EBC40059
S22401B4C000EB4000634A02EB8000C16A404607F097FF0746002107F0C7FD064607F0F4FE85
S22401B4E000B2DCE75E49016070472DE9F0410546002D14DA284607F023FF8046574908F080
S22401B50087F8074657480168384607F079FF064655480168304607F0A7FD044617E0002D93
S22401B52014DD284607F00CFF8046002108F070F807464E480168384607F062FF06464C485B
S22401B5400168304607F090FD044600E000242046BDE8F0812DE9FC5F04464648B0F8C050B7
S22401B560B0F8C460444807684448D0F80080414890F82C040A281ED13649D1F8A400404953
S22401B58007F00AFF08D23B48B0F8C6603D4807683D48D0F800800EE02E49D1F8A4003B4963
S22401B5A007F0FAFF07D23348B0F8C860384807683848D0F80080002C18DA204607F0C0FE81
S22401B5C02649009008F024F88346394607F018FF8246284607F0CCFE5146019007F044FDA5
S22401B5E0814607F08DFE80B2BDE8FC9F204607F0A7FE0021009008F00BF88346414607F095
S22401B600FFFE8246304607F0B3FE5146019007F02BFD814607F074FE80B2E5E72DE9F04185
S22401B62004462046FFF761FF07461B4907F0E8FE064607F049FE05B22846FFF78BFFBDE89C
S22401B640F081C0EBC00202EB4202024B03EB82021165704790DD07200000FB4600007AC4D6
S22401B660E8030010C4030010BC030010C8030010C003001044C90720CC030010D00300107F
S22401B680CDCC4CBED4030010D8030010CDCC4C3EDC030010E0030010000020417A48B0F85F
S22401B6A04600642190FBF1F0404240B2774908707548B0F84200642190FBF1F0404240B295
S22401B6C07249087291F90010704A92F90820881800EBD071491049B26C4A11716A48B0F876
S22401B6E04400642190FBF1F040B2114608736648B0F84800642190FBF1F040B211460875F6
S22401B70091F90C1092F91420881800EBD071491049B25E4A11745C48B0F8B2001146488054
S22401B7205948B0F8AE101046C1805748B0F8AA10104641815448B0F8AC101046C18152481A
S22401B740B0F8B010104641824F48B0F8B4101046C1824189C088081A00B2114608830846B0
S22401B760418AC089081A1146098B084400B211460883B1F9180000EBD07149101183704730
S22401B78010B5FFF78BFF10BD2DE9F04F87B006460D460024002008E03C4901EB800191F9BE
S22401B7A00010A94200DAC4B2401C0528F4DB374901EB840191F9000007F0C2FD0490334A9E
S22401B7C0611C02EB810191F9000007F0B9FD03902E4901EB8401B1F9020007F0B1FD0290E2
S22401B7E02A4A611C02EB8101B1F9020007F0A8FD0190284607F0A4FD8346049907F008FFA0
S22401B8008146DDE9030107F003FF8346DDE9010107F0FEFE5946009007F094FC8246494607
S22401B82007F0EEFD8046029907F01EFC074607F04BFD00B20590144991F8F90007F098FD70
S22401B8401349009007F07EFC82464FF07E5107F0D4FE81460D48B0F91870002F01DB39460F
S22401B86000E07942084607F06BFD8346494607F0C7FD804607F028FD0690DDE90501C6E974
S22401B880000107B0BDE8F08F44C9072038DE07200000C84208B50020034602221A21009036
S22401B8A004F00AF801221A21002003F0B2FF044803F071FB0021024803F074FB08BD00002D
S22401B8C000C0084002468A4201DD104670470846FCE702468A4201DA104670470846FCE7FD
S22401B8E02DE9F04104460D4616461F4632463B462046294607F060FA03D220462946BDE82F
S22401B900F08130463946FAE72DE9F04104460D4616461F4632463B462046294607F012F965
S22401B92003D220462946BDE8F08130463946FAE72DE9F04104460D4616461F4632463B46CD
S22401B9402046294607F038FA03D220462946BDE8F08130463946FAE72DE9F04104460D4669
S22401B96016461F4632463B462046294607F0EAF803D220462946BDE8F08130463946FAE7C3
S22401B9802DE9F04104460D4616461F4632463B462046294607F010FA03D220462946BDE8DE
S22401B9A0F08130463946FAE72DE9F04104460D4616461F4632463B462046294607F0C2F816
S22401B9C003D220462946BDE8F08130463946FAE71048407A20F00300C01C0E494872704702
S22401B9E00C48407A00F00300012801D1002070470120FCE70748407A00F00300022805D06F
S22401BA000448407A00F00300032801D1002070470120FCE7CCDC072010B503201A490870BD
S22401BA20022119480078FEF7EFF810BD10B516480078012806D0022806D0032806D0042894
S22401BA4008D105E0002405E0012403E0022401E0032400BF00BF2046F9F7D0FC0B49088067
S22401BA600B48B0F87A000988B1EB800F01DD012010BD0020FCE705480088B0F57A6F01DB81
S22401BA80002070470120FCE78EC8072090C8072044C9072010B50320174908700021164856
S22401BAA00078FEF7B1F810BD10B513480078012806D0022806D0032806D0042808D105E01B
S22401BAC0002405E0012403E0022401E0032400BF00BF2046F9F792FC084908800848B0F8EE
S22401BAE07A000988B1EB800F01DD012010BD0020FCE7012070470000F0030010F20300105B
S22401BB0044C9072010B504466CB124480078401CC1B2224801702248B0F8F400814202DB8B
S22401BB200120204908704FF40001002001F0AFFC10BD00B589B002208DF8040001208DF8F1
S22401BB40100000208DF81C00174802901748089001A8F9F7C3FB00221146154805F046FAC4
S22401BB601449086040F2DC511248006805F054FA09B000BD0B48007870470120704710B501
S22401BB800446002007490870044908700448B0F8F6100848006805F03FFA10BDF8030010F0
S22401BBA044C90720F903001041420F0005BB0100343A0200F403001010B50446ECB14D4933
S22401BBC08868642804D84C49098801444A4A11804A490978491CC9B2484A11700A290BD161
S22401BBE0454909880A2291FBF2F1454A11700021414A1180414A117002E03E4803F0F5FCE0
S22401BC004FF40001002001F042FC10BD00B58BB001208DF8240032200A9009AA00213548C7
S22401BC2003F046FC334803F0E0FC02208DF8040001208DF8100000208DF81C003148029052
S22401BC403148089001A8F9F749FB002201212F4805F0CCF92E49086064212D48006805F045
S22401BC60DBF90121234803F0B4FC0BB000BD29480078704701207047F0B506460027DFF8DB
S22401BC8094C08CF800701E4F3A78234F3F78974200D1F0BD204F3F78974203DD1E4F3878BB
S22401BCA0114602E010461C4F39785A2800DD5A200A2900DA0A210A2800DA0A205A2900DD2C
S22401BCC05A21C0F15A0CA1F10A076744FDB2471AFCB2A54201DA2B4600E02346052B04DB35
S22401BCE00127DFF830C08CF800700B4F3A7000BFCFE70000004009409CC807209AC8072045
S22401BD0098C8072041420F00B9BB01003C3A020094C8072099C807209EC8072070470020A8
S22401BD2070470120704700007047274800787047012070477CB504460D462448007860B17E
S22401BD4000202149087000220121214805F04EF92049086000201D490870A4B1012C02D0CF
S22401BD60022C18D10EE029466846FFF70DFD1A48DDE9001206C04FF4E1711648006805F04B
S22401BD804BF908E000BF1348006805F051F900200D49087000BF00BF7CBD0F4909680E4AEA
S22401BDA05268891A0D4A1268914208DC0A490968094A52681144094A1268914202DA0121D4
S22401BDC0014A117070470000ACC80720ADC80720443A0200A0C80720A4C80720A00300104E
S22401BDE010B5044622460521022003F02CFD10BD08B500200346012201460090022003F060
S22401BE005BFD01220021022003F003FD2949B1F840006421F5F7EEFE0020FFF7E1FF00219C
S22401BE200120F5F77BFF01220421022003F00BFD08BD2DE9F04106460C4617462046FFF7AD
S22401BE4054FB804607F040FA45B21FB1604204B2684245B226B1012E1AD0022E26D108E0D7
S22401BE600020FFF7BDFF012200211046F5F716FF1CE00120FFF7B4FF142094FBF0F0323084
S22401BE801FFA80F8012241461046F5F707FF0DE00120FFF7A5FFA84605EBD8704010323099
S22401BEA081B201221046F5F7F9FE00BF00BFBDE8F081000044C9072008B5002003460122DC
S22401BEC001460090022003F0F7FC01220021022003F09FFC002003460122022100900846FC
S22401BEE003F0EAFC01220221084603F092FC002000F0B0F80020034602221A21009003F04B
S22401BF00DBFC1B4803F047F808BD2DE9F04107460D461646012F0CD0022F19D1012000F06F
S22401BF2099F80EB1684205B22846FFF713FB044616E0012000F08EF82846FFF76FFB0446E9
S22401BF402EB10020FFF76AFBC4EB400084B207E0002000F07FF80020FFF760FB044600BF74
S22401BF6000BF2146024803F01DF8BDE8F081000000C0084070B5334890F8A800042804D055
S22401BF80052805D0062809D105E00324002508E00424002505E00424032502E000240025CB
S22401BFA000BF00BF04B95DB1264991F82C14012900D100E0002108462A462146FAF7ACFC40
S22401BFC070BD2DE9F04105460C4616461E48407800F0030030B91D48407820F003001B4960
S22401BFE0487006E01948407820F00300401C1749487025B1012D0BD0022D18D107E01348C4
S22401C000407820F003001149487000240FE00EE02046FFF76AFA80460D4907F0F1F9074632
S22401C02007F052F904B20EB1604204B200BF00BF42F210700A2101FB040004494880BDE8D4
S22401C040F081000044C90720CCDC07202CC807200000204110B5044622460521022003F038
S22401C060F2FB22460421022003F0EDFB10BD08B500200346012201460090022003F01CFC29
S22401C08001220021022003F0C4FB00200346012202210090084603F00FFC01220221084663
S22401C0A003F0B7FB6549B1F840004FF47A71F5F7A1FD0020FFF7CEFF00210120F5F72EFE49
S22401C0C000210320F5F72AFE08BD2DE9F05F05460C4616465A480078A84209D15948B0F9B7
S22401C0E00000A04204D15848007808B9BDE8F09F25B1012D4DD0022D0DD10DE00020FFF745
S22401C100A9FF002211460120F5F7C8FD012200210320F5F7C3FD87E00120FFF79BFF002CCF
S22401C12016DD56B1002211460320F5F7B7FDA1B201221046F5F7B2FD2AE0002211460120B8
S22401C140F5F7ACFDA1B201220320F5F7A7FD1FE07EB1002211460120F5F7A0FD271E01DBA9
S22401C160384600E0784281B201220320F5F796FD0EE0002211460320F5F790FD271E01DB85
S22401C180384600E0784281B201221046F5F786FD4AE00120FFF75EFF2046FFF7A6F9814606
S22401C1A00EB189F000490021484607F0F5F912D2002211460120F5F771FD2449484607F09A
S22401C1C01FF9804607F09CF887B2012239460320F5F764FD27E00021484607F0DDF818D239
S22401C1E0002211460320F5F759FD1849484607F007F9834606F00CFF21F00041074606F016
S22401C20049FC1FFA80FA012251461046F5F746FD09E0002211460320F5F740FD012200210F
S22401C2201046F5F73BFD00BF00BF002006490870034805700348048000BF57E744C9072059
S22401C240AEC80720B0C80720B2C807200000204110B5FAF7C4FC01220521022003F0F3FAD9
S22401C26010BD2DE9F04107460C46154627B1012F24D0022F63D10CE0012034490870002126
S22401C2803846FFF757FD00213148C160FAF7A1FE55E001202D49087000202E4908700DB174
S22401C2A0604204B204EB840041002948C160FAF790FE61B23846FFF73DFD40E02348007897
S22401C2C038B925480078401C40B223490870052834D10020204908702046FFF706F9064676
S22401C2E00DB186F000461948007850B9304606F0EBFF40B2174991F90010884201D1BDE859
S22401C300F0811649304607F07BF8804606F0DCFF0F49C860FAF75DFE304606F0D5FF4FFA7B
S22401C32080F841463846FFF705FD304606F0CCFF40B20849087000200449087000BF00BF2D
S22401C34000BFDCE70648006870470000FE0300109003001000040010FF0300100000C84204
S22401C360A003001010B5044622460421022003F06AFA10BD08B50020034601220146009002
S22401C380022003F099FA01220021022003F041FA00200346012202210090084603F08CFA55
S22401C3A001220221084603F034FA6849B1F840006421F5F71FFC0020FFF7D4FF0021012071
S22401C3C0F5F7ACFC00210320F5F7A8FC08BD2DE9F04706460C4617465D480078B04209D1F9
S22401C3E05C48B0F90000A04204D15B48007808B9BDE8F08726B1012E65D0022E0DD10DE005
S22401C4000020FFF7AFFF002211460120F5F746FC012200210320F5F741FC8DE00120FFF776
S22401C420A1FF002C20DD7FB1002211460320F5F735FC0A2094FBF0F01FFA80F80122414670
S22401C4401046F5F72BFC3DE0002211460120F5F725FC0A2094FBF0F01FFA80F801224146D5
S22401C4600320F5F71BFC2DE0B7B1002211460120F5F714FC0A2094FBF0F8B8F1000F01DB50
S22401C480404601E0C8F100001FFA80F9012249460320F5F703FC15E0002211460320F5F7A7
S22401C4A0FDFB0A2094FBF0F8B8F1000F01DB404601E0C8F100001FFA80F90122494610468F
S22401C4C0F5F7ECFB38E00120FFF74CFF2046FFF70CF8804606F0F8FE45B20FB1684245B29F
S22401C4E0002D0ADD002211460120F5F7D7FBA9B201220320F5F7D2FB1DE0002D11DA002239
S22401C50011460320F5F7CAFBB5F1000801DB404601E0C8F1000081B201221046F5F7BEFBEF
S22401C52009E0002211460320F5F7B8FB012200211046F5F7B3FB00BF00BF00200649087038
S22401C540034806700348048000BF51E744C90720B4C80720B6C80720B8C8072010B504461C
S22401C56022460521022003F06EF922460421022003F069F910BD08B5002003460246014625
S22401C5800090022003F098F901220021022003F040F900200346024602210090084603F028
S22401C5A08BF901220221084603F033F900200346024605210090022003F07EF90122052102
S22401C5C0022003F026F900200346024604210090022003F071F901220421022003F019F9CD
S22401C5E00020FFF7BBFF08BD2DE9F04107460E46154627B1012F3AD0022F0DD10DE000202F
S22401C600FFF7ACFF00221146022003F01CF900220221084603F017F97DE00120FFF79EFF29
S22401C620002E0BDD85F001020021022003F00BF92A460221084603F006F917E0002E0BDA4F
S22401C6402A460021022003F0FEF885F001020221084603F0F8F809E000221146022003F0F5
S22401C660F2F800220221084603F0EDF853E00120FFF774FF29498A8CC98C511A01EB8100ED
S22401C68006F05EFE8046264906F05CFD044621462448006806F0B4FE8046002106F07CFE3A
S22401C6A00CD22048046000221146022003F0CBF800220221084603F0C6F82BE01A48D0F800
S22401C6C0F010204606F068FF0DD21648046085F001020021022003F0B6F82A4602210846B3
S22401C6E003F0B1F816E01048D0F8F00080F000482146404606F050FF0CD20A4804602A46A4
S22401C7000021022003F09FF885F001020221084603F099F800BF00BFBDE8F08138C807201E
S22401C7200000FA44BCC8072044C9072010B5044622460521022003F086F8224604210220F7
S22401C74003F081F810BD08B500200346012201460090022003F0B0F801220021022003F064
S22401C76058F800200346012202210090084603F0A3F801220221084603F04BF87549B1F817
S22401C78040004FF47A71F5F735FA0020FFF7CEFF00210120F5F7C2FA00210320F5F7BEFA55
S22401C7A008BD2DE9F04107460C46154627B1012F51D0022F0DD10DE00020FFF7B7FF00225A
S22401C7C011460120F5F76AFA012200210320F5F765FABBE00120FFF7A9FF002C16DD55B15A
S22401C7E0002211460320F5F759FAA1B201221046F5F754FA2EE0002211460120F5F74EFA76
S22401C800A1B201220320F5F749FA23E08DB1002211460120F5F742FAB4F1000801DB404638
S22401C82001E0C8F1000081B201220320F5F736FA10E0002211460320F5F730FAB4F1000874
S22401C84001DB404601E0C8F1000081B201221046F5F724FA7AE00120FFF768FF3E498A8CAB
S22401C860C98C511A01EB810006F06AFD80463B4906F068FC06460021304606F08DFE07D247
S22401C8803448B0F848000A2190FBF1F004B20BE00021304606F080FD06D22E48B0F84600A8
S22401C8A00A2190FBF1F004B231462D48006806F0A7FD8046002106F06FFD0CD2284806603A
S22401C8C0002211460320F5F7E9F9012200211046F5F7E4F939E01F48D0F8F010304606F0D1
S22401C8E05BFE14D21E4806600DB1032100E00121084600221146F5F7D1F9A1B20DB1012292
S22401C90000E0032210460122F5F7C8F91DE01148D0F8F00080F000483146404606F03CFEF3
S22401C92013D20F4806600DB1012100E00321084600221146F5F7B2F9A1B20DB1032200E0F7
S22401C940012210460122F5F7A9F900BF00BFBDE8F081000044C9072038C807200000FA447A
S22401C9600404001010B5044622460521022002F06AFF22460421022002F065FF10BD08B5F0
S22401C98000200346012201460090022002F094FF01220021022002F03CFF00200346012268
S22401C9A002210090084602F087FF01220221084602F02FFF8049B1F840004FF47A71F5F778
S22401C9C019F90020FFF7CEFF00210120F5F7A6F900210320F5F7A2F908BD2DE9FC5F8146C7
S22401C9E00C461646B9F1000F06D0B9F1010F4ED0B9F1020F0DD10DE00020FFF7B3FF0022AC
S22401CA0011460120F5F74AF9012200210320F5F745F9CEE00120FFF7A5FF002C16DD56B149
S22401CA20002211460320F5F739F9A1B201221046F5F734F92AE0002211460120F5F72EF99A
S22401CA40A1B201220320F5F729F91FE07EB1002211460120F5F722F9271E01DB384600E0DB
S22401CA60784281B201220320F5F718F90EE0002211460320F5F712F9271E01DB384600E080
S22401CA80784281B201221046F5F708F991E02046FEF72BFD82460EB18AF0004A47498A8C58
S22401CAA0C98C511A01EB810006F04AFC0746444906F048FB05460120FFF754FF2946414847
S22401CAC0006806F09DFC0746002106F065FC0FD23C480560002211460120F5F7DFF801224A
S22401CAE000210320F5F7DAF800203749087015E03149D1F8F00006F08BFA074688462846EA
S22401CB0006F086FA21F000413A464346CDE9000106F052F902D801202B4908702A48007875
S22401CB20F8B10021504606F037FC1AD225480560002211460320F5F7B1F82449504606F07E
S22401CB405FFC019006F064FA21F00041074605F0A1FF1FFA80FB012259461046F5F79EF82D
S22401CB6026E019480078C8B10021504606F014FD14D214480560002211460120F5F78EF8E6
S22401CB801249504606F03CFC804606F0B9FB87B2012239460320F5F781F809E0002211463B
S22401CBA00120F5F77BF8012200210320F5F776F800BF00BFBDE8FC9F44C9072038C8072015
S22401CBC00000FA44080400100C0400100000204110B5AE490020F7F74DFDAD49086010BD35
S22401CBE010B500221146AB4804F000FAAA49086010BD2DE9FC410446A848407800F07F0034
S22401CC00A7490978012900D100E0002140EAC1108DF80100A148007800F07F00A0490978E6
S22401CC2009B9012100E0002140EAC1108DF800009C48006806F0ECF9054600229A4B05F01B
S22401CC40BDFF074605F026FFC0B28DF802009048006820B1694620468D4A12689047BDE8BF
S22401CC60FC8170B505460E4600219048006804F005F904465CB12570668021468B480068A6
S22401CC8004F039F902218A48006804F063F970BD10B501248748007800B110BD804800789F
S22401CCA0012800D1841E7D487D4A1278805C00EB80004000604301B20220FFF7D2FF0320D3
S22401CCC0FFF797FF01207C4908704FF47A717248006804F0A1F900BFDFE710B5002077495C
S22401CCE00870704908607349087001206C490870002003E00A21694A1154401C0228F9DB73
S22401CD00FFF7C6FF10BD10B504462046FFF771FF00210846FFF7A5FF10BD10B50120654940
S22401CD200870FFF7F0FF10BD10B55C484078642148436349A1F842005848007864214843E3
S22401CD405F49A1F84400F3F74CFF0020FFF751FF40F23310FAF70FFC4FF49A70FAF70BFCF7
S22401CD6010BD00204F4908604D480078012803D100204B49087002E00120494908707047C6
S22401CD802DE9FE4F4B48007808B1BDE8FE8F4A480078012813D1F7F742FC0468A04749490C
S22401CDA0086004F05FF8484908600020424908704FF4FA613848006804F02EF9E5E704F03D
S22401CDC051F841490968421A404800884FF47A7148433F4909884FF47A73594300EB2140B3
S22401CDE0B2FBF0FB584606F0C3FA3A49019006F0A9F9029006F00CF904460D46F7F70FFC75
S22401CE0000680090804701902E480168019806F0FFFB029006F0FCF821F0004106462246D2
S22401CE202B4605F0AFFC804605F0BEFB1D4908604FF0030A28491B48006806F0ADFB0DD88E
S22401CE401E48007808B14FF0020A5046FFF7D1FEFFF787FF0120194908700BE000201749AD
S22401CE6008700E480E490978405C401C0B490C4A12788854BAF1030F02D1FFF709FF02E08E
S22401CE805046FFF740FF00BF7FE70000543A02002C0400104C3A02001004001014040010F8
S22401CEA0160400102404001000005940CC020010C80200102004001028040010290400100C
S22401CEC044C907201C040010180400108C3A02008E3A020000007A448FC2753C10B5E34979
S22401CEE00120F7F7C7FBE249086010BD10B500221146E04804F07AF8DF49086010BD0020B2
S22401CF0010E0002100EB4002DC4B03EB4202117100EB400203F8121000EB400203EB420249
S22401CF205180401C0628ECDB70471CB50446D44800788DF80000D248007800EB4000CF4909
S22401CF4001EB4000007908B1012000E0002000F00301CB48007800EB4000C84A02EB400063
S22401CF6090F90000C00F61F39F008DF80100C449097801EB410102EB410191F9000000283D
S22401CF8001DB014600E04142C9B28DF80210BC48007800EB4000B94901EB40004088ADF8B1
S22401CFA00300B348006820B169462046B04A126890471CBD70B505460E460021B1480068B5
S22401CFC003F05CFF04465CB1257066802146AD48006803F090FF0221AB48006803F0BAFFBB
S22401CFE070BD10B5A948007800B110BD00210846FFF7E0FF0020A249097801EB41019F4A6B
S22401D00002EB410108719E48007800EB4000A04931F910000A2190FBF1F040B298490978CB
S22401D02001EB410102F811000320FFF77EFF0120984908709248007800EB4000944A02EB59
S22401D040400041888C48006803F0E6FF00BFCCE72DE9F0479048B0F842000A2190FBF1F095
S22401D06084B28D48B0F8440090FBF1F085B28A48B0F8460090FBF1F086B28748B0F84800ED
S22401D08090FBF1F087B2A01900EBD071C1F34F08E81900EBD071C1F34F094FF4FA707C494A
S22401D0A048804FF4E170888028B208804FF4FA71774801814FF4E1714181604200B274494D
S22401D0C0C8804FF4FA717248C1814FF4E17101820FFA89F06E4988814FF4FA716C48818299
S22401D0E04FF4E171C182C8F1000000B2684948824FF4FA71664841834FF4E171818338B2C9
S22401D100634908834FF4FA71614801844FF4E1714184704200B25E49C883FFF7F0FE002042
S22401D1205749087059490870FFF75BFFBDE8F08710B504462046FFF7F8FE00210846FFF785
S22401D14039FF10BD10B5012050490870FFF7F0FF10BD10B5494801894F48A0F8AA104748C3
S22401D16041884D48A0F8AC104448818A4A48A0F8AE104248C1894848A0F8B0103F48018CA8
S22401D1804548A0F8B2103D48418B4348A0F8B410F3F727FD0020FFF7C8FE4FF4BB70FAF721
S22401D1A0EAF940F27710FAF7E6F94FF4BC70FAF7E2F940F27910FAF7DEF94FF4BD70FAF7DE
S22401D1C0DAF940F27B10FAF7D6F9FEF7D9FA10BD70B505462D48007800B170BD2D4800783C
S22401D1E0012819D100202B4908702548007800EB4000274A02EB400081881F48006803F091
S22401D2000BFF1F48007800EB4000214A32F910100220FFF7CFFEE0E7FFF794F8044620B2F4
S22401D2201749097801EB4101144A02EB4101488001201349097801EB410102EB41010871B0
S22401D2400320FFF772FE0E480078401C062803D10220FFF76DFF06E009480078401C084933
S22401D2600870FFF7BEFE00BFB7E700006C3A02003C040010643A020034040010A051001040
S22401D28038040010CC020010C802001030040010C45100103104001044C907202DE9F0415B
S22401D2A004460D460121080301F027FE002020604FF40017182001F0FBFD064605EB85109C
S22401D2C0B6FBF0F0461E47EA06272760BDE8F08110B50446206820F40010206000214FF4B9
S22401D2E0805001F00AFE10BD0146434850F82120C2F30B107047026822F0E0620260026826
S22401D30042EA016202607047026822F48032026019B1026842F4803202607047026822F416
S22401D3200012026019B1026842F4001202607047026822F00062026019B1026842F00062D6
S22401D3400260704710B5C36801248C40A343C36022B1C46801238B401C43C46010BD10B5C1
S22401D360036823F0E0630360012A05D1036801248C402343036004E0036801248C40A34337
S22401D380036010BD024602F1100050F82130C3F30B10704710B503460C4603F1100050F83F
S22401D3A0241012B101F0004101E001F0804109B1012010BD0020FCE701464868704702460A
S22401D3C00B46516813B101F0004101E001F0804109B1012070470020FCE770B504460D465D
S22401D3E0002600BF012229462046FFF7D3FF0646002EF7D070BD00001040034018B912B9E5
S22401D4002A4B196017E0022804D11AB9274B2033196010E028B9012A03D1244B1B1D196021
S22401D42009E0022805D1012A03D1204B2433196001E000BFFEE7704703463BB932B91B48FC
S22401D4400C380068C84000F001007047022B07D132B9164814300068C84000F00100F4E79C
S22401D46043B9012A06D1114808380068C84000F00100EAE7022B08D1012A06D10B4818303A
S22401D4800068C84000F00100DFE700BFFEE718B9064A121F116007E0022803D1034A1C3278
S22401D4A0116001E000BFFEE770470000908002404FF0FF31314A1160012230498039C1F8FE
S22401D4C0842049174FF0E022C2F8801201222C490A60002004E000222A490A54411CC8B2E5
S22401D4E02028F8DB70474FF02061274A11600021121D11602549121D11600021121D116022
S22401D500121D1160002005E000221F4914310A54411CC8B22028F7DB00211B4A20321160F9
S22401D520491E121D1160121D1160121D116070471549091D0860704710B503460C4672B6BC
S22401D5401148001D00681249884210D0002207E01048006850F822000D4941F82200521C90
S22401D560312AF5DB4FF08050FFF7E2FF00BF084903F1100041F8204062B610BD80E100E0C1
S22401D58084E200E000E400E004ED00E00000FA0500000010040200102DE9F84F05460E4689
S22401D5A0002700200090FD48854204D11A2001F07FFC009003E01C2001F07AFC00900098C9
S22401D5C0B0FBF6F74FF0010A18241CE0B7FBF4F004FB1070A8B9B7FBF4F0A0F1010B601E04
S22401D5E0C4B2032094FBF0F0401E00F0FF09032094FBF0F0201A401E00F0FF084FF0000A5D
S22401D60003E0A01EC4B2002CE0DC00BFBAF1000F01D000BFFEE7012028604FEA095040EAB2
S22401D620084040F4404040EA0B00686100202860BDE8F88F2DE9F04104460E46D74884424C
S22401D64004D10121480301F058FC03E00121880301F053FC02211A2001F0EAFB02211C20DB
S22401D66001F0E6FB02211E2001F0E2FB0120206000202061A0600E206060E7680020206084
S22401D6800120C7490860002505E00020C54A42F82500681C85B2B5F5007FF6DB0020C04975
S22401D6A048608860C86008614861086031462046FFF772FFBDE8F08110B50446B748844204
S22401D6C005D100214FF4005001F017FC04E000214FF4804001F011FC10BD2DE9F34F86B055
S22401D6E000224FF0010B0698C0F800B0086828B90020DFF8B4B28BF8000071E00120DFF837
S22401D700A8B28BF80000002367E0501C402803DD022008B0BDE8F08F0868057808684488E1
S22401D720086890F801C00026A048007800F0010038BB52B1501EDFF86CB25BF82070C7F3BD
S22401D7400908A04501DD0520E3E7680740EA0C7040EA044040F00066DFF848B25BF82200A1
S22401D76080B2DE464EF822005BF8220030434EF822008E480088401CDFF830B2ABF800007F
S22401D78026E0DFF820B25BF82270C7F30948A04501DD0520BDE7680340EA0C30204340F4F0
S22401D7A00066DFF800B25BF822006FF30F00DE464EF822005BF8220030434EF82200501C46
S22401D7C082B27A480088401CDFF8E0B1ABF800000868001D0860581C83B20879984294DCF5
S22401D7E0886800286AD0002365E0501CB0F5007F01DD02208DE7886805788868448888684C
S22401D80090F801C000266A48007800F0010038BB6748008850B1501EDFF888B15BF82070EC
S22401D820C7F30B08A04501DD052072E7680740EA0C7040EA0446DFF86CB15BF8220080B2B0
S22401D840DE464EF822005BF8220030434EF8220057480088401CDFF858B1ABF8000025E0DB
S22401D860DFF840B15BF82270C7F30B48A04501DD05204EE7680340EA0C3040EA0406DFF8EF
S22401D88024B15BF822006FF30F00DE464EF822005BF8220030434EF82200501C82B24448BF
S22401D8A00088401CDFF808B1ABF800008868001D8860581C83B2087B984296DC0869002845
S22401D8C04CD0002347E0501CB0F5007F01DD02201FE708690578086990F80490086990F8D2
S22401D8E001C00869407905900869408803900869C088029000262F48008858B1501EDFF818
S22401D900A4B05BF82070C7F30B080398804501DD0520FEE6680740EA0C7B03984BEA004086
S22401D92040EA493B05984BEA0030DDF808B040EA0B06DFF870B04BF822601E480088401C63
S22401D940DFF870B0ABF80000501C82B2086908300861581C83B2087D9842B4DC886968B3D1
S22401D960002340E0501CB0F5007F01DD0220D0E68869D0F804A08869057800260E48008849
S22401D980E8B1501EDFF81CB05BF8207027F0704004900498504512D90520BAE60040044034
S22401D9A000C0034000800340400400104204001044040010460400104804001016E04AEAB9
S22401D9C04576DFF8F0B34BF82260FB480088401CDFF8E4B3ABF80000501C82B28869083046
S22401D9E08861581C83B2087F9842BBDC086AE0B3002349E0901CB0F5007F01DD022088E608
S22401DA00086A0578086A90F80190086A40680190086A806800900026E848008870B1501E84
S22401DA20DFF890B35BF8207027F070400490DDF804B00498584501D905206AE6019840EAB4
S22401DA404576104602F1010B1FFA8BF2DFF864B34BF82060009840EA4976104602F1010B93
S22401DA601FFA8BF2DFF84CB300E011E04BF82060D2480088401CDFF844B3ABF80000086ABF
S22401DA800C300862581C83B291F824009842B1DCCB480088401C40108000DFF828B3CBF8E1
S22401DAA004005846D0F804B0C7480088401C40100BEB8000DFF80CB3CBF8080058468068A2
S22401DAC0DFF808B3BBF800B000EB8B00DFF8F4B2CBF80C005846C068DFF8DCB2BBF800B0FB
S22401DAE000EB8B00DFF8DCB2CBF8100058460069DFF8C8B2BBF800B000EBCB00DFF8C4B2B4
S22401DB00CBF81400B248007818B90020CBF8000004E00420DFF8ACB2CBF800000120F8E504
S22401DB202DE9F04F07460B4690464FF00009002400250021002200268C46A648874200D1C2
S22401DB4004E0A548874201D14FF001099C48008800EB400A9A480088401C0AEB600A9A4862
S22401DB600088401C0AEB6000DFF860A2BAF800A05044DFF844A2BAF800A05044DFF83CA24F
S22401DB80BAF800A000EB4A000FFA80FCBCF5007F02DB0220BDE8F08F0120DFF828A2CAF89C
S22401DBA00000B8F1000F73D1C3F30A0343EA49338548007800F0010008BB81480088401C51
S22401DBC04FEA600A80480088401C0AEB600001B2ACEB010006B2DFF8DCA15AF8214008E0A9
S22401DBE0481C01B2DFF8CCA15AF821504AF821402C46301EA6F1010A0FFA8AF6F0D17248F8
S22401DC00008868B96E480088401C401002B24FF6FF7040EA0340DFF89CB14BF82200ABE082
S22401DC206948008801281FD165480088401C401002B2DFF880A15AF82200B3EB104F08D2B4
S22401DC405AF82200000C40EA0340D3464BF8220092E0DFF860A15AF822006FF30F001843C9
S22401DC60D3464BF8220087E055480088401C401001B25548008802B251480088401C4FEAA6
S22401DC80600A51480088401C0AEB600006B218E0A4E0DFF820A15AF82100B3EB104F02D232
S22401DCA0480002B20FE0DFF80CA15AF8210080B2984204D9012000EB410002B203E0481C4B
S22401DCC001B2B142E5DB00BFB14218D13E48007800F0010040B94FF6FF7040EA0340DFF85D
S22401DCE0D4B04BF8210047E0DFF8C8A05AF821006FF30F001843D3464BF821003CE0DFF821
S22401DD00B4A05AF8214002F0010018B9180440EA144503E0200C000440EA0305DFF894A043
S22401DD204AF8215026480088401C4FEA600A26480088401C0AEB6000401E06B20CE0481C28
S22401DD4001B2DFF870A05AF82150280C40EA0440D3464BF821002C46B142F0DB1A48007837
S22401DD6000F0010040B94FF6FF7000EB044A481CDFF840B04BF820A013480088401CDFF882
S22401DD8048A0AAF800000F488068001DDFF834A0CAF808005046C068001DCAF80C005046E3
S22401DDA00069001DCAF8100050464069001DCAF814005DE000800340480400104A04001019
S22401DDC04204001000C00340440400104604001040040010004004400080044043EA4973AD
S22401DDE0FE48B0F800A0FE480088401C0AEB600AFC480088401C0AEB600001B200220AE0CA
S22401DE00DFF8E4A35AF82100984200D907E0481C01B2501C02B2F54800888242F0DB00BF47
S22401DE20DFF8C4A35AF821404AF82130EF480088401CDFF8B8A3AAF8000066460AE0481C6F
S22401DE4001B2501C02B2DFF8A0A35AF821504AF821402C46B242F2DBE5480069001DDFF8AC
S22401DE6090A3CAF8100050464069001DCAF81400DC48008828B90020DFF874A3CAF8000008
S22401DE8004E00420DFF868A3CAF80000012081E62DE9FC4F07460A464FF0000800230024BC
S22401DEA099469A460020019000900021844600250026D048874200D104E0CF48874201D1DE
S22401DEC04FF00108C748008800EB400BC5480088401C0BEB600BC2480088401C0BEB600091
S22401DEE0DFF8F8B2BBF800B05844DFF800B3BBF800B05844DFF804B3BBF800B000EB4B00EC
S22401DF0006B2B6F5FE7F03DAB6480088402802DB0220BDE8FC8F0120DFF8D4B2CBF80000E0
S22401DF20C2F30A02C00240EA4830104382B2AD48007800F00100C0B9BEB1AA48008841101E
S22401DF403546DFF8A4B25BF8213008E0481C01B2DFF894B25BF821404BF821302346281E5C
S22401DF60A5F1010B0FFA8BF5F0D19E48008840B94FF6FF7040EA0240DFF86CB2CBF8000070
S22401DF8097E098480088012818D197480068B2EB104F09D294480068000C40EA0240DFF8D9
S22401DFA048B2CBF8000084E08F4800686FF30F001043DFF834B2CBF800007AE0002189486B
S22401DFC000880FFA80FC87480088401E401005B219E0DFF814B25BF82100B2EB104F03D297
S22401DFE048000FFA80FC10E0DFF8FCB15BF8210080B2904205D9012000EB41000FFA80FCB2
S22401E00003E0481C01B2A942E3DD00BFA94218DD7448007800F0010040B94FF6FF7040EABA
S22401E0200240DFF8C4E14EF8210042E0DFF8B8B15BF821006FF30F001043DE464EF8210090
S22401E04037E0DFF8A4B15BF821300CF0010018B9100440EA134403E0180C000440EA020435
S22401E060DFF884B14BF821405E48008845100CE0481C01B2DFF870B15BF82140200C40EA62
S22401E0800340DE464EF821002346A942F0DB5548007800F0010060B9DFF84CB15BF8210026
S22401E0A06FF30F004FF6FF7B5844DFF83CE14EF821004C480088A0EB0C0005B249480088B0
S22401E0C000EB4000301A0CEB4C0B5844401C01B2DFF814B15BF82130481C5BF82040881CD1
S22401E0E05BF82090002001F1020BDFF8FCE04EF82B0001F1010B4EF82B004EF82100C81C1A
S22401E10001B219E0DFF8E0B05BF821A0481C5BF820000190881C5BF8200000904BF821302F
S22401E120481C4BF82040881C4BF820905346019CDDF80090C81C01B2281EA5F1010B0FFA18
S22401E1408BF5DFD127480088401CDFF898B0ABF8000027484068001DDFF894B0CBF804005E
S22401E16058468068001DCBF808005846C068001DCBF80C0058460069001DCBF810005846E4
S22401E1804069001DCBF814000420CBF800000120BFE62DE9FF4F0C4615464FF00009AC42E8
S22401E1A003D9062004B0BDE8F08FDFF848E00098704502D14FF0000901E04FF0010909489D
S22401E1C0008800EB400E07480088401C0EEB600E03480088401C0EEB600011E0460400100B
S22401E1E04404001042040010008003404804001000C0034000400440008004404A040010A3
S22401E200DFF830E4BEF800E07044DFF82CE4BEF800E07044DFF824E4BEF800E000EB4E00E4
S22401E2200FFA80F80120DFF818E4CEF80000039800287DD1B8F5007F01DB0220B2E7C4F312
S22401E2400A04C5F30A054FEA497040EA044040EA493040EA0502FB480088401C4FEA600EE1
S22401E260F9480088401C0EEB600001B2F148008820B9DFF8D8E34EF8212042E0F1480088D1
S22401E280401C4FEA600EF0480088401C0EEB6000DFF8A0E3BEF800E0704403B213E0DFF8DD
S22401E2A0ACE35EF82160C6F30A4AC6F30A0B554502D84EF8212008E05C4502D3481C01B2A7
S22401E2C001E006206EE79942E9DB00BF994205DBDFF878E35EF821604EF82120A8EB01009F
S22401E2E003B208E0481C01B2DFF860E35EF821704EF821603E46181EA3F1010E0FFA8EF3B5
S22401E300F0D1CC480088401CDFF828E3AEF80000CB48C068001DDFF828E3CEF80C007046F4
S22401E3200069001DCEF8100070464069001D00E002E0CEF814009DE0B8F5FF7F01DD0220BB
S22401E34030E724F0604425F0604544EA497245EA497CBC480088401C4FEA600EBA48008838
S22401E360401C0EEB6000DFF8CCE2BEF800E07044DFF8C4E2BEF800E0704401B2AF4800881A
S22401E38038B9DFF8C8E24EF82120481C4EF820C062E0AC480088401C4FEA600EAA480088B9
S22401E3A0401C0EEB6000DFF88CE2BEF800E07044DFF884E2BEF800E07044DFF880E2BEF89D
S22401E3C000E000EB4E0003B21AE0DFF880E25EF82160481C5EF8207026F0604A27F0604B93
S22401E3E0554506D84EF8212000B201464EF820C008E05C4502D3881C01B201E00620D1E686
S22401E4009942E2DB00BF99420CDBDFF840E25EF82160481C5EF820704EF8212000B2014643
S22401E4204EF820C0A8EB0100401C03B2481C01B210E0DFF818E25EF82120481C5EF820C002
S22401E4404EF821604EF8207016466746881C01B2981E03B2002BECDC78480088401CDFF8E0
S22401E460DCE1AEF80000764840690830DFF8D0E1CEF814000420DFF8C8E1CEF800000120A7
S22401E48090E62DE9F04107460A460120DFF8B0C1CCF800006B480088401C4FEA600C6A4801
S22401E4A00088401C0CEB6000DFF888C1BCF800C06044DFF884C1BCF800C06044DFF87CC19B
S22401E4C0BCF800C000EB4C0086B2002F7ED15D48008818B15B480088824202DB0720BDE847
S22401E4E0F0815110DFF864C15CF8215055480088801A401EC0F34F0302F00100A8B90DE020
S22401E500481CDFF848C15CF82040200C40EA0540E04648F821002546481C81B2181EA3F10F
S22401E520010C1FFA8CF3EBD11CE015E0481CDFF81CC15CF82040280C000440EA1440E046DB
S22401E54048F82100481C5CF820004FEA004C481C48F820C0250481B2181EA3F1010C1FFA27
S22401E5608CF3E3D13748007800F0010098B902F0010040B94FF6FF7000EB0540DFF8CC8036
S22401E58048F8210043E04FF6FF702843DFF8BC8048F821003BE02B480088401C411029482A
S22401E5A0008800EB4000304483B20AE0DFF89CC05CF821C0481EDFF8948048F820C0481CD2
S22401E5C081B28B42F2DC4FF0000C00E05CE0481EDFF8788048F820C019484068001FDFF8AC
S22401E5E060C0CCF8040060468068001FCCF808006046C068001FCCF80C0060460069001FC9
S22401E600CCF8100060464069001FCCF814000D480088401EDFF82CC0ACF8000002EB420009
S22401E620304481B260460088801A401C00EB400083B226E046040010480400104A0400108F
S22401E64000C00340420400104404001000800340C81CDFF830C45CF82000E04648F8210096
S22401E660081D5CF820C0481C48F820C0481DC4465CF820C0881C48F820C0D81E83B2C81C41
S22401E68081B2002BE4D17EE1012F7AD1FE48008818B1FD480088824201DB07201FE7FB4813
S22401E6A00088401C401000EB620081B2DFF8D4C35CF82150F4480088801A401EC0F34F03AC
S22401E6C002F00100A8B90DE0481CDFF8B8C35CF82040200C40EA0540E04648F821002546FC
S22401E6E0481C81B2181EA3F1010C1FFA8CF3EBD11CE015E0481CDFF88CC35CF82040280CEF
S22401E700000440EA1440E04648F82100481C5CF820004FEA004C481C48F820C0250481B2AD
S22401E720181EA3F1010C1FFA8CF3E3D1D648007800F0010098B902F0010040B94FF6FF7038
S22401E74000EB0540DFF83C8348F8210044E04FF6FF702843DFF82C8348F821003CE0CB4833
S22401E7600088401C4FEA600CC7480088401C0CEB600081B2C548008800EB4000304483B224
S22401E7800BE031E0DFF8FCC25CF821C0481EDFF8F48248F820C0481C81B28B42F2DC4FF069
S22401E7A0000C481EDFF8DC8248F820C0B8488068001FDFF8DCC2CCF808006046C068001F57
S22401E7C0CCF80C0060460069001FCCF8100060464069001FCCF81400AB480088401EDFF86B
S22401E7E0A8C2ACF80000CEE0022F49D1A948008818B1A8480088824201DB07206FE6A3484B
S22401E8000088401C4FEA600C9F480088401C0CEB60001044401C81B29C48008800EB4000CD
S22401E820304483B20AE0DFF85CC25CF821C0481EDFF8508248F820C0481C81B29942F2DBA7
S22401E8404FF0000C481EDFF83C8248F820C091480088401EDFF83CC2ACF800008C48C06818
S22401E860001FDFF82CC2CCF80C0060460069001FCCF8100060464069001FCCF8140082E034
S22401E880032F49D18448008818B183480088824201DB072023E67D480088401C4FEA600C98
S22401E8A079480088401C0CEB6000DFF8E8C1BCF800C060441044401C81B27448008800EBAC
S22401E8C04000304483B20AE0DFF8B8C15CF821C0481EDFF8B08148F820C0481C81B29942DA
S22401E8E0F2DB4FF0000C481EDFF8988148F820C069480088401EDFF8A0C1ACF80000644865
S22401E9000069001FDFF888C1CCF8100060464069001FCCF8140036E06048008818B15F4879
S22401E9200088824201DB0720D9E55C480088A6EB400000EB420081B25448008800EB400018
S22401E940304483B20FE0881CDFF838C15CF82000E04648F82100C81C5CF820C0481C48F8EE
S22401E96020C0881C81B29942EDDB4C480088401EDFF828C1ACF80000454840690838DFF80C
S22401E98010C1CCF814000420DFF804C1CCF800000120A4E510B50246D06900F00400002838
S22401E9A03CD0106B20F470201063106B0C7B40EA04401063887B012804D1106B40F0804064
S22401E9C0106303E0106B20F080401063487B012804D1106B40F00040106303E0106B20F090
S22401E9E000401063086850630C79487944EA0024887944EA0044C87944EA006393630C7AE2
S22401EA00487A44EA0024887A44EA0044C87A44EA0063D36321205060012010BDD06900F453
S22401EA20806000284BD0106C20F470201064106C0C7B40EA04401064887B012804D1106CB7
S22401EA4040F08040106403E0106C20F080401064487B012804D1106C40F00040106403E0A5
S22401EA60106C20F000401064086850640C79487944EA0024887944EA0044C87944EA00634F
S22401EA8093640DE000800340440400104204001000C0034046040010480400104A04001004
S22401EAA00C7A487A44EA0024887A44EA0044C87A44EA0063D364412050600120ADE7D06939
S22401EAC000F48020E0B3106D20F470201065106D0C7B40EA04401065887B012804D1106D0E
S22401EAE040F08040106503E0106D20F080401065487B012804D1106D40F00040106503E000
S22401EB00106D20F000401065086850650C79487944EA0024887944EA0044C87944EA0063AB
S22401EB2093650C7A487A44EA0024887A44EA0044C87A44EA0063D3658120506001206CE7F9
S22401EB40FFE7002069E710B50246D06900F00100002825D0106AC00F4873106AC0F38070E4
S22401EB608873106AC0F303400873506A0860887B90B9936A0B711C0A4C711C0C8C711C0E90
S22401EB80CC71D36A0B721C0A4C721C0C8C721C0ECC720420506005E004205060012010BD8B
S22401EBA00020FCE70120FAE72DE9F043804600249D48406A20B19C48446A00261F2706E0D3
S22401EBC09948806A18B19848846A20263F27002C52D0002535464DE004F0010C6408BCF1EC
S22401EBE0000F46D090484069DFF84092484405EB450900EB8902106800F04070B0F1407F08
S22401EC0037D1106820F040701060121D13680B714FEA132981F805904FEA134981F80690F1
S22401EC204FEA136981F80790121D13680B724FEA132981F809904FEA134981F80A904FEA7A
S22401EC40136981F80B90083A1088C0F30A0008601068C0F303400873002048731068C0F330
S22401EC6080708873106800F0407010B90120BDE8F0836D1CBD42AFD90320F8E7024621B15D
S22401EC80012904D0022906D103E090687047D068FCE79069FAE7D069F8E7024611B101299B
S22401ECA004D101E0106870475068FCE79068FAE710B5012A0ED10B2906D101235A4C2360CE
S22401ECC023620423236013E0036901248C40234303610DE00B2906D10123534C2360236222
S22401ECE00023236004E0036901248C40A343036110BD31B1012907D0022908D003290CD121
S22401ED0008E00022026008E00122026005E00222026002E00422026000BF00BF70470829D9
S22401ED206CD2DFE801F0040713273B47535F0023036063E0012A04D1036843F00103036090
S22401ED4003E0036823F00103036057E0036843F001030360012A04D1036843F002030360A3
S22401ED6003E0036823F002030360036823F00103036043E0036843F001030360012A04D1B7
S22401ED80036843F00403036003E0036823F004030360036823F0010303602FE0012A04D1A6
S22401EDA0036843F00803036003E0036823F00803036023E0012A04D1036843F0100303605B
S22401EDC003E0036823F01003036017E0012A04D1036843F02003036003E0036823F02003B7
S22401EDE003600BE0012A04D1036843F08003036003E0036823F08003036000BF00BF7047BF
S22401EE0042680A43426070470146C86870470146086A08B1012070470020FCE7024609B917
S22401EE20506A7047906AFCE700C003400080034010B50A46202801D2034601E0A0F12003AA
S22401EE401946202810D2494B1B6803248C40A343474CC4F8A831454B1B6802FA01F42343A1
S22401EE60434CC4F8A83111E0404B1B1D1B6803248C40A3433E4CC4F8AC313C4B1B1D1B68F3
S22401EE8002FA01F423433A4CC4F8AC3110BD0146202903D20A46354B186804E0A1F12002DC
S22401EEA0324B1B1D186820FA02F303F00300704770B504462F4805682046FFF7E8FF064679
S22401EEC036B1012E06D0022E06D0032E10D105E004260DE001260BE0022609E01A2C03D0F0
S22401EEE01C2C01D01E2C01D1062600E0082600BF00BFB5FBF6F5284670BD012909D11C4A7F
S22401EF00C43212681C4B03401A43194BC3F8C42009E041B9164AC4321268174B83431A403C
S22401EF20134BC3F8C420704700201149C031086030BF704704201149086008200C49C0314A
S22401EF40086030BF704704200C49086009200849C031086030BF7047042008490860032043
S22401EF600349C031086030BF70470000A8C10F4000C00F404C040010DEF7EFEF10ED00E089
S22401EF80026822F480320260012903D1026842F480320260704700B5034600211248FFF7FF
S22401EFA0EFFF00BD036803F48032C1F3090342EA831202607047426822F00F0242600A7801
S22401EFC01AB1426842F0020242604A781AB1426842F0040242608A781AB1426842F008021A
S22401EFE0426070470181704700C0084002461068084008B1012070470020FCE701607047BD
S22401F00010B50A460B4618B901241470546005E0012803D100245C7001241C7010BD2DE9F0
S22401F020FC5F04460E4691464D46CA4601214020FFF763FF00210C20FFF7FAFE0C20FFF720
S22401F04037FF4FF0000807463F2020600020606020676061A062E0642065D6B9287818B90E
S22401F0606868401EE06021E000213A466868A0FB023B01FB07B100FB0810CC4ACDE900300F
S22401F0800023DDE9000100F0B7FE0746781EE0600CE0012E0AD19AF8010000F003019AF8A9
S22401F0A0000061F39F00216F08432067BDE8FC9F10B504460020606000214020FFF71DFF33
S22401F0C010BD012904D1426842F00802426003E0426802F0030242607047012904D1426850
S22401F0E042F00102426003E0426802F00A0242607047416841F002014160416801F009012D
S22401F100416070474A78012A0AD10A7802F0070202EB420301229A4043691A4342610CE085
S22401F1200A7802F0070202EB420301229A40A04B23EA020243691A404261CA78012A0CD12E
S22401F1400A7802F0070202EB4202521C012303FA02F243691A4342610CE00A7802F0070263
S22401F16002EB4202521C01239340914A9A4343691A4042618A78012A0CD10A7802F007020B
S22401F18002EB4202921C012303FA02F243691A4342610CE00A7802F0070202EB4202921C81
S22401F1A001239340824A9A4343691A40426170474A78012A0BD10A7802F0020363F35F0250
S22401F1C0012303FA02F2836A1A4382620BE00A7802F0020363F35F02012393403F229A4396
S22401F1E0836A1A4082628A78012A0CD10A7802F0020363F35F02521C012303FA02F2836A34
S22401F2001A4382620CE00A7802F0020363F35F02521C012393403F229A43836A1A408262BD
S22401F220CA78012A0CD10A7802F0020363F35F02921C012303FA02F2836A1A4382620CE071
S22401F2400A7802F0020363F35F02921C012393403F229A43836A1A4082627047024611B1A9
S22401F260012904D101E0D06A7047106BFCE70020FAE730B5072913D2DFE801F00406080A8A
S22401F2800C0E100082610BE0C26109E0026207E0426205E0026403E0426401E0826400BF1B
S22401F2A000BF6BB3012B21D0022B02D0032B39D10BE0072902DA01248C4000E000243D4DA1
S22401F2C02D682C433B4D2C602CE0072902DA01248C4000E00024374D2D682C43354D2C606D
S22401F2E02C462468046500242C601BE0056D072902DA01248C4000E000242543056511E0C0
S22401F300056D072902DA01248C4000E0002425430565446844F002044460446804F009046B
S22401F320446000BF00BF30BD30B572B9C46C01F00703022B01DA002301E001238B4047F645
S22401F3407C659D432C40C4640AE0C46C01F00703022B01DA002301E001238B401C43C464BB
S22401F36030BD30B5012A0ED1C46C01F00703012B01DA002304E001F10803012505FA03F35A
S22401F3801C43C46410E0C46C01F00703012B01DA002304E001F10803012505FA03F347F662
S22401F3A07C659D432C40C46430BD000040420F00FFFF1F00C0C8072070B5054635B1012D24
S22401F3C009D0022D0CD0032D14D10EE00220FFF76FFD04460EE00420FFF76AFD044609E0D0
S22401F3E02C20FFF765FD044604E02E20FFF760FD044600BF00BF204670BD2DE9F047814625
S22401F4000C464846FFF7D8FF0026054600232946A1FB047C06FB04C205FB0321C44A3846A3
S22401F42000F0EAFC05462846BDE8F08701464FF0FF30B1F1402F01D100200DE0BD4A91429C
S22401F44001D1012008E0BC4A914201D1022003E0BA4A914200D10320704710B50246106814
S22401F46001248C402040C3B20BB1012010BD0020FCE710B50246106801248C402040C3B2C8
S22401F4800BB1012010BD0020FCE701228A400260704701228A400260704720B90A46012360
S22401F4A01370536003E00A460023537000BF70472DE9F04704460F461546B4F1402F08D14D
S22401F4C001210220FFF719FD00210220FFF7B0FC22E09848844208D101210420FFF70DFD2A
S22401F4E000210420FFF7A4FC16E09348844208D101218805FFF701FD00212C20FFF798FC21
S22401F5000AE08E48844207D10121C805FFF7F5FC00212E20FFF78CFCA06A20F00300A062A5
S22401F520A06AA0620020A0602061E060606840F002006060606820F00200606087B92E46D0
S22401F540307818B97068401EE06017E02046FFF76DFF81467168FFF750FF401EE0600DE087
S22401F560A846A06A20F00C00A062454698F80100012803D1A06A40F00400A0624FF0FF30A8
S22401F5802060BDE8F08710B5044600206060B4F1402F04D100210220FFF7AFFC18E0654868
S22401F5A0844204D100210420FFF7A7FC10E06248844205D100214FF48000FFF79EFC07E03B
S22401F5C05E48844204D100214FF48000FFF795FC10BD012904D1426842F00102426003E049
S22401F5E0426822F0010242607047416841F002014160416821F002014160704710B50A7813
S22401F60032B1012A07D0022A08D0032A0CD108E08A6882610AE08A68C26107E08A680262F8
S22401F62004E08A68426201E000BFFEE700BF42690B7803EB43040723A3409A4342614A7854
S22401F6403AB142690B7803EB43040123A3401A434261CA7842B142690B7803EB43035B1C41
S22401F66001249C40224342618A7842B142690B7803EB43039B1C01249C4022434261C26B37
S22401F6800B78042404EB43040323A3409A43C2630A7902F003020B78042404EB43039A4044
S22401F6A0C36B1A43C26310BD31B1012906D0022906D0032908D105E0826107E0C26105E028
S22401F6C0026203E0426201E000BFFEE700BF704710B5826A0B7803EB43040723A3409A43EB
S22401F6E082624A783AB1826A0B7803EB43040123A3401A4382628A7842B1826A0B7803EB35
S22401F70043035B1C01249C4022438262CA7842B1826A0B7803EB43039B1C01249C402243E7
S22401F720826210BD024609B9D06A7047106BFCE740420F0000800040000009400040094096
S22401F74000BFFEE70446012C04D0022C03D0032C03D101E001E000E000BF00BF02F0D2FDCF
S22401F76000BFFEE71A4810B5007848B102F050FC30B1184900EB400001EB4010603810BDFB
S22401F780154810BD154A10B511690346102900D3FEE7134800EB0110491C1860116101F0CA
S22401F7A0EFFF012010BD0A490978002905D000684FF6FF71DFF82CC000DF70470449097851
S22401F7C0002903D00068DFF820C000DF7047000051040010D4120820C4170820C4C8072049
S22401F7E094160820691802009117020040B13049096841F400412E4AC43AC2F8C41007E0C8
S22401F8002B49096821F40041294AC43AC2F8C410704730B55AB1274C04EB40131B680124A4
S22401F8208C402343234D05EB401423600AE0214C04EB40131B6801248C40A3431D4D05EB0C
S22401F8404014236030BD30B53AB101238B40194C202505FB0044A36106E001238B40154CF7
S22401F860202505FB0044E36130BD02461148202303FB0200406901238B40184008B101201A
S22401F88070470020FCE730B5CB430A4C202505FB00442361074B202404FB00335A6130BDE2
S22401F8A001460448202202FB0100406970470000C4C00F4000C009202DE9F04104460D466F
S22401F8C01646069F00212A46102D03DBA5F11000C2B20121DFF818C10CEBC40050F8210065
S22401F8E04FEA42084FF0030C0CFA08FC20EA0C00DFF8FC8008EBC40C4CF82100C4460CEB95
S22401F900C40050F821004FEA420C06FA0CFC40EA0C0008EBC40C4CF821003548403000EBEF
S22401F920C40050F821004FEA42084FF0030C0CFA08FC20EA0C0C2E48403000EBC40040F8CA
S22401F94021C02B48403000EBC40050F821004FEA420C03FA0CFC40EA0C00DFF894C00CF1DB
S22401F960400C0CEBC40C4CF82100012F0ED12048683050F824C00120A8404CEA0000DFF8B8
S22401F98070C00CF1680C4CF824000DE01848683050F824C00120A8402CEA0000DFF850C041
S22401F9A00CF1680C4CF824000020BDE8F0810146012906D10E48806A40F008000C4A90622A
S22401F9C005E00B48806A20F00800094A90620020704702460B460021022A01D141F00501DC
S22401F9E00BB941F00A010248C16700207047000000C002404FF0000080F3108880F3118860
S22401FA0080F314880C480068006880F308880B4880470B480047FEE7FEE7FEE7FEE7FEE77D
S22401FA20FEE7FEE7FEE7FEE7FEE7000005480649064A074B7047000008ED00E0EDFB010094
S22401FA40CD000100205200102828082020620010281808202DE9F04799480068C0F3016034
S22401FA6003287DD196488430006800F0030030B1012830D0022859D003282BD100E000BFF7
S22401FA808F480068C0F30740441C02218C488838D0F88800C0F30E00401CA1FB0001894B32
S22401FAA04FF0000CA0FB037901FB039100FB0C1122466346384600F09FF9054680487C3060
S22401FAC00068C0B2441C22460023284600F094F97D49086056E07A480068C0F30740441C88
S22401FAE0022177488838D0F88800C0F30E00401CA1FB0010754A4FF0000CA1FB027900FB29
S22401FB00029001FB0C0122466346384600F074F905466B487C300068C0B2441C22460023E9
S22401FB20284600F069F9684908602BE064480068C0F30740441C022161488838D0F8880091
S22401FB40C0F30E00401CA1FB00124FF400400023A1FB007902FB009001FB0301224600E044
S22401FB6011E0384600F048F9054655487C300068C0B2441C22460023284600F03DF9524957
S22401FB80086000BF30E04E488430006800F0030030B1012810D0022819D0032823D100E087
S22401FBA000BF47487C300068C0B2401C4549B1FBF0F04549086016E041487C300068C0B2FA
S22401FBC0401C4249B1FBF0F03F4908600BE03C487C300068C0B2401C4FF40041B1FBF0F05B
S22401FBE03949086000BF00BFBDE8F08730203849086033488838D0F8A00100F0200030B1AD
S22401FC0000BF3348006800F040000028F9D003202B497C3108604FF4805029498839C1F870
S22401FC20A80100202A490C310860012024498431086028482249091F0860AA202049091D6E
S22401FC4008605520086001201D4908390860AA201B49091D0860552019498839C1F88C0090
S22401FC6000BF1748006800F080600028F9D00320134908390860AA2011498839C1F88C00E5
S22401FC8055200F49091D086000BF0D48006800F04070B0F1407FF8D1002009498031086033
S22401FCA00D4807498839C1F8C4000020C1F8C8010846006820F4704040F48040086070472C
S22401FCC088C00F4000093D004C040010002D3101A0C10F400E000100DE872C05004870472E
S22401FCE0C41708200B3020F0070070472DE9F04117460E460446FFF7F5FFA042054633D98D
S22401FD00002F1CBF06F10C00FFF74DFD30467468F4B12168A94217D305F1080291423CBF6D
S22401FD206168416007D3626861194A602268521B0A6041602560002F1CBF06F10C00FFF701
S22401FD403DFD201DBDE8F08120466468002CE0D12946304600F087F90028D7D1002F1CBFD2
S22401FD6006F10C00FFF72AFD0020BDE8F08110B5044600F06FF901682046BDE810400122D9
S22401FD80B4E770B516460D46041F002808BF70BD002E1CBF05F10C00FFF705FD2B4658687B
S22401FDA0002818BFA04238BF0346F8D31968CA18A24218BF5C6003D122681C4611441960E9
S22401FDC021680A19824218BF606004D142686260006808442060002E1CBF05F10C00FFF7A0
S22401FDE0EDFC70BD10B5044600F034F901682046BDE810400122C4E753EA020C00F0698005
S22401FE002DE9F04B4FF00006002B1FBFB3FA83F503FA05F424FA05F65E4012BF1643B2FA95
S22401FE2082F502FA05F4C5F120051EBF22FA05FC44EA0C04203556EA044C4FEA144418BFF0
S22401FE40641C4FF000084FF00009904271EB030C39D3002919BFB1FA81F701FA07F6B0FA7E
S22401FE6080F700FA07F6C7F120071EBF20FA07FC46EA0C062037B6FBF4FCA7EB0507103F0E
S22401FE8007F01F0BCBF120060CFA0BFB2CFA06F644BFB3460026202FA4BF5E464FF0000B69
S22401FEA05BEA060C08BF4FF0010B19EB0B09ABFB027C48EB0608C01B06FB02CC0BFB03CCD7
S22401FEC071EB0C01C1E70B46024641464846BDE8F08B13B54FF000004FF00001AFF30080D4
S22401FEE0BDE81C40704710B50446AFF300802046BDE81040F0F759B940EA010310B59B072A
S22401FF000FD1042A0DD310C808C9121F9C42F8D020BA19BA884201D9012010BD4FF0FF30C0
S22401FF2010BD1AB1D30703D0521C07E0002010BD10F8013B11F8014B1B1B07D110F8013B49
S22401FF4011F8014B1B1B01D1921EF1D1184610BD032A40F2308010F0030C00F0158011F8F5
S22401FF60013BBCF1020F624498BF11F801CB00F8013B38BF11F8013BA2F1040298BF00F857
S22401FF8001CB38BF00F8013B11F0030300F02580083AC0F0088051F8043B083A51F804CB6C
S22401FFA0A0E80810F5E7121D5CBF51F8043B40F8043BAFF30080D20724BF11F8013B11F84A
S22401FFC001CB48BF11F8012B24BF00F8013B00F801CB48BF00F8012B704710B5203AC0F087
S22401FFE00B80B1E81850203AA0E81850B1E81850A0E81850BFF4F5AF5FEA027C24BFB1E89A
S2240200001850A0E8185044BF18C918C0BDE810405FEA827C24BF51F8043B40F8043B08BFE0
S2240200207047D20728BF31F8023B48BF11F8012B28BF20F8023B48BF00F8012B704702F090
S224020040FF0343EA032242EA024200F065B870477047704710B5FFF741FE083010BD7047ED
S22402006070477047704738B504460A4600206946AFF30080002808BF38BD024600992046B1
S22402008000F06CF8012038BD012000F086B8F8B5AFF30080054600200C46102000BF0646D9
S2240200A0A819A0420DD9324669460020AFF30080070008BF00F071F80098A04218BF054684
S2240200C0C419FFF7C7FF05600746F01D20F007004619284600F00AF8B44208BFF8BDA21BBC
S2240200E031463868BDE8F84000F038B800210160C0E901100C30FFF745BB1020704710B50B
S22402010000F02AF8006810BD10B5044600F024F8046010BD4FF000020429C0F0128010F095
S224020120030C00F04380CCF1040CBCF1020F18BF00F8012BA8BF20F8022BA1EB0C0100F03B
S22402014035B85FEAC17C24BF00F8012B00F8012B48BF00F8012B7047FFF704BB30B4044635
S2240201608C464368002B18BF634538BF1846F8D303681844604507D0C81C20F0070000F102
S224020180040CACEB0100121A2146CCF8002030BC00220CF10400FFF7F4BD10B500F05EF878
S2240201A0BDE8104000F054B84FF0000200B5134694469646203922BFA0E80C50A0E80C5040
S2240201C0B1F12001BFF4F7AF090728BFA0E80C5048BF0CC05DF804EB890028BF40F8042B33
S2240201E008BF704748BF20F8022B11F0804F18BF00F8012B7047000001491820ABBEFEE7DC
S2240202002600020070477546FFF768FDAE4605006946534620F00700854618B020B5FFF72C
S22402022005FCBDE820404FF000064FF000074FF000084FF0000B21F00701AC46ACE8C0092D
S224020240ACE8C009ACE8C009ACE8C0098D467047002801D0FFF7D0BF7047000010B50128D3
S22402026005D0002103A000F021F8012010BD09A1F8E7000053494752544D454D3A204F75D8
S22402028074206F662068656170206D656D6F7279000000003A2048656170206D656D6F725F
S2240202A07920636F727275707465640070B505460C460A2000E06D1C00F011F835B12878F2
S2240202C00028F8D102E0641C00F009F814B120780028F8D1BDE870400A20AFF3008008B527
S2240202E069468DF800000320ABBE08BD00000000490050EAC12018BF04204A0D18BF40F0B5
S224020300010040F2FF72B2EB515F08BF40F00200012808BF052070472DE9F74F144694B026
S2240203200021C4E902111599079121F00045C9498D4206DC1599C4E9000117B00020BDE88E
S224020340F08FC549DFF814A3A9423CDD0799C44E0029C44FC44A1599534619DD02F06EFDE1
S224020360554506D0C14AC24B02F068FDC4E900010AE04FF0D352BE4B02F060FD32463B464A
S22402038002F05CFDC4E9000117B00120BDE8F08F02F03CF9554506D0B44AB54B02F036F99B
S2240203A0C4E900010AE04FF0D352B14B02F02EF932463B4602F02AF9C4E9000117B04FF063
S2240203C0FF30BDE8F08FAB49A942159978DB21F0004183468846A84AA84B02F0EFFB002217
S2240203E0A74B02F013F902F025FB099002F07FFB06460F469C4A534602F0E0FB43465A46D9
S22402040002F010FD80468A46984A994B3046394602F0D4FB2A0D01250B924246534602F0B7
S22402042001FD032DC4E9000139D00B98C1F30A51401A05EB45111139814230DA9148C34685
S224020440784400EB0510CDF80CA00C90D0E900233046394602F0B2FB02460B460491069098
S2240204605846039902F0EAFC80468A4602460B465846039902F0E2FC049B069A02F0DEFC1F
S22402048083460C9803913946D0E90223304602F095FB5A46039B02F0D1FC6D1CBDE7079836
S2240204A00028A2BF099817B0BDE8F08F616881F000416160099817B04042BDE8F08FFFE7F0
S2240204C084461598C1F31301C0F30A50A0F2F5304FEA601800F01F06C6F1200013900020B2
S2240204E00690079041F4801E05206D4676B1664A08EB00017A4452F8213002EB8101B34097
S2240205004A68139922FA01F1194305E05F4908EB0002794451F82210A1FB0E27A1FB0C13C6
S2240205201A449A4234BF0123002303EB070A05EB8003D3E901B70F448F4234BF0121002100
S22402054093448B4411B1934502D903E0934501D2012100E00021C3E901B7514445F8201062
S224020560011EA0F10100C1DC0298059F00F10050800F12900298DDE90356800002F0B7FA9A
S224020580834628460D9102F0C9FA6FF01D0203F0E6F8CDE90E01304602F0C0FA6FF03D02F6
S2240205A003F0DDF880468A46384602F0B7FA6FF05D0203F0D4F8074642465346119102F036
S2240205C025F8DDE90E2302F021F85A460D9B02F01DF800250E465A4628460D9B02F02EFC5B
S2240205E0DDE90E2302F02AFC4246534602F026FC3A46119B02F016FCDFF898A0244A53466A
S22402060002F0DCFA07468846234A244B3146284602F0D4FA3A46434601F0F8FF0746884663
S2240206204FF0A84253463146284602F0C7FA3A46434601F0EBFF159A12F0004F04D0129AF5
S22402064081F0004152421292C4E90001129817B0BDE8F08FFB21E93F7CD90240FB21F93F37
S2240206607370032E8A19A33B000040543163621A61B4D03DFB21394183C8C96D305FE43F4F
S2240206800000E03F3C370000B83600009A360000182D4454FB21F93D3326A611460B113C26
S2240206A02DE9F0414F1E00EBC7010446D1E9000115461E4637F006020DD02A46334602F021
S2240206C07DFA7F1E04EBC703D3E9002301F09EFF37F00602F1D1022F25D0042F13D0062F77
S2240206E018BFBDE8F0812A46334602F067FAD4E90A2301F08BFF2A46334602F05FFAD4E974
S224020700082301F083FF2A46334602F057FAD4E9062301F07BFF2A46334602F04FFAD4E9D6
S224020720042301F073FF2A46334602F047FAD4E9022301F06BFF2A46334602F03FFAD4E9FE
S2240207400023BDE8F04101F061BF00002DE9F04D04468CB0904821F00047164698460D46F2
S2240207600991874206DA2046294602F063F9002800F0AE808948B8421CDC09980028BCBFBF
S22402078085F0004588F00048854A864B2046294602F048FB04460D463246434682488349FA
S2240207A002F04CFB22462B4601F030FF002604460D46B04622462B461046194602F0FEF9D0
S2240207C08B46824602460B4602F0F8F90246089077480B46009106217844FFF761FFCDE98D
S2240207E00310744806217844009B089AFFF758FF52465B4602F0E2F9CDE9051052465B46AC
S2240208002046294602F0DAF907910090DDE90310DDE9053201F0FAFE079B009A02F0CEF95B
S2240208203246434601F0F2FE52465B4602F0C6F93246434601F0EAFE80460E465E4A5F4B9F
S2240208400799009802F0BAF94246334601F0DEFE82468B4622462B4601F0D8FE80464F4850
S2240208600E46B84214985BDC02F041F9074642463346059101F0CAFECDE9011042463346AF
S2240208801046194602F09AF9DDE9013201F07AFF52465B4602F0D2FA22462B4602F0C2FA36
S2240208A0012202F05CFF3A46059B02F0BBFA04460D460998022101EAA070C0F1010002F0FA
S2240208C016F90CB022462B46BDE8F04D02F076B91498401C384320430BD01498012812D0F2
S2240208E00CB022462B46BDE8F04D0020344901F049BF0CB025F000432246BDE8F04D002066
S224020900304901F03FBF20462946FFF7F1FC042808BF00F063F820460CB02946BDE8F08DBF
S224020920012802BF40460CB0BDE8F08D00270B463A462046294602F075FA52465B4602F009
S22402094071FA04460D464246334600201C4901F019FF83463A4688463346104602F02EF9FA
S2240209600022184B01F052FE06468A4622462B463846414602F022F93246534601F046FE5D
S2240209805A46434602F01AF90CB03A464346BDE8F04D01F03BBE00000000303E2894E53F43
S2240209A0182D4454FB21E93F075C143326A6813C6C3400008E340000635555555555D53F5A
S2240209C00000F0BF0000F03F012202F0C8BE002213461046114601F0D5BE0000024A00207F
S2240209E0110702F0BCBE000001FDFFFF10B5002A06DA22F00042D21D22F00703102203E02D
S224020A00D21C22F003030C2213B19C188C4201D9012010BD024401448360C0E90021C91A72
S224020A20D018884202D810600246F9E70020106010BD00002DE9F84F04460D4621F00040E3
S224020A4000917349814211DC7249884201DC06D12CB120462946BDE8F84FFFF7B5BF6E489B
S224020A60002DCCBF6D496E49BDE8F88F6D49814211DD6D498142D8BF4FF0FF366DDD204683
S224020A802946FFF735FC042808BFFFF7A7FF20462946BDE8F88F6549654F25F000458142AA
S224020AA033DD6449814219DD002632464FF080432046294601F0AAFD80468A46012220468D
S224020AC0294602F04CFE00223B4602F0B7F94246534601F057FE04460D463EE001260022B4
S224020AE0BA463B462046294601F090FD80460F46002253462046294602F0A0F942463B46DC
S224020B0001F040FE04460D4627E04B4981421BDDDFF828A10226002253462046294602F062
S224020B204DF800223B4601F071FD80460F46002253462046294602F081F942463B4601F056
S224020B4021FE04460D4608E0032622462B4600203B4901F017FE04460D4622462B46104672
S224020B60194602F02BF88B46824602460B4602F025F807460246334888460B4606217844A7
S224020B80FFF78EFD52465B4602F018F882462E488B463A46434605217844FFF781FD3A46A4
S224020BA0434602F00BF802460B46002E504659460CDA01F02BFD22462B4601F0FFFF01B03C
S224020BC022462B46BDE8F04F02F02CB901F01EFD22462B4601F0F2FF1C4A7A4402EBC603D9
S224020BE0D3E9002302F02AF922462B4602F026F9174A7A4402EBC603D3E9002302F012F95F
S224020C00009A002AB8BF81F00041BDE8F88F0000000010440000F07F182D4454FB21F93FC0
S224020C20FB21F9BF0000DC3F0000203E0000F33F0000F03F0000E63F008003400000F83FE0
S224020C400000F0BFCE2F00008C2F00002A2F0000F22E000008480068C0010BD5074800689D
S224020C60C00707D0054880380068002802DA04490120087070470000FCED00E0800E00E08A
S224020C80ECC807204FF06042D36F002BFCD0036BD367D36F002BFCD0C07840EA0120A2F85A
S224020CA07C0070474FF06041CA6F002AFCD081F87C0070470EB5802200B109B110460AE02F
S224020CC001780129FAD101A900F046F8042801D0002000E01020DDE9011203B000BD70B52C
S224020CE00D46040003D012B92078012801D0802070BD204600F0F2FB28B12946204600F0B8
S224020D0056F8002070BD812070BD70B50C4600F0FDFF4FF0004108B1220C01D0084670BD4D
S224020D20058BC178A0B200F003F8284670BD00000A460146074810B500EB820050F8040C9B
S224020D40002805D000F01AFEBDE8104000F006BE10BD00001C12082010B50446808900287B
S224020D6024D0608904EB800000690860606840B16078022805D10021204600F0FFFD00F05B
S224020D80EDFD04F10C0000BFD0E85F1F491E8AB2C0E8512F0029F7D16089401C80B2608158
S224020DA0E189884201D100206081042010BD10B500F0E4FDBDE8104000F0D0BDEFF30581C4
S224020DC009B182207047DFF808C000DF7047000021200200EFF3058008B182207047EFF326
S224020DE01480C00703D0DFF80CC000DF704701F021B900003520020088B0EFF3058010B103
S224020E00822008B07047EFF3148010F00301134806D001291BD0022911D0032919D113E0E5
S224020E2008A981F309880078C0070BD05FF0020080F31488BFF34F8FBFF36F8F09E00078DA
S224020E40C00706D10320F3E70078C00701D0FF20D7E7DFF80CC000DFD3E70000943A0200F7
S224020E60A5200200EFF3058008B100207047DFF808C000DF70470000ED200200EFF3058200
S224020E8012B1012201F0D4BA0022DFF808C000DF7047000031240200EFF305820AB10020F4
S224020EA07047EFF31482D20702D1044A52781AB1DFF80CC000DF704701F034B950040010F2
S224020EC025210200EFF3058212B1012201F0DCBA0022DFF808C000DF7047000089240200E7
S224020EE010B530B1006800F011F8102800D1202010BD802010BD20B129B10068002200F03C
S224020F0011B880207047862070470000EFF305820AB1FFF7CFBEDFF808C000DF7047000071
S224020F208B210200EFF305830BB1FFF7D8BEDFF808C000DF70470000C5210200EFF30582C4
S224020F4012B14FF000407047DFF804C000DF7047FB210200EFF305820AB1FFF7D6BEDFF8BD
S224020F6008C000DF704700001F220200EFF305830BB182207047DFF808C000DF7047000015
S224020F8045220200EFF305820AB100207047EFF31482D20702D1044A52781AB1DFF80CC03C
S224020FA000DF704701F078B95004001099220200DFF80CC000DFDFF80CC000DFFEE7000068
S224020FC00523020021230200EFF3058109B182207047DFF808C000DF7047000021230200A4
S224020FE0DFF804C000DF704759230200EFF305830BB100207047EFF31483DB0702D1044BC1
S2240210005B781BB1DFF80CC000DF704701F0B0B95004001071230200EFF305820AB18220D7
S2240210207047DFF808C000DF70470000A9230200EFF3058109B182207047DFF808C000DFF6
S224021040704700000D240200094C4FF0FF3529462068FFF75BFF02460846102AF7D1FFF702
S224021060BFFF0028F3D0024608469047EFE70000C8C80720074801684FF0E020416100210C
S2240210808161072101610448016841F07F41016040177047903A020020ED00E07047000058
S2240210A002480068C0F380607047000004ED00E04FF0E020806902490968081A704700009F
S2240210C0903A020050E8001F31B10B6840E80032002AF7D108467047BFF32F8FFAE710B52A
S2240210E068B161B10B3121F00302016844680B1A1B1B934205D2084609680029F5D1002082
S22402110010BD210007D021180368C1E90032016001F1080010BD4260083010BD70B50D463C
S224021120002812D04FF6FF71084C884204D222680146104600F050FC20684570044800F019
S22402114037F9BDE8704000F00BBD70BDD8C80720941708200F4810B50D4942680E480B689F
S2240211600068934204D00A60CB88421E1A448A808A8880B282420AD100200860054800F02A
S22402118017F90146BDE81040024800F049BC10BDE4C8072094170820E0C8072070B5194DF0
S2240211A0E86800282CD0A88A401EA882002621E0A06838B161684160606810B1A168816005
S2240211C06660A6600F482146183800F029FCA08AA8826078042804D10B49E08A0988084451
S2240211E0A08201206070E068E860E06808B10561E6602661A88A002802D1EC68002CD7D1BC
S22402120070BD0000AC170820E0C8072070B504000FD00D4DA17801262868827891420CD9FC
S22402122000F01AFC286846702046BDE8704000F097BC064800F0BCF8F7E766702146BDE8AB
S2240212407040024800F0ECBBD8C80720941708200321FFF763BF0000054A02EB810151F819
S224021260041C002902D00A8B82430A83704700001C12082010B50446008B084320836278F6
S224021280618B062A18D0052A19D1084217D001EA0002628388432083204600F008FC01203E
S2240212A06070628B0821204600F0FDFB2146BDE81040034800F0B4BB31EA0002EAD010BD49
S2240212C0941708200246154810B500EB810050F8044C002C21D0208B104320836278618B42
S2240212E0062A17D0052A18D1084216D001EA0002628388432083204600F0D9FB012060702D
S224021300628B0821204600F0CEFB2046BDE81040FFF77CBF31EA0002EBD010BD1C1208200A
S22402132070B503460C480D460468208B42B133EA000101D0062109E098432083022070BDBB
S22402134010EA030101D06183F6E7052163832846FFF7E4FE012070BDD8C80720814202D3F7
S22402136042688A4201D80120704702680A60BFF35F8F50E8003F0A689A42F6D140E8001205
S224021380002AF2D10020704768B161B10022083902E00246006830B18842FAD12AB10068A9
S2240213A01060002070470120704700214160F8E70146406842684A600B780022022B05D07C
S2240213C0012B03D0032B01D04260704743680BB19960426082607047810700D000207047E5
S2240213E070B5044600201546207001226270A17084F824106060A060E06020612062A08291
S224021400E0822083608384F82500E08C18B90548FFF758FEE06229462046BDE8704000F00A
S2240214201DB8000088E0072008B1082901D2012070470144091F002201600A60426010465A
S2240214407047000003480021016003490988C18070470000E4C80720843A020070B5C28C26
S2240214601C4D930802D12A88C2F38D03C26A02EB8302540700D5121F4FF0807442E9021424
S22402148000242646B2F1400242F82460641C0E2CFAD3C4691462826201632968C90014D55D
S2240214A0112B12D94FF0FF31103B11EB53014FF0CC3305D042F8043C42F8083D491EF9D1B7
S2240214C0C16A121F8A4200D91360C06A0249016070BD0000803A0200A52E5AE2C189808970
S2240214E0081A704701220270002242708270426002814281103982818908C18170470000F3
S2240215002DE9F041044640680E464FF0000804F10C05E8B36078012701283ED0022813D00B
S22402152003285CD10846FFF7CDFD050057D02046FFF73EFF0446294600F0B2FA67702046E7
S22402154000F0B5FA214621E02046FFF731FF0646002100F0A5FA2189F06904EB8101086118
S224021560D5E85F0F401C81B2C5E8501F0028F7D12089401C80B22081E189884201D1A4F824
S22402158008807770304600F092FA3146174800E00CE0BDE8F04100F043BA2046FFF708FF1B
S2240215A004463246102100F07EFAC7E7A089E189884216D2208904EB80000661D5E85F0F2C
S2240215C0401C81B2C5E8501F0028F7D12089401C80B22081E189884201D1A4F80880BDE8C2
S2240215E0F081BDE8F0410320FEF7ACB89417082070B5164642680D4612B1417801290BD04F
S2240216008189C4890023A14224D19EB11D4C216892B100F005FA16E0FFF7CAFE04462A4690
S224021620102100F040FA204600F041FA2046FFF7EDFD25E0012070BD416021684B602168C0
S22402164088600221417020680821C5613046FFF765FDEFE7018900EB81010D6100F10C01E9
S224021660D1E85F2F521C94B2C1E8524F002AF7D10189491C89B20181C289914200D103810D
S224021680002070BDD8C8072070B50446808915460026C0B3608904EB8000006908606089B1
S2240216A0401C80B26081E189884200D16681606810B1607802280BD014F10C04D4E85F0F23
S2240216C0401E81B2C4E8501F0028F7D1002070BD2046FFF76DFE0546002100F0E1F9218973
S2240216E0E86904EB810108612089401C80B22081E189884200D12681284600F0D8F9284697
S224021700FFF784FDE2E7FFE73DB10B48626801682AB1204600F084F908E0012070BD616083
S22402172001684E60006884600120607008212846FFF7F4FCF1E70000D8C80720002814D026
S224021740411C13D00C4A4FF6FE7190420CD800EB4002C2EBC0120948036803EBC202521EF8
S224021760B2FBF3F0884204D9084670474FF6FF70704780B27047000000093D00A03A0200B0
S224021780032101700021418041608160C16070472DE9F0410446408820B1314DA1682A682E
S2240217A0914202D0FF20BDE8F081401E0004000C608053D12968086AA04209D1E068086265
S2240217C008E0C268A24202D1E268C26002E010460028F6D191F824000A6A06E053681BB118
S2240217E09B78834200D91846D268002AF6D18870DFF870806168012611B32046FFF7D8FD04
S2240218000746002100F04CF9384600F050F96680A760386AE0603C622968D8F804008A7893
S2240218208078824201D3384616E00E4800F0F8F839460C4800F0F4F8286846707E700AE09A
S224021840D8F804108A782968824207D9054800F0E7F8286846700020FFF7D8FC0020A2E771
S224021860D8C807209417082070B51C4D0E4604464188286861B1A268824210D1A1F57F402C
S224021880FF3803D0491C6180002070BDFF2070BDA060016AE160046201206080F4E776B143
S2240218A091788078814203D29070A06800F0DEF8606830B12046296800F0B2F808E0012077
S2240218C070BD286860602968002048602868846009213046FFF722FCF1E70000D8C8072064
S2240218E070B51B48012102685170006800F0B4F8184D6C7818E000BF05EBC4014868027829
S224021900EAB1012A20D000F0FFF8E878641C844200D100240F48801CD0E84F1F491EC9B28D
S224021920C0E8421F002AF7D1A8780028E4D16C700948FFF73DFDBDE8704000F011B90989AA
S22402194089B2FFF797FCE0E78968FFF7D9FDDCE7D8C8072098110820941708200548017844
S22402196011B101214170704703494FF080500860704700005804001004ED00E0F0B4154D57
S224021980AB1CEE784FEA0507D3E84F2FB24202D1BFF32F8F11E0521CD4B2C3E8424F002A13
S2240219A0F2D100BFD7E84F2F541CB44200D10024E4B2C7E8434F002BF4D1EB78934205D929
S2240219C005EBC202C2E90101F0BC7047F0BC0220FDF7B8BE98110820104A10B5D368ABB17D
S2240219E013469B8A03E08CB12246A48A2344D4688B42F8D3C460D0600261C46804B1206158
S224021A00591A8182908A401A908210BD0024C460D060C91A02619182848210BDAC17082067
S224021A2030B502780023022A03D0012A01D0032A00D101238C7800E01046426812B195784C
S224021A40A542F9D24A6041601BB102B19160886030BD0020FBE7000003494A684260002279
S224021A6082604860704700009417082010B5836804462BB9607801280ED1084B03E09B6854
S224021A8018780028FBD0204600F026F82146BDE810401846FFF7C4BF10BD00009417082075
S224021AA0806A01627047806AC0E90812704710B5016900290ED0C268CA60C36800223BB1F4
S224021AC08B8A848A23448B82C3681961C26000E08A82026110BD0000816839B142684A605E
S224021AE04168002901D0806888607047054906E04A68824202D140684860704711460029B1
S224021B00F6D170479417082010B5416881B1FFF74FFC0446FFF7CBFF0120607001462046E4
S224021B20FFF7BEFF2146BDE810400348FFF778BF4188491C418010BD9417082006480068D2
S224021B40D0E90A10814203D300680449884202D00120FDF7F7BD7047D8C80720A52E5AE26B
S224021B600749022248604270064A1278002A05D006C98A4202D0C078FFF794B87047000019
S224021B80D8C80720ECC8072070B5FFF763F800200446204A204902E042F82040401C0B887E
S224021BA09842F9D31D48342201881D48FEF71EFF1C48008880B240F000421B4801681B48FE
S224021BC0FEF714FF1A48082201881A480068FEF70DFF194DFF20194AE870EC8400212846D7
S224021BE0FFF7FEFB164804210170446015480170C4600461848214481549056002206870E1
S224021C001248047044700978C170BDE87040FFF719BC00001C1208207C3A0200A83A020077
S224021C2070DE0720803A0200AC3A020088E00720D03A0200D0C80720E851001041F70100A8
S224021C4094170820AC170820D8C8072098110820B43A02001B4810B5016841F47F01016090
S224021C6000684FF07F4101EA00201649C0431439B0FA80F00968C0F10800C1F3022181425E
S224021C8000D3481C0F49091F0B686FF08072824063F317020A60FFF7EDF90B490028086067
S224021CA00EDB00F1E021FF2281F8002400F01F02012191404009800000F1E020C0F80011FD
S224021CC010BD000020ED00E05C0400100C4810B50268012151700068FFF7BEFEFFF73AFA29
S224021CE008480168491C0160FFF758FA00F0FCFB0548FFF75DFBBDE81040FFF731BF0000B9
S224021D00D8C80720E0C8072094170820002805D0810702D10178002900D0002070470000B2
S224021D2030B50B4C0023626805E095688D4204D813461268491B002AF7D10260816012B1B7
S224021D409568691A91600BB1186030BD606030BD500400100D4B0022596803E0814204D024
S224021D600A4609680029F9D104E019B1016822B1116003E04FF0FF3070475960016819B159
S224021D808A6880681044886000207047500400102DE9F0411E46174680460D4611F0FF0FBB
S224021DA000D14D1C1848FFF78DF9041E16D0280AE762E084E9B242462046E661FFF710FB4E
S224021DC001251248124905E000EB850252F8042C32B16D1C0A889542F6D90020BDE8F08176
S224021DE0002DFAD000EB850040F8044C0948E570007818B101212046FEF744FF2046FFF7EA
S224021E0005FA2846EAE7000070DE07201C1208207C3A0200ECC807202DE9F05F584DDFF83E
S224021E205891DFF8588129684FF0010A002618B1CA78AB46824243D14E70EEF764FA29689B
S224021E408862FFF77BFE2868046A1FE06068C0B12046FFF7ADFA07460021FFF721FE3846E8
S224021E60FFF725FE87F801A039464648FFF7D8FDE168A4F802A0A760386AE0603C620C46EA
S224021E8004E0E0686680A660E6600446002CDDD12868C27808EB820141F8046CC16A3A4823
S224021EA0FFF75CFA2868C66299F8001011B10021FEF7E8FE35482968FFF750FA2E6056E0A6
S224021EC03349098888420CD808EB800858F8045C3DB12846FFF700FE2846FFF7E8FD2C6AE6
S224021EE022E0FF20BDE8F09F6068C0B12046FFF75FFA07460021FFF7D3FD3846FFF7D7FD1C
S224021F0087F801A039461F48FFF78AFDE168A4F802A0A760386AE0603C620C4604E0E068AB
S224021F206680A660E6600446002CDDD148F8046C1548E96AFFF712FAEE6299F8000018B138
S224021F4000212846FEF79EFE29461048FFF706FA0C48DBF8001040688B7882789A4209D903
S224021F6081F801A00748DBF80010FFF759FD0020FFF74CF90020B5E7ECC807201C1208207A
S224021F80D8C807209417082088E0072070DE07207C3A020070B51A4D80B11A4A1288904257
S224021FA01FD8194A02EB800050F8044CCCB1A17084F824102868A04205D014E028688170C1
S224021FC0286880F82410114840688078884215D90E482968FFF724FD296801204870002085
S224021FE00AE0FF2070BD2046FFF740FD6078012804D10648FFF7DCF9FFF708F9002070BDD8
S224022000D8C807207C3A02001C1208209417082002480068002800D0C0787047D8C80720B1
S22402202010B5002804D0FFF789FBFFF711F9402010BD000010B5134C207860B912484007BB
S22402204005D1124801681048FFF7EEF908B1852010BDFFF799FD0E49FF200968887020787D
S22402206058B900210B4800F07EF80B49086000210A4800F011F90A490860012020700020B9
S224022080607010BD5004001098E40720B03A0200D8C80720C83A0200C8C80720B83A020033
S2240220A0C4C8072070B50F4D687808B1002070BD0D4C206890F824100020FFF76BFF20685A
S2240220C0C178FF2903D1816A203181F30988616811B9606000202060FFF7BCFD01206870E8
S2240220E0E4E7000050040010D8C8072070B5FEF7DFFF0446FEF7D4FF0849094E0D686D1C33
S22402210048B1FEF7D5FFA04200D204463068401C05FB004070BD3068FAE70000903A020052
S224022120E0C8072070B504000BD0216849B162683AB1A06828B1D0E9005010B10DB12B7881
S2240221400BB1002070BDD21C22F0030251430C31FEF74CFC20888000103081B22846FFF75D
S224022160C1F9A06870BD10B5040005D0216819B1606808B102780AB1002010BD890010310B
S22402218089B2FFF7AFF9606810BD3EB504000D464FF0800012D0217801290FD12846FFF7D8
S2240221A0CDFA0246204601A9FFF76EFA012801D0102003E00DB1402000E00020DDE9011297
S2240221C003B030BD70B50E460400154602D02078012801D0802070BD1046FFF7AFFA024612
S2240221E031462046FFF704FA012801D0002070BD0DB1C12070BD812070BD70B50C46FFF7B9
S22402220085FD4FF0004108B1220C01D0084670BD058BC178A0B2FFF71FF8284670BD70B59A
S2240222200C46FFF773FD4FF0004108B1220C01D0084670BD058BC178A0B2FFF743F8284672
S22402224070BD000070B504460D46000C01D086201EE008462CB1FFF771FA0146A0B20122BF
S22402226005E0FFF76BFA014600224FF6FF70FFF757F8022802D04DB1402008E008200CB18E
S224022280214605E003490968498B01E000200021324670BDD8C8072070B50E46040029D056
S2240222A0206838B3606810F1030F23DB032821DCE16829B11048FEF712FF05001AD000E053
S2240222C000256068E168001D40EA012133462A462068FFF75DFD40B1084901EB8000084998
S2240222E050F8040C826A516370BD1DB129460248FFF74AF8002070BD98E407201C120820AD
S224022300B10F020010B5FFF783FE002804D0034901EB800050F8040C10BD00001C12082089
S22402232010B5FFF7F3FC18B1C18C19B1C46A02E0802010BD0024C078FFF76EFDFF2806D0D5
S2240223401CB121460348FFF71FF8002010BD812010BD000098E4072010B5FFF73DF820B12B
S22402236041690A680169104610BD0020014610BD10B503000CD0186850B15868002808D094
S22402238009B1012904D1074C24680CB104790CB1002010BD00240460012404714171C0E93D
S2240223A0042310BDC4C8072070B50E46FFF714F8040016D0BEB1144A00214FF47A73106874
S2240223C01268401E41F1FF35E6FB030529460023FDF712FD0546207901280CD0022808D14E
S2240223E003E0802070BD862070BD2046FFF7B2FC20B1812070BD02202071E56029462046DD
S224022400FFF78EFC002070BDA03A020010B5FEF7E3FF18B10179022908D101E0802010BDDB
S22402242001210171FFF796FC0028F8D0812010BD70B50D46002806D0D0E9004010B10CB12E
S22402244012B10DB1002070BDFEF73CFE060017D1B5B10C4861680029016803D02046FFF746
S224022460DFFA07E0616002680021516000688460032060702846FFF761F90821FEF74EFE31
S224022480304670BDD8C8072070B5164648B1D0E9004534B12DB12846FEF760FF18B186205F
S2240224A070BD802070BD6068E0B16078032819D136B129462046FFF761FAFFF74FFA11E098
S2240224C02846FEF7FFFD05000CD02046FEF770FF04462946FFF7E4FA2046FFF7E8FA2046BA
S2240224E0FEF794FE002070BD2DE9F041134E7468002C1CD0A068124F401E4FF00108A06056
S22402250012E0254624687460002229463868FEF7E6FB10B10420FDF715F96879012808D027
S22402252085F80480002C02D0A0680028E9D0BDE8F0812846E968FFF7F3FBF3E750040010B5
S224022540C8C8072010B5164B21F00042012486B09A4203DC0022134600941CE0114B9A42EB
S22402256008D140B94FF00100FDF7CEFDFEF72FFA06B010BD03DBFEF727FA06B010BD02AABF
S224022580FDF7CAFE00F00100A4EB40000DF1080C00909CE80F00FEF7D9F806B010BD00003A
S2240225A0FB21E93F0000F07F21F00042A2F16052B2F5801F01F0004328BFD2F17F6C0BD9D6
S2240225C05FEA001C43EAC20242EB507018BF704728BF20F001007047B2F5801FBCBF184655
S2240225E070474FEA410C1CF5001F02D2084600F0CEBF70B500F08CFB00000089FFF7F6BFF8
S2240226004FF00040A0F580007047000010B591EA030F48BF83F0004300F11884841A71EBD2
S224022620030C05D2121943EB0C03001B61EB0C01DFF824E14FEA1154A4EB135C1EEA430FFF
S22402264018BF9EEA445F73D023EA0E03DCF1200E21EA045143F4801332D322FA0CFE10EBC5
S2240226600E0023FA0CFE41EB0E01CCF1200E03FA0EFE10EB0E0051F10001B1F5801FCCF1A1
S224022680200E32D201EB045112FA0EF2BDE8104058BF7047401C38BF5FEA420218BF704783
S2240226A0002814BF20F0010041F100014FEA410313F5001F38BF7047A1F1C04100F076BBCE
S2240226C0012A43EB0302ACF1200CDCF11F0E32BF4FF0000E23FA0CF310EB030041EB0451F9
S2240226E0B4EB115FD0D0A1EB045101F5801149085FEA300001EB04510ED350F1000038BF98
S22402270012FA0EFE08D1BDE81040C9E7401C38BF5FEA4202CAD1C3E7BDE810404FEA410385
S22402272013F5001F38BF7047A1F1C04100F03EBB9EEA445F08D011EA5E0FBDE8104004BF1E
S22402274001F0004100207047BDE8104070B500F0DFFA00BF64FBBE3E0000E0FF02494FF003
S224022760000000F0CABF00BF0000F87F491058BFC1F140415B1058BFC3F140438B42EFF398
S224022780008070472DE9C04130B4DFF8A0C23CEA111418BF3CEA131400F0EC8081EA030589
S2240227A01CEA111444EAD57418BF1CEA131500F0C780A4EB05044FF0004545EAC12145EAD8
S2240227C0C32341EA505143EA525304F17F74994204F500344FEAC0204FEAC22208BF9042AF
S2240227E000F09C804FEA13650FF24016765D4FEA134506FB05F7C7F1807706FB07F74FEA76
S224022800D737A7FB03687642C8F58038A7FB06CE38BFA8F1010807FB08E64FF0000EA6FB7C
S224022820028CE6FB03CEDCF1000CCEF1004E38BFAEF1010EA6FB0C584FF000074FF0000537
S224022840E6FB0E87A1FB08C6A0FB07CE16EB0E0645F10005E1FB076515F1E04E7EBFA4F57F
S22402286080345FEA46066D4116F1800745F100054FEA17274FEA066647EA0567A6F1DE461D
S224022880B6F1805F4FEA15251FD9384624F0010C05EBC471BCF1FE6F01EB0C1102D8F0BCD3
S2240228A0BDE8008124425CBF01F5801E9EEAC47F02D4F0BCBDE80081244238D4F0BCA1F1B3
S2240228C0C041BDE8004100F071BA4FEAD22242EA43524FEAD323A7FB02864FEAD02040EA55
S2240228E0415007FB03661EEA0E0F4FEAD12105FB026658BFA6EB0056B6EB00564FEA520E8F
S2240229004EEAC37E18EB0E0E56EB530EBDD518EB02085E417F1C55F10005B6E74FF48015DD
S2240229204FF000074FF000064FF00008ADE7F0BC4FF0000001F1C04101F00041BDE80081F4
S22402294011EA0C1F0CEA131500D00CE013EA0C1F00F025804FF00000F0BC81EA030101F068
S2240229600041BDE80081F0BCBDE8004181EA030100F01CBAF0BCBDE8004170B500F0C8F9BA
S224022980097EFC3E00F007B881EA03014FF0000001F00041704781EA030100F007BAF0BC5D
S2240229A0BDE800414FF0000021497047FFFDFBF9F7F5F4F2F0EEEDEBE9E8E6E4E3E1E0DE35
S2240229C0DDDBDAD8D7D5D4D3D1D0CFCDCCCBCAC8C7C6C5C4C2C1C0BFBEBDBCBBBAB9B8B7E1
S2240229E0B6B5B4B3B2B1B0AFAEADACABAAA9A8A8A7A6A5A4A3A3A2A1A09F9F9E9D9C9C9BDC
S224022A009A9999989797969595949393929191908F8F8E8E8D8C8C8B8B8A898988888787B0
S224022A208685858484838382828181800000FF070000F87F4FEA41034FEA5353A3F5806317
S224022A40D3F11E03C8BFD3F1210C0CDD4FF0004242EAC12242EA505232FA03FC8CEAE17CCD
S224022A60ACEBE1707047102BC4BF0020704703F5787CBCF1FF3F04D06FF0004282EA210042
S224022A80704770B500F044F94992248000207047F2E700004FEA1153A3F58063D3F11E03FA
S224022AA0A8BFD3F1200C08DB4FF0004242EAC12252EA505232FA03F0704709420BD4102B2C
S224022AC0C4BF0020704703F5787CBCF1FF3F05D04FF0FF3070474FF00000704770B500F0B9
S224022AE017F900BF4992248000207047F0E710F0004248BF4042B0FA80F310FA03F10AD013
S224022B00C3F11D0303F580634FEA415002EB035202EBD12170474FF000007047B0FA80F34A
S224022B2010FA03F10AD0C3F11D0303F580634FEA41504FEA035202EBD12170474FF00000DA
S224022B407047000051EA030C17D41CF5801F58BFBCF5801F00F10680994218BF704708BFC4
S224022B609042704707D711F5801F58BF13F5801F19D499427047894270471CF5801F08D5F6
S224022B80BCF5801FF7D58B4218BF704708BF824270474FF4001C1CEB410F38BF1CEB430F6F
S224022BA001D28B42704770B500F0B2F8922449004FF000514FF08053FFF7D8BDDFF848C1EC
S224022BC070B51CEA111E1EBF1CEA13159EEA0C0F95EA0C0F00F06F8081EA030423EA4C138F
S224022BE04EEAD47E21EA4C1141F4801143F48013AE44A1FB024CA0FB0365AEF17F7E361982
S224022C0055EB0C05A1FB034C4CF10003A0FB021C16EB0C06654153F10003094218BF46F020
S224022C20010613F4007F0BD14FEA03314FEA0530340341EA155140EA16506FF003020AE0A3
S224022C404FEAC3214FEAC520F40241EA555140EA56506FF0020202EB2E4201EB025585EA29
S224022C60CE710AD05FEA440C18BF24F0004450F1000041F1000120EAD47040F2FE7C624557
S224022C8000D270BDA84214BF4FF080444FF04044002E08BF0024BEF1806FA8BFA1F1C041FA
S224022CA0BDE8704080F282804FF0000001F1C04101F0004170479EEA0C0F0CEA131518BF91
S224022CC095EA0C0F06D04FF0000081EA030E0EF0004170BD00F01CF88900013E00F007B8DB
S224022CE000F009B84FEA430C5FEA5C5C08D081EA030100F05BB84FEA410C5FEA5C5CF6D1FB
S224022D004FF00000014970470000FF070000F87F0EF1020E2EF0030E5EF8046B364205D49B
S224022D20012A43EB030515F5001F12D8012841EB010C1CF5001F0CD80ED14FEAD17C15F533
S224022D40001F0CEB4C0C0CF1020C08BF4CEBD37C04E04FF0080C01E04FEAD37C0CEB4C05BE
S224022D6026FA05F606F00706B6F1040C06D20EEB860CBDE870404CF0010C6047DFE80CF00C
S224022D80090B02024FF000414FF00000A1F5002170BD19461046012851EB010418BFD4F5B2
S224022DA0001484BF002001F0004170BD0808A0F500114FEA3101704753EA010C17D41CF518
S224022DC0801F58BFBCF5801F00F106808B4218BF704708BF8242704707D713F5801F58BF36
S224022DE011F5801F19D48B4270479B4270471CF5801F08D5BCF5801FF7D5994218BF704710
S224022E0008BF904270474FF4001C1CEB430F38BF1CEB410F01D2994270470FB40CBC03BCA6
S224022E20FFF7C1BE91EA030F10B581F000413FF5F5AB83F0004300F009B8000010B591EA97
S224022E40030F48BF83F000433FF5E8AB841A71EB030C07D212198CF0004C43EB0C03001BA8
S224022E6061EB0C01DFF8A4E14FEA1154A4EB135C1EEA430F18BF9EEA445F00F0B08023EA71
S224022E806E03524221EA0451C3EB6E0338BF5B1EDCF1200E25D322FA0CFE10EB0E0043FAD8
S224022EA00CFE41EB0E01CCF1200E03FA0EFE10EB0E0051F10001CCF1200E29D412FA0EF292
S224022EC001EB0451BDE8104058BF7047401C1CBFB2F1004F704700280CBF491C20F001009E
S224022EE0704712EB020E43EB030218BF4FF0010E4EEA4202ACF1200CDCF11E0E54D943FA07
S224022F000CFE10EB0E0051F1FF31CCF11E0ED5D50EF1010E12FA0EFE404141EB010101EBD1
S224022F20445C5FEA5C5C10D910EBDE7001EB045138BFBEF1004FBDE8104018BF70470028D6
S224022F400CBF491C20F00100704730D24FEAD42C11F5001124F400641BD0B1FA81F20B3A56
S224022F60A41AA41ED2F12003914030FA03F31943904001EBCC71002C01EB0451BDE810403C
S224022F80A8BF704701F1C0414FF0000001F000417047B0FA80F310FA03F100D110BDE41A3A
S224022FA0173C4805C90AE4E701EB045110BD491001EB0451BDE810404FEA300002E04FF0A5
S224022FC0000170474A0008BF0042F8D0B2F5001F28BF704701F000414FF0000070479EEA03
S224022FE0445F07D011EA5E0FBDE8104004BF002100207047BDE8104070B5FFF789FE00BFE2
S22402300040DFF63E83F00041104670470000E0FF43004FEAD30C4FEA3C0C43401FBF400732
S2240230200CF1605113F0FE4F70471CF0006F03D100200CF0004170470CF0004343EA507045
S22402304010B540EACC0000F05CFA00BF000000924FEA0001FFF7AABE4FF000414FF00000C0
S224023060A1F500217047000090EA010F48BF81F0004100F1D482421A3CBF801A89184FEA86
S224023080D0524FF07F4C1CEA410FA2EBD15318BF9CEA026F00F03B804FF0004C4CEA00209C
S2240230A04CEA012121FA03FC10EB0C0C1ED202F1FF325FEA1C2040EBC25038BF70471CF0F4
S2240230C07F0F4FEA400C18BFBCF17F4F38BF7047C3F12003994008BF20F00100BCF17F4FD3
S2240230E038BF7047A0F1C04000F051BA4FEA3C00000A40EBC25028BF1CF0FF0F4FEA400C4D
S224023100E6D018BFBCF17F4F38BF7047EAE79CEA026F05D010EA5C0F08BF00F00040704742
S22402312010B500F0EEF900BF64FBBE3E401058BFC0F14040491058BFC1F140418142EFF3F2
S224023140008070474FF47F0C1CEAD0121EBF1CEAD11392EA0C0F93EA0C0F00F0858090EA16
S224023160010F48BF42F4807240F4000C41F400002CF07F4120F07F4000B58142A2EB0302DF
S2240231800FF2081CACEB504EC0F100009EF800E04FEA4E0E00FB0EFC38BF49004FEA2C1C4C
S2240231A002F5FA020CFB0EF34FEACE1E4FEA112C4FEAC1210EEB635E42EB22420EFB0CFCFB
S2240231C04FEA1C5300FB03114FEA112C4FEA01310EFB0CFC4FEADC4C00FB0C11C14228BFDC
S2240231E009184CEB03335DF804EB10EB410143EBC250B2F57C0F38BF704729D512F0F00F9A
S2240232001CBF00F1C04000F000407047008182838485868788898B8C8D8E8F9192939596A5
S22402322097999A9C9D9FA0A2A3A5A7A8AAACAEB0B2B3B5B7B9BCBEC0C2C5C7C9CCCED1D43E
S224023240D7D9DCDFE2E6E9ECF0F3F7FAFE0000004FEA400C0CF1807CBCF17E4F28BF7047F7
S224023260B0F1C04000F093B990EA010F0CEAD11348BF42F48072624538BF634507D213F4B1
S2240232807F0F16D080EA010000F00040704710B500F037F9097EFC3E00F005B880EA0100A3
S2240232A000F00040704780EA010000F0004000F06EB912F47F0F04BF0248704780EA0100AB
S2240232C000F065B90000C07F41000B0ED3F19E0208D950F400034FEA032323FA02F048BF3F
S2240232E04042704710B500F00CF900BF49922480002070476FF0004282EA200070470000DB
S224023300C10DD1F19E0206DB4FEA002343F0004323FA02F07047004207D54FEA4001B1F1C3
S224023320FE4F02D24FF00000704710B500F0E9F849922480002070476FEA20007047000053
S22402334010F0004148BF4042B0FA80F310FA03F2C3F19D030BD051EAC35101EB122053068B
S22402336038BF704700F1010008BF20F001007047B0FA80F310FA03F2C3F19D030AD0D905EF
S22402338001EB1220530638BF704700F1010008BF20F001007047000050EA010C00F11380B5
S2240233A01CF5000F58BFBCF5000F01D48842704707D710F5000F58BF11F5000F15D48842E8
S2240233C07047894270471CF5000F04D5BCF5000FF7D5814270474FF0807C1CEB400F38BF26
S2240233E01CEB410F01D28142704710B500F089F8922449004FF000504FF08051FFF796BE04
S2240234004FF47F0C1CEAD0121EBF1CEAD11392EA0C0F93EA0C0F00F0478090EA010F48BFB1
S22402342042F480724FF0004C4CEA00204CEA012102EB0302A0FB0113A2F50002002918BFEA
S22402344043F001035B0028BF4FEA330342EB22425FEA132C4CEBC2502EBFBCEB436FB2F52E
S2240234607C0F70474FEA036CBCF1004F08BF20F00100B2F57C0F38BF70470BD582F0FF0254
S22402348012F5803FC8BF704700F1C040D8BF00F00040704700F5000C5FEA4C0C48BF704752
S2240234A0B0F1C04000F073B890EA010F0CEAD11348BF42F48072624538BF634504D280EA30
S2240234C0010000F00040704710B500F01AF800BF8900013E00F007B800F009B85FEA410CB9
S2240234E05FEA1C6C08D080EA010000F050B85FEA400C5FEA1C6CF6D14FF00040A0F58000F8
S22402350070470EF1020E2EF0030E5EF8044B244204D44FEA4102B2F17F4F11D84FEA40037A
S224023520B3F17F4F0CD80ED14FEAD07CB2F17F4F0CEB4C0C0CF1020C08BF4CEBD17C04E0D0
S2240235404FF0080C01E04FEAD17C0CEB4C0324FA03F404F00704B4F1040C06D20EEB840C3A
S224023560BDE810404CF0010C6047DFE80CF0070802024FF00040A0F5800010BD0846420098
S22402358018BFD2F1807288BF00F0004010BDFF2141EAD050C005704751EA000C00F11380A2
S2240235A01CF5000F58BFBCF5000F01D48142704707D711F5000F58BF10F5000F15D48142F4
S2240235C07047894270471CF5000F04D5BCF5000FF7D5884270474FF0807C1CEB410F38BF1C
S2240235E01CEB400F01D28842704780EA010081EA000180EA0100FFF7F8BE80F0004090EA02
S224023600010F7FF538AD81F0004100F008B8000090EA010F48BF81F000413FF52CAD421A2C
S22402362004D882F00042A0EB020011444FEAD0524FF07F4C1CEA410FA2EBD15318BF9CEA48
S224023640026F4AD04FF0004C4CEA00204CEA012121FA03FCB0EB0C0C0FD412F0FE0F36D0DA
S2240236605FEA4C001DD5001240EBC25038BF70471CF03F0F18BF70470BE0A2F101025FEA0D
S2240236801C2040EBC25038BF70471CF07F0F18BF7047C3F12003994014BF401E20F00100E2
S2240236A0704780084FEA122308BF7047B0FA80FCA2EB0C02CCF1280C60FA0CF093EA122F12
S2240236C004BF00EBC25070474FEAC3707047130A5FEADC1008BF7047F6E79CEA026F04D0D1
S2240236E010EA5C0F08BF0020704710B5FFF709FF40DFF63E81F0004070470CF00F03092B00
S22402370008BF082000F059800A2B0BD0082B18BF704708BF1CF0400F0AD04FF000004FF09F
S224023720000170471CF0400F18BF4FF0004070471CF0100F08D020F0704300F07F4242EABF
S224023740D3014FEA4370704700F0604021F07F4242EA000201F07F4040EA727070474FF0A9
S224023760FF0C4CF4E06C1CEA11531CBF9CEA030C9445C2BFDA4201EB02517047002B0DD05D
S224023780BCF1000F0FD0002A01F00041A4BF41F0E04141F07F614FF00000704701F000413D
S2240237A04FF00000704750EA01334FF09B0C18BF4CF0806C7EF4D2AF70471CF4801F11D07F
S2240237C01CF4E02F03D06FEACC31490070474FF04050EFF3008222F0704242EA000282F300
S2240237E0008870474FF000007047000049050100F0C807207505010008C90720C505010021
S22402380020C9072000400440008004408813DC05DC05581B581B0000A000BC02D5010000D2
S2240238200E01B4000000000040787D01E803000080969800B80B000048F4FFFF0000011ED3
S2240238400100000200024A0101003203021400000000C8420000C8420000ECFF88FF38FF08
S22402386014007800C800A000BC02D501001E00000000F401FA00FA00FA00000013000000A5
S2240238800000000707010000D0121300E0930400204E000032000000CEFFFFFF0000C84231
S2240238A00000C8426400FA006400FA00000000000000AF00A00000000000C03F0A00E803F8
S2240238C0004106040319881388130002030000008613060000512502E8030000809FD50049
S2240238E0B80B000048F4FFFF8A130000A0252600E803000040420F00B80B000048F4FFFFC3
S22402390006006400FA001A000600000025450100000000000100000000040000100000009C
S22402392004000000D00200101345010098CE072023450100B0CE072023480100000000003A
S22402394001000000000400000100000002000000F4020010C3470100A4080010B74901008A
S224023960180900104B4A010030090010E951010000000000010000000004000000190018BF
S2240239800017011EC3580100000000000100000000020000B35801001CD00720075A01004A
S2240239A06CD00720596201000000000001000000000400003762010084D00720476201001D
S2240239C09CD007205F64010000000000010000000004000085000000100000005403001088
S2240239E085000000100000005C03001085000000100000006403001085000000100000001B
S224023A006C03001003680100000000000100000000020000F3670100B4DC072021007611F7
S224023A2049000000BF870100C8330010F9870100E03300107FBB01004051001079BC01002E
S224023A40585100109BBD010054DE072081CD010070510010E1CB0100DBCC01001BCD010096
S224023A6029CD0100D1D1010088510010EDCE010051D0010045D1010053D101000A00000098
S224023A8000040A0105000100C06878044B000000F7240100010000000200010052000400A5
S224023AA0E8030000000000001402000010040000002D000010000000491002000200000050
S224023AC001000000900100002000000044120820000000005D02010000000000010000004E
S224023AE000040000000000004FBB610567ACDD3F182D4454FB21E93F9BF681D20B73EF3F6B
S224023B00182D4454FB21F93FE2652F227F2B7A3C075C143326A6813CBDCBF07A8807703C15
S224023B20075C143326A6913CC4EB98999999C9BF711623FEC671BCBF6D9A74AFF2B0B3BF09
S224023B409AFDDE522DDEADBF2F6C6A2C44B4A2BF0D5555555555D53FFF8300922449C23F4A
S224023B606E204CC5CD45B73F513DD0A0660DB13FEB0D76244B7BA93F11DA22E33AAD903F50
S224023B8000004054FB21F93F3163621A61B4D03D0000601A61B4D03D7370032E8A19A33BD3
S224023BA00000002E8A19A33BC14920259A837B3900000000000000006E83F9A22915444ED3
S224023BC0D15727FCC0DD34F5999562DB4190433CAB6351FE61C5BBDE3A6E24B7E0D24D4232
S224023BE0EA2E49061C92D1091CEB1DFE3EA729B1F53582E88444BB2E26709CE9417E5FB4BC
S224023C0039D69139F43953838B5F849C3B28F9BDFF97F81F0F9805DE8B112FEF1F6D0A5ABD
S224023C20CF7E366DB709CB27663F464F2DEA5F9EC7BA27757BF1E5EBF739073DEA92528A68
S224023C40B15FFB6B085D8D1F7AFE10111111C13F37D60684F464963F280356C9226D6D3FD2
S224023C600165F2F2D844433FA69237A0887E143F735360DBCB75F3BEFE41B31BBAA1AB3FA9
S224023C8093846EE9E326823F1583E0FEC8DB573F68108D1AF726303FE9A7F0320FB8123FC1
S224023CA0D47ABF74702AFB3EE83C02000002001060020000080101008C3D020000C0072053
S224023CC0F0080000080101008C3D020060040010C05D000064010100C8400200F0C8072030
S224023CE0385F00006401010061120103170908220114372601147F2A0114392C0114B72B5E
S224023D00011AA7040114140D54011A1304C11A3D341A4104411ACD381AE3045A2D101A530A
S224023D20081AA1581A63081A69041A6F04146B23011A73082511C7BA3C0B14803F6A011A3A
S224023D408009FCCD07204CCE07200213021380081B109404015813480914106C0B1410C8E9
S224023D60131410EC151C10481E101A20101A28100A1C2A781401400613350C13FFB1FBFF92
S224023D801F1C019F0510C068780400002301FA500870C907200201011AFF011A0214DA7416
S224023DA0141A0914DA6014111914DA5C141A300B2A78141189141A0A28DA7C281A320B1AE7
S224023DC08414120152042310271A33143A86147A02141A3414DA88141A3514DA8A141A36B9
S224023DE014DA8C141A37141A8E14214914297E1A38059A902823FF031A3914DA92141A3ADF
S224023E0014DA94141A3B14DA96501A3C05AA982822FF1A3D14DA9A141A3E14DA9C3C1A3F8C
S224023E20051AA0145A0214111DCA9A3B4014DAA4141A4114DAA8141A42141AAC145A0514C3
S224023E401440420F1A43145AB0141CC0BDF076211A64141AE4143A0672411CFA43650BDACD
S224023E60E8141A440B9AB4B4411A45149AB6B429511A46149AB714325A1A48143AB914526E
S224023E800432031A4A149ABA2829141A4C14DABB141A4E14DABC141A47149AB81429A61AA4
S224023EA049051B74CDB46A01B41CC8424B0BDA78141A4D0BDA7C141A4F0BDA80141A500B69
S224023EC09ABDB41909111A51141ABE146A01F0198D1A5514DAEC281A56141A7050114A0106
S224023EE028320C1A5714DAC6B41A5805DAC7141A59059AC81432FF1A5A14DAC9141A5B1469
S224023F00DACA141A5C14DACB141A5F141AD0145A0214111DCA9A3B6014DAD4141A6114DA38
S224023F20D8141A62141ADC145A05141440420F1A63145AE0142CC0BDF063111A76141AEE44
S224023F40142A04281A8078227F1A7914DAF0141A7714DAF2141A7A14DAF4141A7814DAF633
S224023F60141A7B14DAF8141A7C141AFA146A01F022031A7D14DAFC141A7E14DAFE141A7F7F
S224023F80141124CA07204914290F1A80059A0114325A1A81149A021432041A52141A04142A
S224023FA0A9501A5314DA06141A5414DA08141A8214DA0A141A8314DA0C141A6914AA0E145E
S224023FC022FF1A6A14DA10141A6B14DA1C141A6C14CB84CD141A6D14DA12281A6E14DA147D
S224023FE0141A6F141A18146A0314311A70141A1914214914190F111A71053A1A14290E49FD
S224024000061A72051A8678A9141A7305DA87141A7405DA1B501A8405DA1E141A66051A20E0
S224024020145A063C211CFA43670BDA24141A850B9A283C32641A8614DA29A01A87059A2ACC
S2240240401429DC1A880BDA2B141A890BDA2C3C1A8A059A2D1429641A8B0B1A2E146A013CC6
S22402406022031A8C0BDA303C1A8D05BA34B41CC8428E0B5A383C29161AFE791A8F095A3A2C
S224024080145A0A141A6814DA3C501A9005DA3D8C1A910B1A3E1412037A02C8021B631A0129
S2240240A0AC0119091A1C011BB20872807281728242835290A29132B022705A849C01373A0B
S20C0240C00139493E09364400AD
S2240300004055001025BA030047BA030049BA03004BBA03004DBA03004FBA03000000000029
S2240300200000000000000000000000006903030053BA030000000000E10303001D0403002E
S22403004059BA030059BA030059BA030059BA030059BA030059BA030059BA030059BA0300E8
S22403006059BA030059BA030059BA030059BA030059BA030059BA030059BA030059BA0300C8
S22403008059BA030059BA030059BA030059BA030059BA030059BA030059BA030059BA0300A8
S2240300A059BA030059BA030059BA030059BA030059BA030059BA030059BA030059BA030088
S2240300C059BA030059BA030059BA030000F002F800F06CF80AA090E8000C82448344AAF142
S2240300E00107DA4501D100F061F8AFF2090EBAE80F0013F0010F18BFFB1A43F001031847B8
S22403010048F2000088F200000A444FF0000C10F8013B13F0070408BF10F8014B1D1108BF28
S22403012010F8015B641E05D010F8016B641E01F8016BF9D113F0080F1EBF10F8014BAD1CC3
S2240301400C1B09D16D1E58BF01F801CBFAD505E014F8016B01F8016B6D1EF9D59142D6D3C9
S22403016070470000103A24BF78C878C1FAD8520724BF30C830C144BF04680C607047000091
S2240301800023002400250026103A28BF78C1FBD8520728BF30C148BF0B6070471FB59DE8D5
S2240301A003000BF089FF1FBD10B510BD0CF033F81146FFF7F3FF0FB400F00CF80FBC00F06B
S2240301C03DF80BF0A8FE03B4FFF7EEFF03BC0CF01BF8000004B00CF0FBFA044800210CF0CB
S2240301E0CFFB0CF007FB0BF096FE00009CF2030070B504461D4981F82C441D48407820F024
S224030200F00040301A4948700846407820F00F00C01C487005200870012C02D0022C08D1FF
S22403022003E000F001FA054603E002F048FB054600BF00BF284600F0F9F970BD70B50524F1
S2240302400CF0C6FA0220FFF7D3FF00F0F2F9456E284601F06AF8204601F01EF800F070FBD9
S22403026000F056F90CF0C6FA002070BD1803001000C0072070B50446B4F5E02F00D070BDF8
S2240302804FF480620D490E480BF077FE0D490B482C38C0F840120C4D72B62946204601F0B7
S2240302A06FFD00B1EBE74FF480620549204601F0C2FD00B1E3E762B600BFE0E7440300104E
S2240302C060C30720AA5555AAFF7F070064200CF073FA00BFBFF34F8F0648006800F4E06023
S2240302E005490843001D03490860BFF34F8F00BF00BFFEE70CED00E00000FA05FFFFFFFFC5
S22403030080F309887047EFF309807047684680F3098804480078C00714BF0220032080F330
S224030320148870475CF20300DFF818C0EFF305831B0618BF6047EFF31483DB0708BF604790
S22403034000DF7047D9CA0300DFF818C0EFF305831B0618BF6047EFF31483DB0708BF6047D8
S22403036000DF704771CD0300EFF30980816911F8021CF1B990E80F10E047EFF3098C8CE8CF
S2240303800700144B93E8060091420FD039B12CE9F00FC1F828C00CB40DF0DAF80CBC1A604C
S2240303A0D2F828C0BCE8F00F8CF309886FF0020E704710B5084A1268914209D8074C54F8C6
